:100000000C94D2140C94FD140C94FD140C94FD1457
:100010000C94FD140C94FD140C94FD140C94FD141C
:100020000C94FD140C94FD140C94FD140C94FD140C
:100030000C94FD140C9443500C94FD140C94FD147A
:100040000C94FD140C947C4F0C94D9C30C94FD14A7
:100050000C94CD4D0C94F74D0C94FD140C94FD14A0
:100060000C94FD140C94FD140C94FD140C94FD14CC
:100070000C94FD140C94FD140C94FD140C94FD14BC
:100080000C94FD140C94FD140C94FD14E09B0E9C38
:100090003C9C2E9D07AC07AC07AC07AC07AC07AC8B
:1000A00007AC07AC07AC6B9CAA9CEB9C07AC07ACFD
:1000B00007AC07AC07AC07AC07AC07AC07AC07ACA8
:1000C00007ACB59F16A077A0D8A039A19AA1FBA133
:1000D0007FA208A703A37BA3F3A368A4DCA450A575
:1000E000C4A530A69CA607AC07AC07AC07AC07AC10
:1000F000839EEB9E07AC5FA7D3A742A8B8A8E0A851
:1001000036A973A9B0A90FAA70AACFAA2EAB5AAB71
:1001100008A907AC07AC07AC07AC07AC07AC07AC49
:1001200007AC07AC07AC07AC07AC179E4C9E07ACFE
:1001300007AC07AC07AC07AC07AC07AC07AC07AC27
:1001400007ACAA9E07AC07AC07AC93ABD0AB07AC2F
:1001500007AC07AC07ACD29B07AC07AC719DAA9D5E
:10016000F79D509F084AD73B3BCE016E84BCBFFD34
:10017000C12F3D6C74319ABD56833DDA3D00C77F77
:1001800011BED9E4BB4C3E916BAAAABE0000008010
:100190003F05A84CCDB2D44EB93836A9020C50B99F
:1001A000918688083CA6AAAA2ABE000000803F00CB
:1001B0000001000F0015000E001200FFFF160017CF
:1001C000000E001300FFFF030002001A001400FFDE
:1001D000FF1B00FFFF0D000C000400010000000EDB
:1001E00000070006001F00536574204D6963726F9D
:1001F0007374657070696E670048656174696E67D5
:10020000204265640048656174696E6720457874B2
:100210007275646572004649524D574152455F4EB2
:10022000414D453A52657065746965725F302E398B
:1002300031204649524D574152455F55524C3A681C
:10024000747470733A2F2F6769746875622E636FC8
:100250006D2F72657065746965722F526570657473
:100260006965722D4669726D776172652F205052F3
:100270004F544F434F4C5F56455253494F4E3A31BE
:100280002E30204D414348494E455F545950453A20
:100290004D656E64656C2045585452554445525F17
:1002A000434F554E543A31205245504554494552DA
:1002B0005F50524F544F434F4C3A32004465627581
:1002C000673A006F6B000D0A004E414E00494E46E2
:1002D000004572726F723A00496E666F3A0057615C
:1002E000726E696E673A00526573656E643A0045D6
:1002F00063686F3A006F6B200057726F6E67206300
:100300006865636B73756D004D697373696E672003
:10031000636865636B73756D00466F726D61742001
:100320006572726F7200446F6E65207072696E74D0
:10033000696E672066696C650020580020590020AE
:100340005A0020450020460020530020500020493C
:1003500000204A00205200534420726561642065E9
:1003600072726F72004572726F723A65787065636F
:10037000746564206C696E65200020676F742000CE
:10038000736B69702000424C4B200073746172746F
:1003900000506F77657255700045787465726E61B4
:1003A0006C2052657365740042726F776E206F75B2
:1003B00074205265736574005761746368646F6775
:1003C00020526573657400536F667477617265209F
:1003D000526573657400556E6B6E6F776E20636F38
:1003E0006D6D616E643A00467265652052414D3A0A
:1003F00000583A0020583A0020593A00205A3A0052
:1004000020453A00543A0020423A0020403A002069
:1004100054002040002042403A0020524157003A08
:10042000002F00202F0053706565644D756C746952
:10043000706C793A00466C6F774D756C7469706CAE
:10044000793A0046616E73706565643A005072696E
:100450006E7465642066696C616D656E743A0050F7
:1004600072696E74696E672074696D653A006D20FB
:10047000002064617973200020686F75727320001A
:10048000206D696E00496E76616C696420617263EB
:10049000002C002000593A005A3A0045303A0045F5
:1004A000313A004D53312C4D53322050696E730058
:1004B000536574206F7574707574200020746F20FC
:1004C000004820004C2000785F6D696E3A00785F2C
:1004D0006D61783A00795F6D696E3A00795F6D61A0
:1004E000783A007A5F6D696E3A007A5F6D61783AAA
:1004F000004A65726B3A00205A4A65726B3A0020D6
:100500006C696E6561722073746570733A00207156
:1005100075616472617469632073746570733A0005
:100520002C2073706565643D00454550524F4D2049
:1005300075706461746564006C696E656172204CED
:100540003A0020717561647261746963204B3A00EE
:10055000546172676574457874720054617267659E
:10056000744265643A00504944204175746F747553
:100570006E652073746172740020626961733A2041
:100580000020643A2000206D696E3A2000206D61E1
:10059000783A2000204B753A20002054753A20000C
:1005A00020436C61737369632050494400204B7091
:1005B0003A2000204B693A2000204B643A2000503A
:1005C0004944204175746F74756E65206661696C6D
:1005D0006564212054656D70657261747572652063
:1005E000746F206869676800504944204175746FD2
:1005F00074756E65206661696C6564212074696D2F
:10060000656F757400504944204175746F74756E40
:10061000652066696E6973686564202120506C618D
:10062000636520746865204B702C204B6920616ED7
:1006300064204B6420636F6E7374616E7473206901
:100640006E2074686520436F6E66696775726174A9
:10065000696F6E2E68206F7220454550524F4D00D5
:100660004D54454D503A006865617465642062657B
:100670006400657874727564657220003A20746550
:100680006D702073656E736F722064656665637448
:10069000003A20776F726B696E67005072696E74F2
:1006A00065722073657420696E746F20647279209E
:1006B00072756E206D6F646520756E74696C207242
:1006C00065737461727421004175746F6C65766531
:1006D0006C696E6720656E61626C6564004175745B
:1006E0006F6C6576656C696E672064697361626CB6
:1006F0006564005A2D70726F6265206661696C6571
:1007000064005A2D70726F6265206D61783A0050F6
:1007100072696E746572206865696768743A0077FB
:10072000616974004731205A3320463630300A4719
:100730003120583130205931302046363030300A9F
:100740004731205A302E3220463630300A004731A9
:10075000205A3320463630300A473120583139305C
:10076000205931302046363030300A4731205A3057
:100770002E3220463630300A004731205A33204688
:100780003630300A4731205831393020593139302C
:100790002046363030300A4731205A302E3220463B
:1007A0003630300A004731205A3320463630300A7E
:1007B00047312058313020593139302046363030D9
:1007C000300A4731205A302E3220463630300A0067
:1007D000436F6E66696775726174696F6E207374BA
:1007E0006F72656420746F20454550524F4D2E0046
:1007F000436F6E66696775726174696F6E206C6FA6
:10080000616465642066726F6D20454550524F4D9E
:100810002E00436F6E66696775726174696F6E2032
:10082000726573657420746F2064656661756C749D
:10083000732E0050726F746F636F6C2076657273E5
:10084000696F6E206368616E6765642C20757067E0
:10085000726164696E6700457874722E004550526B
:100860003A3020004550523A3120004550523A3239
:1008700020004550523A3320004261756472617421
:10088000650046696C616D656E74207072696E7486
:100890006564205B6D5D005072696E7465722061E5
:1008A0006374697665205B735D004D61782E206905
:1008B0006E6163746976652074696D65205B6D7324
:1008C0002C303D6F66665D0053746F7020737465E5
:1008D0007070657220616674657220696E61637400
:1008E0006976697479205B6D732C303D6F66665D47
:1008F000005820686F6D6520706F73205B6D6D5DB3
:10090000005920686F6D6520706F73205B6D6D5DA1
:10091000005A20686F6D6520706F73205B6D6D5D90
:100920000058206D6178206C656E677468205B6D7F
:100930006D5D0059206D6178206C656E677468206C
:100940005B6D6D5D005A206D6178206C656E67741B
:1009500068205B6D6D5D0058206261636B6C617334
:1009600068205B6D6D5D0059206261636B6C617323
:1009700068205B6D6D5D005A206261636B6C617312
:1009800068205B6D6D5D004D61782E206A65726B2D
:10099000205B6D6D2F735D004D61782E205A2D6A9E
:1009A00065726B205B6D6D2F735D00582D617869EA
:1009B0007320737465707320706572206D6D0059BB
:1009C0002D6178697320737465707320706572206F
:1009D0006D6D005A2D617869732073746570732092
:1009E000706572206D6D00582D61786973206D619E
:1009F000782E206665656472617465205B6D6D2F6D
:100A0000735D00592D61786973206D61782E2066C1
:100A100065656472617465205B6D6D2F735D005A4E
:100A20002D61786973206D61782E2066656564722A
:100A3000617465205B6D6D2F735D00582D61786961
:100A40007320686F6D696E67206665656472617496
:100A500065205B6D6D2F735D00592D617869732082
:100A6000686F6D696E672066656564726174652084
:100A70005B6D6D2F735D005A2D6178697320686F0F
:100A80006D696E67206665656472617465205B6D73
:100A90006D2F735D00582D61786973206163636504
:100AA0006C65726174696F6E205B6D6D2F735E3261
:100AB0005D00592D6178697320616363656C6572AF
:100AC0006174696F6E205B6D6D2F735E325D005ACD
:100AD0002D6178697320616363656C657261746907
:100AE0006F6E205B6D6D2F735E325D00582D6178E7
:100AF00069732074726176656C20616363656C65EF
:100B0000726174696F6E205B6D6D2F735E325D0074
:100B1000592D617869732074726176656C20616308
:100B200063656C65726174696F6E205B6D6D2F73A8
:100B30005E325D005A2D617869732074726176654A
:100B40006C20616363656C65726174696F6E205BB4
:100B50006D6D2F735E325D004F5053206F70657264
:100B60006174696F6E206D6F6465205B303D4F6608
:100B7000662C313D436C61737369632C323D466171
:100B800073745D004F5053206D6F766520616674FD
:100B900065722078252072657472616374205B250C
:100BA0005D004F5053206D696E2E2064697374612F
:100BB0006E636520666F722066696C2E20726574A4
:100BC00072616374696F6E205B6D6D5D004F505391
:100BD0002072657472616374696F6E206C656E67F4
:100BE0007468205B6D6D5D004F50532072657472A8
:100BF000616374696F6E206261636B6C61736820FE
:100C00005B6D6D5D004265642048656174204D61D7
:100C10006E61676572205B302D335D004265642034
:100C2000504944206472697665206D6178004265A0
:100C30006420504944206472697665206D696E00B5
:100C40004265642050494420502D6761696E00421E
:100C500065642050494420492D6761696E004265F2
:100C6000642050494420442D6761696E00426564E8
:100C700020504944206D61782076616C7565205B59
:100C8000302D3235355D0073746570732070657278
:100C9000206D6D006D61782E2066656564726174EB
:100CA00065205B6D6D2F735D0073746172742066D7
:100CB00065656472617465205B6D6D2F735D0061A5
:100CC0006363656C65726174696F6E205B6D6D2F17
:100CD000735E325D0068656174206D616E61676589
:100CE00072205B302D335D00504944206472697678
:100CF00065206D61780050494420647269766520F2
:100D00006D696E0050494420502D6761696E2F64F3
:100D10006561642D74696D650050494420492D67F3
:100D200061696E0050494420442D6761696E00502E
:100D30004944206D61782076616C7565205B302DAB
:100D40003235355D00582D6F6666736574205B73B0
:100D5000746570735D00592D6F6666736574205BF2
:100D600073746570735D0074656D702E20737461AB
:100D700062696C697A652074696D65205B735D00DA
:100D800074656D702E20666F722072657472616377
:100D900074696F6E207768656E2068656174696E2E
:100DA00067205B435D0064697374616E63652074E2
:100DB0006F2072657472616374207768656E206855
:100DC000656174696E67205B6D6D5D006578747236
:100DD0007564657220636F6F6C65722073706565F2
:100DE00064205B302D3235355D00616476616E6361
:100DF00065204B205B303D6F66665D006164766107
:100E00006E6365204C205B303D6F66665D00534429
:100E100020436172642072656D6F7665640053448F
:100E2000204361726420696E736572746564005357
:100E30004420696E6974206661696C006572726F26
:100E4000722077726974696E6720746F2066696CAE
:100E50006500426567696E2066696C65206C697320
:100E60007400456E642066696C65206C697374005B
:100E700046696C65206F70656E65643A0020536941
:100E80007A653A0046696C652073656C65637465C4
:100E9000640066696C652E6F70656E206661696CB2
:100EA0006564005344207072696E74696E672062D5
:100EB00079746520004E6F74205344207072696EFF
:100EC00074696E67006F70656E206661696C656439
:100ED0002C2046696C653A200057726974696E6708
:100EE00020746F2066696C653A2000446F6E65203F
:100EF000736176696E672066696C652E0046696C61
:100F0000652064656C657465640044656C6574692E
:100F10006F6E206661696C65640044697265637414
:100F20006F727920637265617465640043726561F4
:100F300074696F6E206661696C6564005344206556
:100F400072726F72436F64653A000701061C151CCC
:100F5000143A21002243141F1F730FE30F3710A709
:100F600010F710DF1100006312EB12F7134714C3E0
:100F70001400000000A00F5C0060096900100979EE
:100F800000C0088C007008A2002008BD00D007DE59
:100F9000008007050130073401E0066D019006B2BC
:100FA0000140060702F0056D02A005E80250057B2E
:100FB0000300052B04B004F8046004EB06C00335FD
:100FC0000920037F0B8002650DE001B00E40011D7A
:100FD0000FF000480FC8006C0FA000ED0F60FFFE7F
:100FE0000F48FE0400801AD8009808AC0120078042
:100FF0000250065403C80528045805FC040005D017
:1010000005B004A4066804780728044C08E8032007
:1010100009B003F4097003C80A38039C0BF8027086
:101020000CB002440D6802180E0802EC0E8801C0D4
:101030000F8800F00F00000400001B5400600964DA
:101040000010097400C008840070089C002008B8D3
:1010500000D007D8008007000130072C01E00668A7
:10106000019006AC0140060002F0056802A005E010
:10107000025005740300052404B004F0046004DC8D
:10108000051004E406C00304087003300920037847
:101090000B8002600DE001A80E4001680FA000C0A7
:1010A0000F0000E80F60FF0400700DD8004804AC8A
:1010B0000158038002D8025403800228043802FC3D
:1010C000040002D005C801A4069801780770014CFD
:1010D00008480120091801F409F000C80AC8009C5A
:1010E0000BA000700C7000440D3800180E0000ECCE
:1010F0000EA8FFC00FE8FE380060093B0038094029
:101100000010094600E8084C00C008520098085931
:10111000007008620048086C0020087600F807801C
:1011200000D0079100A8079C008007A8005807BBC3
:10113000003007D0000807E300E006F800B806100A
:101140000190062D016806500140067201180690B4
:1011500001F005C201C805EC01A005280278056769
:10116000025005B2022805EE0200053E03D804989D
:1011700003B004F20388045E046004BF0438043240
:10118000051004B405E8033A06C003D80698036CBA
:10119000077003F8074803980820032E09F802D4C3
:1011A00009D0026F0AA8020F0B80029F0B58022B76
:1011B0000C3002B30C08022F0DE001980DB801FCB1
:1011C0000D90014C0E68019C0E40011D0FF000486F
:1011D0000FC8006C0FA000ED0F60FFFE0F48FE3837
:1011E000006009BB00D0076702F005B202C805EE37
:1011F00002A0053E03780598035005F20328055E1A
:10120000040005BF04D80432058804B40560043A1C
:10121000063804D80610046C07E803F807C00398E2
:101220000898032E097003D40948036F0A10030FAE
:101230000BE0029F0BA8022B0C6002B30C4002983B
:101240000DF001FC0DA0014C0E70019C0E40011D23
:101250000FF000480FC8006C0FA000ED0F60FFFEFC
:101260000F48FE0000401F450060094F0010095C58
:1012700000C0086B0070087D0020089200D007AC09
:10128000008007CC003007DE00E006230190065EF8
:10129000014006A601F005FF01A0056D025005F30F
:1012A0000200059603B0045A046004400510044887
:1012B00006C0036E077003A8082003EB09D00223C1
:1012C0000B8002410C3002390DE001040E9001A2A6
:1012D0000E4001170FF000690FA000A20F5000C6CA
:1012E0000F0000DD0FB0FFEB0F60FF0400681D4C26
:1012F00000500B94005809DC0050082401A8076C2A
:10130000012807B401C006FC017006440228068CBF
:1013100002F005D402B8051C03880564035805AC27
:10132000033005F40310053C04E8048404C804CC2D
:1013300004A804140590045C057004A4055804EC8A
:10134000053804340620047C060804C406F0030CA7
:1013500007D8035407C8039C07B003E40798032C7D
:1013600008800374087003BC085803040948034C40
:1013700009300394091803DC090803240AF0026CFD
:101380000AE002B40AC802FC0AB002440BA0028CB4
:101390000B8802D40B70021C0C5802640C4002AC87
:1013A0000C2802F40C10023C0DF001840DD801CC85
:1013B0000DB801140E98015C0E7001A40E4801ECEA
:1013C0000E1801340FD8007C0F8800C40F0800FCF1
:1013D0000F000000000000000000000000000000FE
:1013E00000000000000000000000000000000000FD
:1013F0000000000000000004000016D800C006AC89
:101400000178058002C004540348042804E803FC62
:10141000049803D0055003A40618037807D8024C9B
:1014200008A80220097002F4093802C80A08029CC0
:101430000BD001700C9001440D5001180EF800EC17
:101440000E8800C00F00000400401D900060091CC1
:1014500001B007A801D00634023806C002C8054C06
:10146000036805D80318056404D804F00498047CC4
:1014700005600408063004940600042007D003AC7D
:1014800007A80338088003C408580350093003DC58
:10149000090803680AE002F40AB802800B88020C0B
:1014A0000C6002980C3002240DF801B00DC0013C14
:1014B0000E8001C80E3001540FB800B40F2800E0B0
:1014C0000F00000400081D900058091C01B007A877
:1014D00001C80634023006C002C0054C036805D8B6
:1014E0000318056404D004F00498047C0560040823
:1014F000063004940600042007D003AC07A8033884
:10150000088003C408580350093003DC0908036845
:101510000AD802F40AB002800B88020C0C60029810
:101520000C3002240DF801B00DC0013C0E8001C842
:101530000E3001540FB800B40F2800E00F00005324
:1015400044206572726F7220666978656400534446
:10155000206572726F7220646964206E6F742072ED
:1015600065636F7665722100534420526561642083
:101570004572726F720042696E6172793A00436F10
:101580006D6D616E644275666665720000000000F4
:1015900000000000000000000000000024F403D957
:1015A00050C38EB1C2A23D96828B3582127AE3720D
:1015B000816CCB66A861015DC758EB546151204E28
:1015C0001E4B5648C14559431A41013F093D2F3B27
:1015D0007139CD374036C93465331432D430A32F36
:1015E000802E6B2D632C672B752A8E29B028DC2763
:1015F00010274B268F25D9242B248223E022432237
:10160000AC211A218D200420801F001F841E0C1E77
:10161000971D261DB81C4E1CE61B821B201BC11AE1
:10162000641A0A1AB2195D190A19B9186A181C182D
:10163000D11788174017FA16B51673163116F1151B
:10164000B31576153A150015C7148F1458142214C3
:10165000EE13BA13881356132513F612C7129912F4
:101660006C1240121512EB11C11198117011481132
:101670002111FB10D610B1108D10691046102410E6
:101680000210E10FC00FA00F800F610F420F230F58
:10169000060FE80ECB0EAF0E930E770E5C0E410ECA
:1016A000270E0D0EF30DDA0DC10DA80D900D780D5E
:1016B000600D490D320D1B0D050DEF0CD90CC30C3F
:1016C000AE0C990C850C700C5C0C480C350C210C84
:1016D0000E0CFB0BE80BD60BC40BB20BA00B8E0B46
:1016E0007D0B6B0B5A0B4A0B390B290B180B080B94
:1016F000F80AE90AD90ACA0ABB0AAC0A9D0A8E0A84
:10170000800A710A630A550A470A390A2C0A1E0A16
:10171000110A040AF709EA09DD09D009C409B70961
:10172000AB099F09920987097B096F096309580969
:101730004C09410936092B09200915090A09000934
:10174000F508EB08E008D608CC08C208B808AE08CF
:10175000A4089A08900887087D0874086B08610837
:1017600058084F0846083D0834082C0823081A0872
:10177000120809080108F807F007E807E007D8078A
:10178000D007C807C007B807B007A807A10700001F
:10179000420FA1071605D0030D038B022E02E801AC
:1017A000B2018601630145012C0117010401F40017
:1017B00049646C6500486F6D65205A00486F6D651F
:1017C000205900486F6D652058005374657070652E
:1017D000722044697361626C6564004B696C6C656E
:1017E000640055706C6F6164696E672E2E2E005315
:1017F00044207072696E742073746F707065642019
:10180000627920757365722E0000002110422063FA
:10181000308440A550C660E770088129914AA16BC9
:10182000B18CC1ADD1CEE1EFF13112100273325261
:1018300022B5529442F772D662399318837BB35A19
:10184000A3BDD39CC3FFF3DEE36224433420040131
:1018500014E664C774A44485546AA54BB528850969
:1018600095EEE5CFF5ACC58DD55336722611163001
:1018700006D776F6669556B4465BB77AA7199738B9
:1018800087DFF7FEE79DD7BCC7C448E5588668A741
:10189000784008611802282338CCC9EDD98EE9AF09
:1018A000F9488969990AA92BB9F55AD44AB77A96A1
:1018B0006A711A500A333A122AFDDBDCCBBFFB9E59
:1018C000EB799B588B3BBB1AABA66C877CE44CC571
:1018D0005C222C033C600C411CAEED8FFDECCDCDA9
:1018E000DD2AAD0BBD688D499D977EB66ED55EF441
:1018F0004E133E322E511E700E9FFFBEEFDDDFFCF9
:10190000CF1BBF3AAF599F788F8891A981CAB1EB9D
:10191000A10CD12DC14EF16FE18010A100C230E3C6
:10192000200450254046706760B9839893FBA3DA82
:10193000B33DC31CD37FE35EF3B1029012F322D216
:10194000323542145277625672EAB5CBA5A8958912
:10195000856EF54FE52CD50DC5E234C324A0148166
:10196000046674476424540544DBA7FAB79987B822
:10197000975FE77EF71DC73CD7D326F2369106B0B6
:101980001657667676154634564CD96DC90EF92F22
:10199000E9C899E9898AB9ABA94458654806782706
:1019A00068C018E1088238A3287DCB5CDB3FEB1EC2
:1019B000FBF98BD89BBBAB9ABB754A545A376A1656
:1019C0007AF10AD01AB32A923A2EFD0FED6CDD4D52
:1019D000CDAABD8BADE89DC98D267C076C645C45A6
:1019E0004CA23C832CE01CC10C1FEF3EFF5DCF7C62
:1019F000DF9BAFBABFD98FF89F176E367E554E74F6
:101A00005E932EB23ED10EF01E7C3C3E5E2B3D3FDF
:101A10002F5B5D3B2C2A225C004E6F206572726F3B
:101A20007220666F756E642E0043616E2774206F9E
:101A300070656E20726F6F74206469726563746F75
:101A400072792E00496E76616C696420666F726DE2
:101A500061742C207265666F726D61742053442E20
:101A6000004E6F20636172642C2077726F6E672066
:101A7000636869702073656C6563742070696E2C8F
:101A8000206F72205350492070726F626C656D3FF9
:101A90000043616E27742061636365737320534450
:101AA00020636172642E20446F206E6F7420726513
:101AB000666F726D61742E000001FF00FF0000016F
:101AC000010000FF00FF0100416374696F6E3A2559
:101AD0006C61000310270200D11C0310270200D5FF
:101AE0001C0100000100D91C0200000800DB1C03DF
:101AF000ED030400EB1C03EE030400F31C03EF03EF
:101B00000400FB1C03FA030400031D03FB03040091
:101B10000B1D03FC030400131D0200000B001B1D22
:101B20000200000600311D0200000C003D1D526540
:101B3000717565737450617573653A004E6F20530B
:101B400044204361726400436F6F6C646F776E0072
:101B5000556E6C6F61642046696C616D656E7400D2
:101B60004C6F61642046696C616D656E74005072E3
:101B70006568656174204142530050726568656113
:101B80007420504C41008025000040380000004B7C
:101B900000008070000000960000C0DA000000E144
:101BA0000000002C010008B2010000C2010000F496
:101BB00001000084030090D0030000E80300000847
:101BC000070020A1070000100E0040420F0060E354
:101BD0001600000000000200000900551D671D6E80
:101BE0001D751D7C1D4F6E004F66660059657300A4
:101BF0004E6F00030004004E2F4100003A002064A5
:101C00006179732000503830324D5F380042616E88
:101C10006742616E6700536C6F7742616E67004484
:101C20006561642054696D650050494400507269D3
:101C30006E74696E672E2E2E00206465662000008B
:101C400000003FCDCC4C3D0AD7A33B6F12033A5264
:101C5000657065746965722D302E3931005A6F6E6A
:101C60006573746172203344205072696E746572BA
:101C700000503830324D5F3800503830324D5F38C8
:101C80005F56312E36005072696E7465722072652F
:101C90006164792E0000401454040E15041C0000E9
:101CA00000040A040000000000001F1F1F1F1F0087
:101CB00000001F1111111F0000040A0A0A0E1F1F45
:101CC0000E001C1F11111F0000001F1511151F1FF2
:101CD00000831D8A1D911D981D9F1D9F1DA61DAD72
:101CE0001DB41DBB1DC21DC91DD01DD71DDE1DE5A8
:101CF0001DEC1DF31DFA1D011E081E0F1E161E1DD4
:101D00001E241E2B1E321E391E401E471E4E1E55FF
:101D10001E5C1E631E6A1E711E781E9F1D7F1E861E
:101D20001E8D1E941E9B1EA21EA91EB01EB71EBE97
:101D30001E9F1DC51ECC1ED31EDA1EE11E9F1D7FD9
:101D40001EE81EEF1EF61EFD1E041F0B1F121F199C
:101D50001F201FDA1E9F1D271FA61D2E1F351F3C8B
:101D60001F431F4A1F511F0000000400581F00009E
:101D7000000400601F0000000400681F0000000451
:101D800000701F781F0000000000861F0000000088
:101D900000971F0000000000A51F0000000000B613
:101DA0001F03E8030000BD1F03F5030102C81F0362
:101DB000F6030204D41F0354040200DF1F03F703D9
:101DC0000400EE1F03F8030100FB1F03F9030001E9
:101DD000062003F4030102122000000000001B2073
:101DE00000000000002B2000000000003B2000004D
:101DF0000000003C20000000000045200000000022
:101E00000055200000000000652000000000006672
:101E10002000000000006F2000000000007F200074
:101E2000000000008F200000000000902000000053
:101E3000000099200000000000A920000000000020
:101E4000B9200000000000BA200000000000C320FC
:101E50000000000000D3200000000000E32000008C
:101E6000000000E4200000000000ED200000000061
:101E700000FD2000000000000D2100000000000E09
:101E80002103FD0300201721041F04000029210461
:101E9000480400003B2103370400004721034704A6
:101EA0000000532103C00F0000612103C10F000097
:101EB000712103380400007A2103310400108821C5
:101EC00003420400209821043C040000A821043DA2
:101ED000040000B821033A040000C72102D6210003
:101EE00000DD210343040000E82103FE030020EF8E
:101EF0002103FF030020F6210300040020FD21023E
:101F0000041B0000092202EF1A00001422020B1B1E
:101F10000000202202F61A00002B2202121B0000F1
:101F2000372202FD1A0000422202191B0000512232
:101F300002271B00005A2202201B00006322026DB0
:101F4000220000742202E81A00007C22028622008D
:101F5000008D22029B220000A222A922B022B722D9
:101F6000BE22C522CC22D322DA22E122E822EF22AD
:101F7000F622FD2204230B23436F6E666967757298
:101F80006174696F6E0073746F72656420696E208E
:101F9000454550524F4D00436F6E666967757261DB
:101FA00074696F6E006C6F6164656420662E2045F5
:101FB0004550524F4D004261636B200100507269E1
:101FC0006E742066696C650050617573652050728F
:101FD000696E740053746F70205072696E740043A0
:101FE0006F6E74696E7565205072696E7400556EFF
:101FF0006D6F756E742043617264004D6F756E7401
:1020000020436172640044656C6574652066696C88
:102010006500583A257830206D6D004D696E206559
:102020006E6473746F703A257378004D6178206523
:102030006E6473746F703A2573580000593A2578AE
:1020400031206D6D004D696E20656E6473746F7024
:102050003A257379004D617820656E6473746F70F2
:102060003A25735900005A3A257832206D6D004D9B
:10207000696E20656E6473746F703A25737A004DD3
:10208000617820656E6473746F703A25735A00002E
:10209000583A257830206D6D004D696E20656E646C
:1020A00073746F703A257378004D617820656E64A3
:1020B00073746F703A2573580000593A25783120AF
:1020C0006D6D004D696E20656E6473746F703A2596
:1020D0007379004D617820656E6473746F703A2572
:1020E000735900005A3A257832206D6D004D696EA3
:1020F00020656E6473746F703A25737A004D617851
:1021000020656E6473746F703A25735A0000486FCF
:102110006D6520416C6C005370656564204D756C75
:102120002E3A256F6D25252500466C6F77204D755D
:102130006C2E203A256F662525250050726568654E
:10214000617420504C410050726568656174204193
:102150004253004C6F61642046696C616D656E741A
:1021600000556E6C6F61642046696C616D656E74BC
:1021700000436F6F6C646F776E0053657420746FEB
:10218000204F726967696E0044697361626C6520F3
:1021900073746570706572004265642054656D707B
:1021A0003A2025456202430054656D702E20313A75
:1021B00020202545300243004578747275646572AD
:1021C0002031204F666600457874722E20706F7340
:1021D0006974696F6E0003F0030200122353657483
:1021E000204F726967696E00486F6D65205800481E
:1021F0006F6D65205900486F6D65205A005820505A
:102200006F732E2046617374005820506F73697489
:10221000696F6E005920506F732E204661737400F1
:102220005920506F736974696F6E005A20506F7334
:102230002E2046617374005A20506F736974696F61
:102240006E00517569636B2053657474696E6773B2
:1022500000506F736974696F6E00457874727564AD
:1022600065720046616E207370656564000200004F
:10227000070016235344204361726400446562756D
:102280006767696E670002000005002423436F6ED4
:1022900066696775726174696F6E000200000800FC
:1022A0002E233E2300000000005123000000000008
:1022B0006023000000000075230000000000792367
:1022C0000000000000822300000000008B230000BB
:1022D000000000942300000000009823000000008C
:1022E00000A9230000000000BA230000000000BB8A
:1022F000230000000000BF230000000000CD2300E9
:1023000000000000D1230000000000E223000000D4
:102310000000E823EF239F1DF623FD2304240B2454
:10232000122419249F1D202427242E2435249F1D88
:102330003C2443244A24512458245F246624052540
:1023400065632F25456302072565422F25456202F7
:10235000005A3A25783220204275663A256F4200AD
:102360004D756C3A20256F6D202020466C6F773AB2
:1023700020256F6600256F7300583A257830206D50
:102380006D00593A257831206D6D005A3A25783222
:10239000206D6D00256F730045313A2565302F257E
:1023A000453002437E256F300020423A2565622F7A
:1023B00025456202437E256F620000256F73005041
:1023C00072696E74696E672074696D650025557455
:1023D0000046696C616D656E74207072696E74651B
:1023E0006400255566206D006D2400000000007615
:1023F00024000000000085240452040000962403F9
:102400001A040800A324031B040000B124031C04C5
:102410000000BF24031D040000CD24031E0400009F
:10242000DA240332040000E6240333040000F2241B
:102430000334040000FE2403350400000A250212C0
:10244000250000192502262500002D25023625002D
:10245000003D2502462500004D2503060400005DD1
:102460002503070400006C25027F250000453A255E
:102470007833206D6D003120636C69636B203D20E3
:1024800031206D6D0046616E2073706565643A257C
:102490004673252525005475726E2046616E204FC7
:1024A0006666005365742046616E20323525252509
:1024B000005365742046616E203530252525005374
:1024C00065742046616E20373525252500536574D7
:1024D0002046616E2046756C6C004563686F202055
:1024E000203A25646F00496E666F2020203A2564EB
:1024F00069004572726F7273203A256465004472F8
:10250000792072756E3A2564640047656E65726164
:102510006C0002000004008625416363656C6572EF
:102520006174696F6E0002000009008E25466565C2
:102530006472617465000200000700A0254578748C
:102540007275646572000200000F00AE2553746F4F
:10255000726520746F20454550524F4D004C6F619D
:102560006420662E20454550524F4D004C657665DF
:102570006C696E6720617578696C696172790002B7
:1025800000000700CC259F1DDA25E125E8259F1DC9
:10259000EF25F625FD2504260B26122619262026D2
:1025A0009F1D27262E2635263C2643264A269F1D7C
:1025B000512658265F2666266D2674267B2682269F
:1025C0008926902697269E26A526AC269F1D7F1E2F
:1025D000B326BA26C126C826201FCF260410040021
:1025E00000DC2602ED260000F42602022700000986
:1025F000270408040000152704090400002127040B
:102600000A0400002D27040B0400003927040C04E1
:1026100000004527040D0400005127040E040000AB
:102620005D27040F040000692704140400007327C9
:1026300004150400007D27041604000087270411F8
:10264000040000922704120400009D2704130400D4
:1026500000A8270429040000B527042C040000C2A8
:1026600027042B040000CD27042A040000D72704E8
:102670002E040000E527044D040000F827044C0454
:1026800000000928042D040000152804220400007D
:10269000222804230400002C2804240400003628E7
:1026A0000425040000442804260400005228042FB6
:1026B0000400005E2803B10F00006A2803B20F0077
:1026C00000762803B30F0000822803B40F000042F5
:1026D000617564726174653A256F63005374657047
:1026E00070657220496E6163746976650003200429
:1026F00002008E284D61782E20496E6163746976E0
:102700006500035804020092285072696E742058C4
:102710003A256178005072696E7420593A256179C2
:10272000005072696E74205A3A25617A004D6F76B6
:10273000652058203A256158004D6F766520592054
:102740003A256159004D6F7665205A203A25615A25
:10275000004A65726B2020203A25616A005A2D4A92
:1027600065726B203A25614A004D617820583A2500
:102770006678004D617820593A256679004D617878
:10278000205A3A25667A00486F6D6520583A2566CA
:102790005800486F6D6520593A25665900486F6D9D
:1027A00065205A3A25665A0053746570732F4D4D53
:1027B0003A2553650053746172742046523A255885
:1027C00066004D61782046523A25584600416363C1
:1027D000656C3A25584100537461622E54696D65E9
:1027E0003A255877005761697420556E6974733AB9
:1027F00020255855206D6D00576169742054656D12
:10280000702E20255854024300436F6E74726F6C13
:102810003A2558680044542F50494420503A2558CE
:10282000700050494420493A2558690050494420D5
:10283000443A255864004472697665204D696E3AC1
:1028400025586D004472697665204D61783A2558A7
:102850004D00504944204D61783A25584400476F57
:10286000746F20506F73692E3100476F746F205062
:102870006F73692E3200476F746F20506F73692E2B
:102880003300476F746F20506F73692E34009628A1
:102890009D28A428AB28B2280000000000C1280011
:1028A00000000000CB280000000000DA2800000033
:1028B00000004469732E2041667465723A2569737D
:1028C000005B735D20303D4F6666004469732E20C7
:1028D00041667465723A256970005B735D20303D16
:1028E0004F66660000002100240027002A00000037
:1028F0002200250028002B000000200023002600D5
:102900002900020202020202020204040404040476
:102910000404030303030303030301010101010191
:102920000101010204081020408001020408102067
:1029300040800102040810204080804020100804DC
:10294000020100000001020000000000000004037A
:10295000070600000000000000000000000000006A
:102960000000494E46494E4954594E414ECDCCCCBB
:102970003D0AD7233C17B7D13877CC2B329595E653
:10298000241FB14F0A000020410000C84200401C33
:102990004620BCBE4CCA1B0E5AAEC59D7400384FB3
:1029A000EE794C9A11241FBECFEFD0E4DEBFCDBF2D
:1029B00012E0A0E0B1E0E8EFF6E901E00BBF02C0F1
:1029C00007900D92A236B107D9F71BBE10E1A2E61F
:1029D000B2E001C01D92AD39B107E1F719E2C4EAD6
:1029E000D9E204C02297FE010E942CCBCE39D10738
:1029F000C9F70E9408C60C947ACB0C940000CF93C0
:102A0000DF93BC018230910510F462E070E0A09188
:102A10009910B0919A10ED01E0E0F0E040E050E054
:102A200021C0888199818617970769F48A819B81E3
:102A3000309719F09383828304C090939A10809307
:102A40009910FE0134C06817790738F44115510513
:102A500019F08417950708F4AC01FE018A819B8167
:102A60009C01E9012097E9F641155105A9F1CA0138
:102A7000861B970B049708F4BA01E0E0F0E02AC047
:102A80008D919C91119784179507F9F46417750738
:102A900081F412968D919C911397309719F093833E
:102AA000828304C090939A1080939910FD0132960E
:102AB0004CC0CA01861B970BFD01E80FF91F6193FB
:102AC000719302978D939C9340C0FD018281938105
:102AD0009C01D9011097A1F68091971090919810C0
:102AE000892B41F4809114019091150190939810D5
:102AF000809397104091160150911701411551058F
:102B000041F44DB75EB78091120190911301481BBB
:102B1000590B2091971030919810CA01821B930B8A
:102B20008617970780F0AB014E5F5F4F84179507BC
:102B300050F0420F531F5093981040939710F90193
:102B40006193719302C0E0E0F0E0CF01DF91CF919B
:102B50000895CF93DF93009709F450C0EC012297BA
:102B60001B821A82A0919910B0919A10109709F1C6
:102B700040E050E0AC17BD0708F1BB83AA83FE011B
:102B800021913191E20FF31FAE17BF0779F48D91B8
:102B90009C911197280F391F2E5F3F4F398328834F
:102BA00012968D919C9113979B838A8341155105B1
:102BB00071F4D0939A10C093991020C012968D9101
:102BC0009C911397AD01009711F0DC01D3CFFA016E
:102BD000D383C28321913191E20FF31FCE17DF0718
:102BE00069F488819981280F391F2E5F3F4FFA01C0
:102BF000318320838A819B8193838283DF91CF916C
:102C00000895A0E0B0E0E7E0F6E10C9449CBEC01D8
:102C10005B016115710519F0FB0191838083F990C7
:102C20008F2D90E00E9430CB892BC9F7FDE2FF1673
:102C300021F4F990EE24E39405C02BE2F21609F496
:102C4000F990EE248E0101501040C80162E679E24D
:102C500043E050E00E949018892B01F58E010E5F31
:102C60001F4FC80165E679E245E050E00E949018E8
:102C7000892B19F48E01095F1F4FA114B10419F0BB
:102C8000F50111830083E0FC04C070E090E080E86F
:102C900014C070E090E080E86FEF08C1C8016AE6F8
:102CA00079E243E050E00E949018892B69F4A11466
:102CB000B10429F470E090E080EC6FE7F7C0229651
:102CC000F501D183C083F6CF8824992440E050E0F9
:102CD00060E070E0EF2DE053EA30A0F5F2E0EF2A7B
:102CE0008E2D90E09C0128703070E2FE06C0232BF0
:102CF00079F50894811C911C2BC0232B19F00894A2
:102D000081089108DB01CA0112E0880F991FAA1FF0
:102D1000BB1F1A95D1F7480F591F6A1F7B1F440F1D
:102D2000551F661F771F4E0F511D611D711D4839BC
:102D300029E9520729E9620729E1720748F084E08E
:102D4000E82A06C0EE3F31F4E3FC39C098E0E92AF6
:102D5000F990C0CFE53311F0E53189F529912D3295
:102D600019F4E0E1EE2A05C02B3219F081E090E081
:102D700003C0299182E090E0E22FE053EA3018F09E
:102D8000C81BD90B1CC020E030E0FCE020383F0716
:102D90005CF4C901880F991F880F991F280F391FEC
:102DA000220F331F2E0F311DE991E053EA3068F3F3
:102DB000E4FE03C0309521953F4F820E931ECE2C2A
:102DC000DD24E1FE07C0A114B10421F02197F50133
:102DD000D183C083CB01BA010E94A8C77B018C01BB
:102DE000F3E0CF22DD2423E0C216D10421F417FB47
:102DF000109517F9109557016801C801B70120E037
:102E000030E040E050E00E9408C7882309F44AC03F
:102E100097FE0DC021E8E22E29E2F22E90948194D3
:102E200091089394C0E2D0E000E010E012C099E96C
:102E3000E92E99E2F92EF6CFF701259135914591CA
:102E40005491C601B5010E94B8C95B016C018C1A8E
:102E50009D0A8C169D0684F7D595C7950F5F1F4F69
:102E60000630110529F08CEF9FEFE80EF91EF1CF27
:102E7000C501D6017C018D018C2D880F8D2D881FF9
:102E80008F3F51F0C601B50120E030E040E050E056
:102E90000E9408C7882331F482E290E090939C104E
:102EA00080939B107E2D9F2D802F612F272F392FF0
:102EB000482F562FB901CA01CDB7DEB7ECE00C940C
:102EC00065CB2F923F925F926F927F928F929F92EB
:102ED000AF92BF92CF92DF92EF92FF920F931F9328
:102EE000CF93DF938C011B01EA016115710519F085
:102EF000FB0191838083209749F0CE01029783974D
:102F000028F020E030E040E050E0F6C0F801A19069
:102F10008F018A2D90E00E9430CB892BB9F7FDE21A
:102F2000AF1631F4F801A1908F015524539407C0D6
:102F3000FBE2AF1619F4F801A1908F0155242097F8
:102F400019F0C031D105C1F4F0E3AF1679F4F801FE
:102F50008081883711F0883549F4F801A1800E5F2F
:102F60001F4FF2E05F2AC0E1D0E006C0209721F4B5
:102F700080E3A816E9F427C0C830D10531F1C93083
:102F8000D10524F4C230D10531F50CC0CA30D105C9
:102F900089F0C031D105F9F4C12CD12CE12CB8E075
:102FA000FB2E28C0C12CD12CE12CA0E4FA2E22C08B
:102FB000CAE0D0E0FCECCF2EFCECDF2EFCECEF2ED8
:102FC000FCE0FF2E17C0C8E0D0E0C12CD12CE12CD2
:102FD000E0E1FE2E0FC09E01442737FD4095542F9F
:102FE00060E070E080E090E80E94E1CAC901DA0187
:102FF0006C017D0120E030E040E050E060E03E0107
:10300000882477FC8094982C70EDB72EBA0CE9E0F8
:10301000EB1570F48A2D81548A3118F499ECB92E8D
:1030200006C08A2D81568A3150F589EAB82EBA0C2D
:103030008B2D90E08C179D0714F56F3FE1F0C216C1
:10304000D306E406F506B0F0CA01B901A401930164
:103050000E948ECA9B01AC012B0D311D411D511DDB
:103060002130F0E03F07F0E04F07F0E85F0710F491
:1030700061E001C06FEFF801A1908F01C5CF21146D
:10308000310481F0662331F001501040F1011183C9
:10309000008308C051FE1AC002501040F101118394
:1030A000008314C067FF12C050FC05C02FEF3FEF34
:1030B0004FEF5FE704C020E030E040E050E882E2FC
:1030C00090E090939C1080939B1016C050FE08C017
:1030D00050954095309521953F4F4F4F5F4F0CC015
:1030E00057FF0AC082E290E090939C1080939B105F
:1030F0002FEF3FEF4FEF5FE7B901CA01DF91CF91AB
:103100001F910F91FF90EF90DF90CF90BF90AF9005
:103110009F908F907F906F905F903F902F90089539
:10312000FB01DC014150504088F08D9181341CF04E
:103130008B350CF4805E659161341CF06B350CF4BA
:10314000605E861B611171F3990B0895881BFCCF9B
:10315000FB01DC0102C001900D9241505040D8F7B4
:103160000895FB01DC010D900020E9F71197019013
:103170000D920020E1F70895FC018191861721F05E
:103180008823D9F7992708953197CF010895FB0136
:10319000DC018D91019080190110D9F3990B0895EC
:1031A000FB01DC0101900D920020E1F70895FB0185
:1031B000DC014150504048F001900D920020C9F7C9
:1031C00001C01D9241505040E0F70895FC0181E09C
:1031D00090E00190061609F4CF010020D1F7019785
:1031E0000895A0E0B0E0E7EFF8E10C944DCB7C014E
:1031F000EB018A01690109C0CE012196F60109950A
:10320000F70181937F010150104001151105A1F7CD
:10321000CDB7DEB7E8E00C9469CBBF92CF92DF92D6
:10322000EF92FF920F931F937B018C01FB01099595
:10323000B82EC8010196F7010995C82EC80102965B
:10324000F7010995D82EC8010396F7010995982F23
:103250006B2D7C2D8D2D1F910F91FF90EF90DF90A6
:10326000CF90BF900895DF92EF92FF920F931F933C
:103270007B018C01FB010995D82EC8010196F7014D
:103280000995982F8D2D1F910F91FF90EF90DF9052
:103290000895A0E0B0E0EFE4F9E10C944DCBEC012F
:1032A0007B018A01690109C0CE012196F701619174
:1032B0007F01F60109950150104001151105A1F794
:1032C000CDB7DEB7E8E00C9469CBBF92CF92DF9226
:1032D000EF92FF920F931F93D52EC62EB72E790132
:1032E0008C01642FF9010995C80101966D2DF70134
:1032F0000995C80102966C2DF7010995C80103963E
:103300006B2DF70109951F910F91FF90EF90DF90C2
:10331000CF90BF900895DF92EF92FF920F931F938B
:10332000D72E7A018C01FA010995C80101966D2DFD
:10333000F70109951F910F91FF90EF90DF9008958D
:103340009C01F999FECF32BD21BDF89A80B5089550
:103350000895609118017091190180911A0190915E
:103360001B016817790744F470931B0160931A01DD
:1033700087EE93E00E94C22A0895BC01893191052D
:103380001CF469E170E005C0893C910514F068EC1B
:1033900070E070934D0C60934C0C85E394E00E94B8
:1033A000C22A0895EF92FF920F931F93CF93DF935A
:1033B000EC01893191051CF4C9E1D0E006C081E03F
:1033C000C53FD80714F0C4EFD1E0BE01882777FDD0
:1033D0008095982F0E94AAC77B018C0160914A0CAE
:1033E00070914B0C882777FD8095982F0E94AAC773
:1033F0009B01AC01C801B7010E940FC79B01AC0142
:103400006091460C7091470C8091480C9091490C4A
:103410000E94B8C96093460C7093470C8093480C87
:103420009093490CD0934B0CC0934A0C86E294E0E5
:10343000BE010E94C22ADF91CF911F910F91FF9090
:10344000EF9008950E94EB509C018091180190919B
:1034500019012817390724F4309319012093180112
:1034600008950E94884D08952F923F924F925F9247
:103470006F927F928F929F92AF92BF92CF92DF9284
:10348000EF92FF920F931F93DF93CF93CDB7DEB7E9
:1034900028970FB6F894DEBF0FBECDBFA090CB0B20
:1034A000B090CC0BC090CD0BD090CE0B2090CF0B1A
:1034B0003090D00B4090D10B5090D20B8091D30B19
:1034C0009091D40BA091D50BB091D60B89839A83A0
:1034D000AB83BC832091F30B3091F40B4091F50B3F
:1034E0005091F60B6090F70B7090F80B8090F90BF1
:1034F0009090FA0B8091FB0B9091FC0BA091FD0B2F
:10350000B091FE0B8D839E83AF83B8878091870B2C
:10351000882359F40F2EF0E0EF2EF0E0FF2EF0E8B4
:103520000F2FFFE31F2FF02D0AC00F2EF0E7EF2E15
:10353000F2E4FF2EF1E20F2FFDE31F2FF02DC60165
:10354000B5010E9442C6A80197010E94B8C9AB010B
:10355000BC0181EF93E022E00E94FD2B8091870B5C
:10356000882359F40F2EF0E0EF2EF0E0FF2EF0E864
:103570000F2FFFE31F2FF02D0AC00F2EF0E7EF2EC5
:10358000F2E4FF2EF1E20F2FFDE31F2FF02DC20119
:10359000B101A40193010E9442C6A80197010E94B3
:1035A000B8C9AB01BC0188EF93E022E00E94FD2B7B
:1035B0008091870B882359F40F2EF0E0EF2EF0E076
:1035C000FF2EF0E80F2FFFE31F2FF02D0AC00F2E64
:1035D000F0E7EF2EF2E4FF2EF1E20F2FFDE31F2FB5
:1035E000F02D69817A818B819C812D813E814F8173
:1035F00058850E9442C6A80197010E94B8C9AB0134
:10360000BC018CEF93E022E00E94FD2B2091C70BC0
:103610003091C80B4091C90B5091CA0BA090940BEC
:10362000B090950BC090960BD090970B8091870B24
:10363000882359F40F2EF0E0EF2EF0E0FF2EF0E893
:103640000F2FFFE31F2FF02D0AC00F2EF0E7EF2EF4
:10365000F2E4FF2EF1E20F2FFDE31F2FF02DCA0140
:10366000B9010E94AAC7A60195010E94B8C9A80184
:1036700097010E94B8C9AB01BC0180E094E022E050
:103680000E94122C28960FB6F894DEBF0FBECDBF55
:10369000CF91DF911F910F91FF90EF90DF90CF902E
:1036A000BF90AF909F908F907F906F905F904F9062
:1036B0003F902F9008950F931F9303E214E0C801E9
:1036C0006DE00E94074FC8016AE00E94074F1F91FA
:1036D0000F9108956F927F928F929F92AF92BF92B7
:1036E000CF92DF92EF92FF920F931F93DF93CF93CE
:1036F00000D000D0CDB7DEB76091640C7091650C3E
:103700008091660C9091670C2FE632E143E85AE312
:103710000E94B8C97B018C01CE01019661E870E07E
:1037200044E050E020EA39E10E94F118C801B701F5
:1037300029813A814B815C810E9442C6AB01BC0168
:103740008DE494E022E00E94FD2B8EE694E00E943E
:103750009F2AE091CC01F091CD0163857485858528
:10376000968520E030E040E751E40E9416C9181623
:103770000CF47AC06624772443018DE790E060EA78
:1037800079E10E940D197B018C01E60CF71C081DE4
:10379000191DC801B70120E831E541E050E00E9461
:1037A00003CB922E832E742E652E622F732F842FBF
:1037B000952F20E83EEA4EEF5FEF0E948ECA5B0134
:1037C0006C01AE0CBF1CC01ED11E8FE594E0492DCC
:1037D000582D672D762D0E94E92AC601B50120E1FA
:1037E0003EE040E050E00E9403CB122F032FF42E66
:1037F000E52E81E794E0422F502F6F2D7E2D0E9401
:10380000E92A612F702F8F2D9E2D20EF31EF4FEF82
:103810005FEF0E948ECAA60EB71EC81ED91EC60133
:10382000B5012CE330E040E050E00E9403CB88E794
:1038300094E0BA01A9010E94E92A80E894E00E947C
:10384000262B0F900F900F900F90CF91DF911F912B
:103850000F91FF90EF90DF90CF90BF90AF909F902F
:103860008F907F906F9008950E9421C42091600CEA
:103870003091610C4091620C5091630C621B730B90
:10388000840B950B28EE33E040E050E00E94E1CA43
:10389000C901DA013C014D0170CF1F93182FE0914F
:1038A0007502F091760244A555A566A577A584E03A
:1038B00094E022E00E94FD2BE0917502F0917602E7
:1038C00040A951A962A973A983E294E020E00E9473
:1038D000FD2B0E946638AB01BC0187E094E022E03A
:1038E0000E94FD2B409196015091970160919801A3
:1038F0007091990183E294E020E00E94FD2B112356
:1039000091F08AE194E061E070E00E94FA2A6CEFA5
:103910007FE080918E0190918F01681B790B8FE180
:1039200094E00E94FA2AE0918B01F0E0E85BFB4F03
:10393000608185E194E070E00E94FA2AE0911E0126
:10394000EF3F29F4E0917502F0917602E081F0E01A
:10395000E85BFB4F60818BE094E070E00E94FA2A04
:103960000E945B1B1F910895809164028823C1F01F
:10397000109264020E94764180911D0181508093D3
:103980001D01882349F480911C01833010F40E94AA
:10399000383B85E080931D018EE69FE00E9437C191
:1039A000089508C00E946D4A0E94B41C8EE69FE0F4
:1039B0000E944B9A8091810B8823A1F70895CF93A1
:1039C000DF9397FD10C0EC018F3F910521F01CF0B3
:1039D000CFEFD0E002C0009731F08091010C8860F9
:1039E0008093010C07C08091010C877F8093010CAC
:1039F000C0E0D0E0662311F00E94D11C80914B04FE
:103A000090E0C817D90729F083E494E0BE010E9432
:103A1000C22AC0934B04DF91CF9108952F923F9219
:103A20004F925F926F927F928F929F92AF92BF92CE
:103A3000CF92DF92EF92FF920F931F93DF93CF937A
:103A4000CDB7DEB7E0970FB6F894DEBF0FBECDBF9F
:103A50006C0180912702282F84FF19C0D6018C9118
:103A600082FD09C081FF13C016968D919C91179716
:103A70008F36910561F00E9421C4609340047093D9
:103A8000410480934204909343040C949D29F601D1
:103A90000081118102FF75C3808591858431910574
:103AA00009F42DC28531910558F48430910520F434
:103AB000029708F040C020C0049709F056C3E1C146
:103AC0008A35910509F465C28B35910540F485313D
:103AD000910509F418C24C9709F047C317C28C35F9
:103AE000910509F45DC28C35910508F455C28C39F5
:103AF000910509F03AC30EC312FF12C0F601878D7B
:103B000090A1A1A1B2A12091000C0097A105B1053F
:103B100019F0822F806202C0822F8F7D8093000C6B
:103B2000C6010E94DE6F882309F41FC381E061E0B3
:103B30000E943D661AC38091CB0B9091CC0BA09153
:103B4000CD0BB091CE0B89879A87AB87BC878091CC
:103B5000CF0B9091D00BA091D10BB091D20B8D8750
:103B60009E87AF87B88B8091D30B9091D40BA09197
:103B7000D50BB091D60B898B9A8BAB8BBC8BC601C6
:103B80000E94DE6F882309F4F0C2FE01319688E0BE
:103B9000DF011D928A95E9F7F601828180FD05C05B
:103BA00020E030E040E050E007C0D60197962D912C
:103BB0003D914D915C919A978091870B882351F0AC
:103BC000CA01B90123E333E34BEC51E40E94B8C9C5
:103BD0009B01AC0129833A834B835C83F60182818C
:103BE00081FD05C020E030E040E050E007C0D60194
:103BF0009B962D913D914D915C919E978091870B65
:103C0000882351F0CA01B90123E333E34BEC51E4BB
:103C10000E94B8C99B01AC012D833E834F83588716
:103C2000FE01759680E1DF011D928A95E9F780918A
:103C3000CB0B9091CC0BA091CD0BB091CE0B8D8B7B
:103C40009E8BAF8BB88F8091CF0B9091D00BA091B2
:103C5000D10BB091D20B898F9A8FAB8FBC8F809193
:103C6000D30B9091D40BA091D50BB091D60B8D8F27
:103C70009E8FAF8FB8A36091EF0B7091F00B809186
:103C8000F10B9091F20B0E94AAC72091940B3091F6
:103C9000950B4091960B5091970B0E94B8C969A360
:103CA0007AA38BA39CA3F601828182FFC7C087A45D
:103CB00090A8A1A8B2A88091870B882351F0C501D4
:103CC000B40123E333E34BEC51E40E94B8C94B0148
:103CD0005C016D897E898F89988D29853A854B8510
:103CE0005C850E9441C66DA77EA78FA798AB698DA2
:103CF0007A8D8B8D9C8D2D853E854F8558890E94B0
:103D000041C62B013C01C501B40120E030E040E890
:103D100050E40E94B8C9A50194010E94B8C97B0172
:103D20008C016DA57EA58FA598A99B01AC010E9471
:103D3000B8C99B01AC01C801B7010E9441C67B0113
:103D40008C01C301B201A30192010E94B8C99B0179
:103D5000AC01C801B7010E9441C60E9425CA7B017F
:103D60008C016DA57EA58FA598A9A30192010E9443
:103D700023C99B01AC0117FB109517F91095C801D9
:103D8000B7010E940FC77B018C01A80197010E9417
:103D900072CA882329F085E894E00E942B2BE5C1A4
:103DA000D60118968D919C911997039721F417FBD2
:103DB000109517F91095C501B40120E030E040E0FE
:103DC00050E00E9408C7882344F417FB109517F9A8
:103DD0001095B7FAB094B7F8B094C301B201A80136
:103DE00097010E94B8C99B01AC016DA57EA58FA566
:103DF00098A90E9441C620E030E040E05FE30E94C5
:103E0000B8C969837A838B839C836DA57EA58FA5B2
:103E100098A9A80197010E94B8C99B01AC01C301F0
:103E2000B2010E9442C620E030E040E05FE30E9421
:103E3000B8C96D837E838F8398870CC069817A812E
:103E40008B819C812D813E814F8158850E9423C9A1
:103E50004B015C01E0E0D60118968D919C91199779
:103E6000029709F4E1E0CE010996BE016B5E7F4F37
:103E7000AE014F5F5F4F95018401EE2E0E94E85620
:103E800074C10E94D11CF6018081918193FD04C010
:103E9000EE24FF24870107C0D6019396ED90FD9094
:103EA0000D911C91969792FF0DC0F601678D70A140
:103EB00081A192A128EE33E040E050E00E948ECA3A
:103EC0007B018C010E9421C45B016C01AE0CBF1C04
:103ED000C01ED11E04C00E946D4A0E94B41C0E94E4
:103EE00021C4A6019501261B370B480B590BDA019B
:103EF000C90180509449A543B74768F336C181E0B2
:103F00008093870B32C11092870B2FC1C801887331
:103F10009070892B11F080E008C0C80156E096959A
:103F200087955A95E1F78095817006FF08C0109239
:103F3000C70B1092C80B1092C90B1092CA0B8823A2
:103F400021F041E051E061E01DC0D6012D913C918E
:103F5000C90188739070892BC1F0C90143E096951F
:103F600087954A95E1F7582F5170C90134E096952D
:103F700087953A95E1F7682F617025FD02C040E012
:103F800001C041E0852F0E94927480E00E943C6B4A
:103F9000ECC01092B90BE9C081E08093B90BE5C089
:103FA000A090F30BB090F40BE090F50BF090F60BB3
:103FB0006090F70B7090F80B8090F90B9090FA0BD3
:103FC0002090FB0B3090FC0B4090FD0B5090FE0BB3
:103FD00003FF21C0F60122853385448555858091F4
:103FE000870B882351F0CA01B90123E333E34BEC7B
:103FF00051E40E94B8C99B01AC01CA01B9012091EA
:10400000CB0B3091CC0B4091CD0B5091CE0B0E943D
:1040100041C65B017C0104FF23C0D6011E962D9191
:104020003D914D915C9151978091870B882351F080
:10403000CA01B90123E333E34BEC51E40E94B8C950
:104040009B01AC01CA01B9012091CF0B3091D00B7B
:104050004091D10B5091D20B0E9441C63B014C01C3
:1040600005FF21C0F6012289338944895589809151
:10407000870B882351F0CA01B90123E333E34BECEA
:1040800051E40E94B8C99B01AC01CA01B901209159
:10409000D30B3091D40B4091D50B5091D60B0E948D
:1040A00041C61B012C01B501C7019301A401710197
:1040B00082010E941B6BD6018C9186FF56C05696DA
:1040C0002D913D914D915C9159978091870B88235B
:1040D00051F0CA01B90123E333E34BEC51E40E94F0
:1040E000B8C99B01AC01CA01B9012091E701309127
:1040F000E8014091E9015091EA010E94B8C90E948B
:1041000077C76093C70B7093C80B8093C90B9093CC
:10411000CA0B2BC080E061E040E00E94927400D0A6
:1041200000D02091360C3091370C4091380C5091D2
:10413000390C8091FF0190910002A0910102B09191
:104140000202EDB7FEB781839283A383B48360E854
:104150007FE483EC97E47B018C015B016C010E949E
:104160004B730F900F900F900F900E9421C460939B
:1041700040047093410480934204909343040C9450
:104180009D2901FD02C00C948B29D60116968D91B4
:104190009C9117978237910509F4C9C68337910519
:1041A00008F081C08A32910509F47EC18B329105F5
:1041B000C8F58931910509F427C18A319105C8F400
:1041C0008631910509F404C18731910548F48431A1
:1041D000910509F4F3C0459711F00C949D29F3C0A3
:1041E0008731910509F4F9C0489711F00C949D2985
:1041F00006C18C31910509F42BC18D31910548F42C
:104200008A31910509F406C14B9711F00C949D2950
:104210001AC18E31910509F427C1809711F00C94D1
:104220009D2931C18336910509F427C6843691054D
:10423000D8F48435910509F49AC58535910550F473
:104240008235910509F48CC58335910511F00C94E4
:104250009D2989C58535910509F4A5C58C3591053C
:1042600011F00C949D29C0C58A36910509F45CC5EE
:104270008B36910550F48836910509F45DC1893675
:10428000910511F00C949D2907C28D36910509F412
:104290000DC28F36910509F430C68B36910511F0A9
:1042A0000C949D2953C58E3C910509F468C78F3C39
:1042B0009105E8F58E3B910509F4E9C38F3B910523
:1042C000D8F48537910509F435C68637910550F441
:1042D0008337910509F424C68437910511F00C94B5
:1042E0009D297DC48737910509F435C68C38910521
:1042F00011F00C949D2996C18B3C910509F4E3C6FD
:104300008C3C910550F4893C910509F450C68A3CD7
:10431000910511F00C949D2990C68C3C910509F4EF
:10432000E5C68D3C910511F00C949D2925C7B1E09F
:1043300080399B0709F498C7E1E081399E07E0F4D2
:104340008D3D910509F480C78E3D910550F48F3C59
:10435000910509F418C78C3D910511F00C949D2925
:1043600061C7F1E08F329F0709F4AAC48E559140CE
:1043700011F00C949D29CAC731E0843F930709F4DA
:10438000ACC741E0853F940750F451E0813995076F
:1043900009F46DC78259914009F0CFC76BC7B1E0EE
:1043A000863F9B0709F4AFC7E1E0863F9E0708F40C
:1043B0009CC7875F914009F0C0C7DEC682ED9CE0D4
:1043C0000E94797BBAC782ED9CE00E94EC7EB5C763
:1043D00082ED9CE00E94AF79B0C717FFAEC782EDB7
:1043E0009CE060E00E94078AD601D3966D917C9193
:1043F000D49782ED9CE040E00E94E27A9EC782ED75
:104400009CE00E94C77999C782ED9CE060E00E9421
:10441000387E93C712FF91C7F601478D50A161A165
:1044200072A180913C0D882309F487C74093330D16
:104430005093340D6093350D7093360D82E19DE0FD
:104440000E9498877AC782ED9CE00E94BD7A75C76A
:1044500017FF73C7D601D3966D917C91D49782EDE7
:104460009CE00E947E7A69C717FF67C782ED9CE0D7
:1044700060E00E94078AF60163A974A982ED9CE0BE
:104480000E942F7A5AC717FF58C782ED9CE060E060
:104490000E94078AD601D3966D917C91D49782EDC4
:1044A0009CE00E94F37949C712FF47C713FF45C735
:1044B000F601878D90A1A1A1B2A1B7FD3EC78F3FA4
:1044C0009105A105B10511F00CF037C703A114A1A6
:1044D00020E030E0F901EE0FFF1FE155FE4FE491BF
:1044E0008E2F90E08017910709F427C72F5F3F4F69
:1044F0002833310579F717FD20C7802F61E00E942E
:1045000058C5802FD6015F966C910E94D5C5F601E3
:10451000678D70A1802F0E94DAC480EB94E0B8010F
:104520000E94FA2AD6015F966D917C9190978CEB50
:1045300094E00E94C22A01C70E94EA3A882309F047
:10454000FCC60E9421C46093400470934104809390
:104550004204909343048091270283FDEEC6F60146
:104560008081918193FD0AC092FF0AC0878D90A13E
:10457000A1A1B2A10097A105B10511F40E94D11C1F
:10458000D6018D919C91119792FFD7C65F968D9021
:104590009D90AD90BC9092979C012070317091FFDE
:1045A0001EC05E960C91232B11F410E00FC010E09A
:1045B000F601628D738D848D958D20E030E040E0B2
:1045C00050E00E9416C918160CF411E0C501B401A0
:1045D0000E94AAC7402F212F0E94373FAEC6E0910C
:1045E0007502F09176020081232B11F410E011C0C6
:1045F00010E0D6015A966D917D918D919C915D97B9
:1046000020E030E040E050E00E9416C918160CF49B
:1046100011E0C501B4010E94AAC7402F212F0E94BA
:10462000373F8BC60E94EA3A882309F086C60E946B
:1046300021C460934004709341048093420490939A
:1046400043048091270283FD78C6F6018081918121
:1046500092FF73C6E78CF0A001A112A190FD02C0E9
:10466000BB2412C0BB24D6015A966D917D918D91C9
:104670009C915D9720E030E040E050E00E9416C938
:10468000181614F4BB24B394C801B7010E94AAC73A
:104690004B2D0E94733B51C683E0169507958A9572
:1046A000E1F7802F81700E944D1C47C60E94EA3AB4
:1046B000882309F042C60E9421C46093400470938D
:1046C000410480934204909343048091270283FD28
:1046D00034C68EE69FE065E072E040E00E945199AA
:1046E0008EE69FE00E94E5B60E94D11C8090750284
:1046F00090907602F6012081318131FF07C0868DCE
:10470000882321F41FE1812E11E0912E32FF27C072
:10471000D6015F96ED90FD900D911C919297F4015A
:10472000A08030FD02C0BB2412C0BB24D6015A9623
:104730006D917D918D919C915D9720E030E040E0FE
:1047400050E00E9416C9181614F4BB24B394C80193
:10475000B7010E94AAC74A2D2B2D0E94373FF401B2
:1047600064A575A586A597A520A931A942A953A935
:104770000E9441C67B018C0120E030E040E050E027
:104780000E9416C918165CF4C801B70120E030E099
:1047900040E050E40E9408C7882364F4CEC5C801F5
:1047A000B70120E030E040E050EC0E9416C9181636
:1047B0000CF4C3C53324D4019A962D913C919B9758
:1047C00098968D919C9199978217930714F43324AE
:1047D00033940E9421C469A77AA78BA79CA744247D
:1047E0005524320110E00E9421C46DA37EA38FA343
:1047F00098A7DC01CB0129A53AA54BA55CA5821B96
:10480000930BA40BB50B895E9340A040B04058F0C9
:1048100080E00E944D1C8DA19EA1AFA1B8A589A7E3
:104820009AA7ABA7BCA70E94B41C80917502909177
:1048300076028816990609F067C0D4019396ED9028
:10484000FC9094971E141F040CF05EC0112309F015
:104850005BC0332009F458C091966D917C9192977A
:10486000882777FD8095982F0E94AAC79B01AC01ED
:10487000F40164A575A586A597A50E9416C918160A
:104880000CF042C000D000D000D00DB71EB70F5FB3
:104890001F4F662777276E197F09882777FD809538
:1048A000982F0E94AAC72091E7013091E80140911A
:1048B000E9015091EA010E94B8C90E9477C75B01E3
:1048C0006C01F40187859089A189B289F801808300
:1048D0009183A283B3831482158260E070E080E04C
:1048E00090E020E030E040E050E0EE24FF2487013B
:1048F0000E94166A11E02DB73EB72A5F3F4F0FB6F0
:10490000F8943EBF0FBE2DBF4114510461047104E1
:1049100009F053C03320C9F0D401D0966D917D9138
:104920008D919C91D39720E030E040E85FE30E94B6
:1049300041C69B01AC01F40164A575A586A597A5A8
:104940000E9416C987FF1AC04ECFD401D0966D9130
:104950007D918D919C91D39720E030E040E85FE31A
:104960000E9442C69B01AC01F40164A575A586A511
:1049700097A50E9408C718160CF435CFD4015F968E
:104980006D917C919097882777FD8095982F28EEE0
:1049900033E040E050E00E948ECA2B013C012DA183
:1049A0003EA14FA158A5420E531E641E751E411410
:1049B00051046104710409F416CFD301C2012DA181
:1049C0003EA14FA158A5821B930BA40BB50B8050A1
:1049D0009449A543B74708F406CF112309F44AC008
:1049E00080917502909176028816990609F042C06E
:1049F00000D000D000D00DB71EB70F5F1F4FD401FD
:104A000093966D917C919497882777FD8095982F48
:104A10000E94AAC72091E7013091E8014091E90185
:104A20005091EA010E94B8C90E9477C75B016C01EE
:104A3000F40187859089A189B289F80180839183E7
:104A4000A283B3831482158260E070E080E090E07E
:104A500020E030E040E050E0EE24FF2487010E9497
:104A6000166A2DB73EB72A5F3F4F0FB6F8943EBF88
:104A70000FBE2DBF1092AE0F0E9421C46093400460
:104A800070934104809342049093430456C423FDE1
:104A900054C48EE69FE069EF71E040E00E945199B6
:104AA0008EE69FE00E94E5B60E94D11CD6018D9152
:104AB0009C91119792FF21C05F96ED90FD900D9112
:104AC0001C91929790FD02C0BB2410C0BB24F6013C
:104AD000628D738D848D958D20E030E040E050E054
:104AE0000E9416C9181614F4BB24B394C801B70168
:104AF0000E94AAC74B2D0E94733B60919201709156
:104B000093018091940190919501209196013091AB
:104B1000970140919801509199010E9441C67B01F3
:104B20008C0120E030E040E050E00E9416C91816E9
:104B30005CF4C801B70120E030E040E450E40E949A
:104B400008C7882364F4F9C3C801B70120E030E046
:104B500040E450EC0E9416C918160CF4EEC30E94F3
:104B600021C47B018C0114C00E9421C46E197F09ED
:104B7000800B910B695E73408040904038F080E07C
:104B80000E944D1C0E9421C47B018C010E94B41C18
:104B9000609192017091930180919401909195019F
:104BA00020E030E040E05FE30E9442C620919601A1
:104BB0003091970140919801509199010E9408C746
:104BC00087FDD2CF1092AE0F0E9421C460934004A3
:104BD000709341048093420490934304AEC323FD39
:104BE000ACC30E9421C44B015C010E9421C468191E
:104BF00079098A099B09695E73408040904038F0CA
:104C000080E00E944D1C0E9421C44B015C010E9467
:104C1000B41CC090CC01D090CD01D6011B96ED9074
:104C2000FD900D911C911E97C801B70120E030E066
:104C300040EF51E40E9416C91816A4F4C801B70148
:104C4000F60127813085418552850E9441C69F77B4
:104C500020E030E040E85FE30E9416C9181614F423
:104C6000772402C077247394C090CE01D090CF01F6
:104C7000D6011B96ED90FD900D911C911E97C801D9
:104C8000B70120E030E040EF51E40E9416C9181649
:104C90009CF4C801B701F601278130854185528512
:104CA0000E9441C69F7720E030E040E85FE30E9429
:104CB00016C918160CF499CF772009F496CF3DC386
:104CC00012FD03C026E930E005C0D6015F962D91A4
:104CD0003C91909713FD03C0CC24DD240AC0F6015B
:104CE000C3A0D4A0F2E0CF16D1041CF0B2E0CB2ECA
:104CF000D12CF601EE0FFF1FE453FE4FE080F18050
:104D0000B901882777FD8095982F0E94AAC7AB012B
:104D1000BC01E3E016950795EA95E1F70170C7013C
:104D20002C2D0E94DA3B09C312FD03C08FEF90E0E7
:104D300005C0D6015F968D919C919097612F6695E5
:104D40006695669561700E94DF1CF7C2612F6695BB
:104D500066956695617080E090E00E94DF1CEDC270
:104D60001092BA0BEAC281E08093BA0BE6C212FF3E
:104D700014C0F601678D70A181A192A128EE33E0E5
:104D800040E050E00E948ECA6093D1017093D2013E
:104D90008093D3019093D401D0C20E94D11C81E0B2
:104DA0000E94D575CAC212FF16C0D6015F966D91DA
:104DB0007D918D919C91929728EE33E040E050E0F8
:104DC0000E948ECA60934404709345048093460405
:104DD00090934704B2C2109244041092450410927A
:104DE000460410924704A9C203FF0DC0F601828554
:104DF0009385A485B5858093DB019093DC01A09316
:104E0000DD01B093DE01D6018C9184FF0EC01E96A9
:104E10008D919D910D90BC91A02D8093DF01909379
:104E2000E001A093E101B093E201F601808185FFEA
:104E30000CC082899389A489B5898093E3019093FA
:104E4000E401A093E501B093E6010E947F76D601CC
:104E50008C9186FF72C2E0917502F09176025696AF
:104E60002D913D914D915C915997218732874387D0
:104E7000548780810E94FD3F60C212FD07C040E15F
:104E8000842E47E2942EA12CB12C0DC0F601678D23
:104E900070A181A192A128EE33E040E050E00E9491
:104EA0008ECA4B015C0103FD5E9A04FD5E9A05FD0E
:104EB000159A0E9421C47B018C01E80CF91C0A1D83
:104EC0001B1D02C00E9423760E9421C4A8019701E5
:104ED000261B370B480B590BDA01C901805A96483B
:104EE000A140B04078F3D6013C9133FD5E9834FD8B
:104EF0005E9835FF22C2159820C212FF04C0F60149
:104F0000878D809327028091270283FF16C260E07D
:104F100070E080E090E040E020E00E94373F0DC26A
:104F200086E192E00E94262B0E946A1B06C20E9424
:104F3000341A03C217FF01C2D601D3966D917C913A
:104F4000D4978EE69FE040E00E947D998EE69FE038
:104F50000E94E5B6F2C10E94D11C87EC94E00E9449
:104F60009F2A329B03C084EC94E002C081EC94E061
:104F70000E949F2A85ED94E00E949F2A339B03C0E4
:104F800084EC94E002C081EC94E00E949F2A83EEBE
:104F900094E00E949F2A349B03C084EC94E002C0FA
:104FA00081EC94E00E949F2A0E945B1BC6C103FF14
:104FB0000DC0F60182859385A485B585809307028F
:104FC00090930802A0930902B0930A02D6018C9133
:104FD00084FF0EC01E968D919D910D90BC91A02DC9
:104FE00080930B0290930C02A0930D02B0930E02DB
:104FF000F601808185FF0CC082899389A489B589D7
:1050000080930F0290931002A0931102B0931202AA
:10501000D6018C9186FF0EC056968D919D910D9074
:10502000BC91A02D8093130290931402A0931502BB
:10503000B09316020E947F7680C103FF0DC0F60177
:1050400082859385A485B585809317029093180275
:10505000A0931902B0931A02D6018C9184FF0EC05E
:105060001E968D919D910D90BC91A02D80931B0259
:1050700090931C02A0931D02B0931E02F601808142
:1050800085FF0CC082899389A489B58980931F020A
:1050900090932002A0932102B0932202D6018C911A
:1050A00086FF0EC056968D919D910D90BC91A02DBE
:1050B0008093230290932402A0932502B0932602AA
:1050C0000E947F763AC112FF38C1F601278D30A1C8
:1050D00041A152A112161306140615061CF02093C6
:1050E0001C012BC181E080931C0127C180917502B6
:1050F0009091760212FD03C0FC01B59610C0F60136
:10510000878D90A1A1A1B2A1B7FD17C10097A105FC
:10511000B10519F4E4E4F1E002C0EBE8F1E003FFCB
:105120000BC0D6011A962D913D914D915C911D9722
:10513000228F338F448F558FD6018C9184FF0AC004
:105140001E962D913D914D915C915197268F378FF1
:1051500040A351A3D6018C9185FF0AC052962D9190
:105160003D914D915C91559722A333A344A355A340
:10517000CF010E941A38E1C00E94432DDEC0C60153
:105180000E94AE35DAC003FF0DC0F601828593851B
:10519000A485B58580934E0C90934F0CA093500C32
:1051A000B093510CD6018C9186FF11C0E09175022D
:1051B000F091760256962D913D914D915C915997C3
:1051C000278B308F418F528F80810E94FD3FF601E7
:1051D000808185FF0CC082899389A489B5898093D9
:1051E000520C9093530CA093540CB093550C4091D7
:1051F0004E0C50914F0C6091500C7091510C81EFFE
:1052000094E022E00E94FD2B4091520C5091530CEF
:105210006091540C7091550C87EF94E022E00E944D
:10522000122C8BC012FD05C024E630E040E050E0B7
:1052300007C0D6015F962D913D914D915C9192975B
:10524000C9010E94D21979C012FD05C024E630E0E0
:1052500040E050E005C0F601278D30A141A152A1E8
:10526000C9010E94BD1969C00E94D11C66C00E947C
:105270000A6C63C010FF08C0D6015A96CD90DD902D
:10528000ED90FC905D9708C0C090460CD090470C04
:10529000E090480CF090490CB80134E076956795A1
:1052A0003A95E1F76170A80125E0569547952A9552
:1052B000E1F74170980196E0369527959A95E1F7C8
:1052C000217083E0169507958A95E1F7802F81700C
:1052D000870176010E94267530C080E00E94BD2FB4
:1052E00080ED97E00E94452B28C00E94A432E091F7
:1052F0007502F091760280810E94FD3F80EF97E079
:105300000E94452B1AC00E94293617C087EE91E0F3
:105310000E94262B12C011FF07C00E94D11CF6016B
:10532000868D0E94FD3F09C022FF07C086ED93E0F5
:105330000E949F2AC6010E94A544E0960FB6F894E9
:10534000DEBF0FBECDBFCF91DF911F910F91FF90B8
:10535000EF90DF90CF90BF90AF909F908F907F9015
:105360006F905F904F903F902F900895CF93DF9371
:105370000E946D4A0E949444EC018EE69FE00E94D8
:105380004B9A2097D1F080913D0D882381F0888140
:1053900081FF04C08E819F814D9791F082ED9CE04A
:1053A000BE010E941F7CCE010E94634903C0CE0152
:1053B0000E940E1DCE010E9474490E942376D8CF10
:1053C00082ED9CE00E945E7AEECFCF93DF9320C007
:1053D00080913D0D882381F0888181FF04C08E81FA
:1053E0009F814D9739F182ED9CE0BE010E941F7CA8
:1053F000CE010E94634903C0CE010E940E1DCE0162
:105400000E9474490E94B41C8EE69FE00E944B9A51
:105410008091810B882329F40E949444EC01009729
:1054200071F00E946D4A8EE69FE00E944B9A209791
:1054300079F6E8CF82ED9CE00E945E7AD9CFDF91C9
:10544000CF910895CF93DF93EC0105C0219683E2BD
:1054500094E00E94074F68816623C1F7DF91CF91E6
:105460000895AF92BF92CF92DF92EF92FF920F9387
:105470001F93DF93CF93CDB7DEB72B970FB6F8947A
:10548000DEBF0FBECDBFC62ED92E1B869BE0A92E38
:10549000B12CAC0EBD1E6C2D9D2D2AE030E040E0FD
:1054A00050E00E94E1CAD52E7901042F152F80E328
:1054B000C80EC801B7012AE030E040E050E00E9489
:1054C0008ECAC61AF501C2925F01CE2C7F2D802FA5
:1054D000E114F10401051105F1F6CF010E94222A21
:1054E0002B960FB6F894DEBF0FBECDBFCF91DF91E4
:1054F0001F910F91FF90EF90DF90CF90BF90AF90F2
:105500000895EF92FF920F931F937B018C0197FFF9
:105510000DC083E294E06DE20E94074F1095009564
:10552000F094E094E11CF11C011D111DC801B701AC
:105530000E94312A1F910F91FF90EF900895CF9311
:10554000DF93EC0104C083E294E00E94074FFE0168
:10555000649121966623B9F7DF91CF910895EF9278
:10556000FF920F931F937A018B010E949F2AC8011B
:10557000B7010E94312A0E945B1B1F910F91FF907F
:10558000EF900895EF92FF920F931F937B010E947B
:105590009F2A0027F7FC0095102FC801B7010E9431
:1055A000812A0E945B1B1F910F91FF90EF9008953D
:1055B000EF92FF920F931F937A018B010E949F2A13
:1055C000C801B7010E94312A1F910F91FF90EF90FF
:1055D0000895EF92FF920F931F937A018B010E941F
:1055E0009F2AC801B7010E94812A1F910F91FF9045
:1055F000EF900895EF92FF920F931F937B010E940B
:105600009F2A0027F7FC0095102FC801B7010E94C0
:10561000812A1F910F91FF90EF9008950F931F9390
:105620008B010E949F2AC8010E94222A1F910F917C
:1056300008950F931F938B010E949F2AC8010E9417
:10564000222A0E945B1B1F910F9108950E949F2A9E
:105650000E945B1B08950F931F938C0181ED92E0D4
:105660000E949F2AC8010E94262B1F910F91089526
:105670000F931F938C0188ED92E00E949F2AC8012E
:105680000E94262B1F910F9108950F931F938C0159
:1056900088ED92E00E949F2AC8010E949F2A1F91D4
:1056A0000F9108959F92AF92BF92CF92DF92EF92A7
:1056B000FF920F931F93CF93DF937B018C01942E66
:1056C000A80197010E9472CA882319F089EC92E020
:1056D00020C0C0E0D0E057016801E894D7F8C601C7
:1056E000B5012FEF3FEF4FE75FE70E9472CA8823B3
:1056F00051F4C601B5012FEF3FEF4FE75FE70E947E
:1057000008C7181614F0C1E0D0E0219729F08DECFD
:1057100092E00E949F2A65C0C801B70120E030E0F6
:1057200040E050E00E9408C788234CF483E294E0F4
:105730006DE20E94074F17FB109517F9109520E0B6
:1057400030E040E05FE3DD240BC0CA01B90120E096
:1057500030E040E251E40E940FC79B01AC01D394BA
:10576000D91498F3C801B7010E9442C65B016C01CD
:105770000E947CC77B018C010E94312A992029F06C
:1057800083E294E06EE20E94074FC801B7010E94D5
:10579000A8C79B01AC01C601B5010E9441C61FC04C
:1057A00020E030E040E251E40E94B8C97B018C0166
:1057B0000E9477C75B016C01CC24B7FCC094DC2C41
:1057C000C601B5010E94812AC601B5010E94AAC77F
:1057D0009B01AC01C801B7010E9441C69A9499206F
:1057E000F9F6DF91CF911F910F91FF90EF90DF902D
:1057F000CF90BF90AF909F900895DF92EF92FF926D
:105800000F931F937A018B01D22E0E949F2AC80109
:10581000B7014D2D0E94522B1F910F91FF90EF90D9
:10582000DF900895DF92EF92FF920F931F937A011A
:105830008B01D22E0E949F2AC801B7014D2D0E94D4
:10584000522B0E945B1B1F910F91FF90EF90DF90F6
:1058500008959C01F999FECF32BD21BDF89A80B51B
:1058600008959C01F999FECF1FBA32BD21BD60BDDC
:105870000FB6F894FA9AF99A0FBE0895885C904092
:1058800022E08835920778F464E670E00E94BACA94
:105890006F5F7F4F87E598E00E94FA2A83E294E0E9
:1058A00060E20E94074F08950F931F93CF93DF93F9
:1058B000EC018B018DE598E0BE010E94FA2A83E29B
:1058C00094E060E20E94074FF999FECFD2BDC1BDBE
:1058D000F89A60B570E0882777FD8095982F0E9430
:1058E000812A83E294E060E20E94074FCE010E9489
:1058F0003E2CC8010E94262BDF91CF911F910F9162
:105900000895CF92DF92EF92FF920F931F938C0135
:105910006B0184E698E0B8010E94FA2A83E2E82E3F
:1059200084E0F82EC70160E20E94074FC80169E2D7
:105930007CE20E943319AA2797FDA095BA2FBC01DB
:10594000CD010E94812AC70160E20E94074FC80171
:105950000E943E2CC6010E94262B1F910F91FF90A2
:10596000EF90DF90CF900895CF92DF92EF92FF9269
:105970000F931F938C016B018BE698E0B8010E9496
:10598000FA2A93E2E92E94E0F92EC70160E20E9420
:10599000074FC80169E27CE20E940D190E94812A2A
:1059A000C70160E20E94074FC8010E943E2CC60159
:1059B0000E94262B1F910F91FF90EF90DF90CF90C8
:1059C0000895F999FECF12BC11BCF89A80B58131C7
:1059D00071F48BE490E069E27CE20E940D1960931F
:1059E000D5017093D6018093D7019093D801089583
:1059F000DF93CF9300D000D0CDB7DEB7BC01CE018E
:105A0000019644E050E029E23CE20E94F11829812D
:105A10003A814B815C81B901CA010F900F900F90C0
:105A20000F90CF91DF910895BF92CF92DF92EF92C6
:105A3000FF920F931F938C016B01B42E82E798E0C5
:105A4000B8010E94FA2A23E2E22E24E0F22EC701D6
:105A500060E20E94074FC8010E94F82C4B2D0E9463
:105A6000522BC70160E20E94074FC8010E943E2CE2
:105A7000C6010E94262B1F910F91FF90EF90DF909F
:105A8000CF90BF9008958BE490E069E778E00E94A2
:105A9000B42C81E890E062E878E043E00E94142DA5
:105AA0008DE790E067E978E00E94B42C8FE490E005
:105AB0006AEA78E00E94B42C83E590E068EC78E034
:105AC0000E94B42C83E090E06BEA79E044E00E940D
:105AD000142D87E090E06FEB79E044E00E94142DF4
:105AE0008BE090E063ED79E044E00E94142D8FE0BC
:105AF00090E067EE79E043E00E94142D83E190E0AE
:105B000063E07AE043E00E94142D87E190E06FE1CA
:105B10007AE043E00E94142D8BE190E06BE37AE0A1
:105B200043E00E94142D8FE190E069E57AE043E0C4
:105B30000E94142D83E290E067E77AE043E00E9440
:105B4000142D87E290E067E879E043E00E94142D8D
:105B50008FE290E068E979E043E00E94142D85E847
:105B600090E061EF78E043E00E94142D89E890E036
:105B700061E079E043E00E94142D8DE890E061E15E
:105B800079E043E00E94142D81E990E061E279E040
:105B900043E00E94142D85E990E063E379E043E05F
:105BA0000E94142D89E990E065E479E043E00E94C9
:105BB000142D83E390E065E97AE043E00E94142D20
:105BC00087E390E062EB7AE043E00E94142D8BE3E0
:105BD00090E06FEC7AE043E00E94142D8FE390E0B8
:105BE0006CEE7AE043E00E94142D83E490E060E1E3
:105BF0007BE043E00E94142D87E490E064E37BE0C7
:105C000043E00E94142D8AE690E065E07CE00E946B
:105C1000542C8BE690E06CE17CE00E94542C8CE7E5
:105C200090E06EE27CE00E94542C8CE690E060E410
:105C30007CE043E00E94142D80E790E06FE47CE07C
:105C400043E00E94142D84E790E06EE57CE043E0A1
:105C50000E94142D88E790E06DE67CE00E94542CB1
:105C600088EC90E067E87CE043E00E94142D8CEC27
:105C700090E064E97CE043E00E94142D80ED90E028
:105C800069EA7CE043E00E94142D84ED90E06FEB24
:105C90007CE043E00E94142D88ED90E065ED7CE00F
:105CA0000E94542C89ED90E068EE7CE00E94542C18
:105CB00085EF90E066EF7CE00E94542C8AED90E046
:105CC00064E07DE044E00E94142D8EED90E069E1F7
:105CD0007DE044E00E94142D82EE90E064E27DE0DD
:105CE00044E00E94142D86EE90E06FE27DE00E9479
:105CF000542C87EE90E065E47DE00E94B42C8BEE9E
:105D000090E066E57DE00E94B42C8FEE90E067E6BF
:105D10007DE00E94812C8AEF90E060E87DE00E94A7
:105D2000812C8CEF90E066EA7DE00E94812C8EEF62
:105D300090E06CEC7DE00E94542C0895DF93CF93AB
:105D400000D000D0CDB7DEB749835A836B837C8304
:105D5000BE016F5F7F4F44E050E021E33CE20E94D0
:105D600049190F900F900F900F90CF91DF910895E8
:105D700088E293E040E050E060EA70E40E949E2EEA
:105D80008CE293E040E050E060E070E40E949E2EE0
:105D900088E493E040E050E068E473E40E949E2EC3
:105DA00080E293E040E050E060E070E00E949E2ED0
:105DB00084E293E040E050E060E070E00E949E2EBC
:105DC00080E393E040E050E066E173E40E949E2EA1
:105DD00084E393E040E050E060EA70EC0E949E2E85
:105DE00088E393E040E050E066E173E40E949E2E79
:105DF0008CE393E040E050E060E273E40E949E2E6A
:105E000080E493E040E050E060EF71EC0E949E2E51
:105E100084E493E040E050E060E273E40E949E2E50
:105E200081EA93E040E050E060E870E40E949E2E3A
:105E30000895EF92FF920F931F936091640C7091FD
:105E4000650C8091660C9091670C20E030E040E09A
:105E500050E00E9408C7882309F48AC00E9421C428
:105E60002091600C3091610C4091620C5091630C58
:105E7000621B730B840B950B28EE33E040E050E07F
:105E80000E94E1CA79018A018DE790E069E27CE233
:105E90000E940D19E60EF71E081F191F8DE790E0EE
:105EA000B801A70121E33CE20E94651981E890E076
:105EB0000E94F82C7B018C016091640C7091650C40
:105EC0008091660C9091670C2FE632E143E85AE32B
:105ED0000E94B8C99B01AC01C801B7010E9442C62B
:105EE000AB01BC0181E890E00E949E2E80E090E032
:105EF000A0E0B0E08093640C9093650CA093660CD6
:105F0000B093670C0E9421C46093600C7093610C85
:105F10008093620C9093630C20E030E040E02836E0
:105F2000310539F0F999FECF32BD21BDF89A80B51F
:105F3000480F2F5F3F4F88E02030380781F7F999ED
:105F4000FECF88E690E092BD81BDF89A80B54817F3
:105F500069F0F999FECF1FBA88E690E092BD81BD45
:105F600040BD0FB6F894FA9AF99A0FBE0E946A1BC8
:105F70001F910F91FF90EF9008951F93182F40915C
:105F8000D5015091D6016091D7017091D8018BE471
:105F900090E021E33CE20E94651940914404509155
:105FA000450460914604709147048FE490E021E33A
:105FB0003CE20E9465194091D1015091D20160915B
:105FC000D3017091D40183E590E021E33CE20E948B
:105FD00065194091DB015091DC016091DD01709108
:105FE000DE0183E090E00E949E2E4091DF015091FF
:105FF000E0016091E1017091E20187E090E00E9490
:106000009E2E4091E3015091E4016091E501709171
:10601000E6018BE090E00E949E2E4091EB015091B2
:10602000EC016091ED017091EE018FE090E00E9433
:106030009E2E4091EF015091F0016091F10170911D
:10604000F20183E190E00E949E2E4091F301509175
:10605000F4016091F5017091F60187E190E00E94F2
:106060009E2E4091FB015091FC016091FD017091C9
:10607000FE018BE190E00E949E2E4091FF01509125
:10608000000260910102709102028FE190E00E9493
:106090009E2E40910302509104026091050270917E
:1060A000060283E290E00E949E2E40914E0C509199
:1060B0004F0C6091500C7091510C87E290E00E945F
:1060C0009E2E4091520C5091530C6091540C709143
:1060D000550C8FE290E00E949E2E40910702509155
:1060E00008026091090270910A0283E390E00E9425
:1060F0009E2E40910B0250910C0260910D02709106
:106100000E0287E390E00E949E2E40910F02509174
:10611000100260911102709112028BE390E00E94D4
:106120009E2E4091170250911802609119027091B1
:106130001A028FE390E00E949E2E40911B02509124
:106140001C0260911D0270911E0283E490E00E9487
:106150009E2E40911F025091200260912102709169
:10616000220287E490E00E949E2E20919E01F999E0
:10617000FECF1FBA8AE690E092BD81BD20BD0FB66A
:10618000F894FA9AF99A0FBE2091A301F999FECFDB
:106190001FBA8BE690E092BD81BD20BD0FB6F8948A
:1061A000FA9AF99A0FBE2091A401F999FECF1FBA6D
:1061B0008CE790E092BD81BD20BD0FB6F894FA9AAD
:1061C000F99A0FBE4091A5015091A6016091A701D7
:1061D0007091A8018CE690E00E949E2E4091A9014A
:1061E0005091AA016091AB017091AC0180E790E001
:1061F0000E949E2E4091AD015091AE016091AF0181
:106200007091B00184E790E00E949E2E2091B10130
:10621000F999FECF1FBA88E790E092BD81BD20BDFD
:106220000FB6F894FA9AF99A0FBE4091320C509139
:10623000330C6091340C7091350C85E890E00E942D
:106240009E2E40913A0C50913B0C60913C0C709109
:106250003D0C89E890E00E949E2E4091420C5091A6
:10626000430C6091440C7091450C8DE890E00E94C5
:106270009E2E40912E0C50912F0C6091300C7091FD
:10628000310C81E990E00E949E2E4091360C509195
:10629000370C6091380C7091390C85E990E00E94C0
:1062A0009E2E40913E0C50913F0C6091400C70919D
:1062B000410C89E990E00E949E2E8DE990E040E03B
:1062C00050E060E070E00E949E2E81EA90E040E0A5
:1062D00050E060E070E00E949E2E85EA90E040E091
:1062E00050E060E070E00E949E2E409128015091A5
:1062F000290160912A0170912B0188EC90E00E94A5
:106300009E2E40912E0150912F016091300170918D
:1063100031018CEC90E00E949E2E4091360150910C
:106320003701609138017091390180ED90E00E9451
:106330009E2E409132015091330160913401709151
:10634000350184ED90E00E949E2E20915701F9992D
:10635000FECF1FBA88ED90E092BD81BD20BD0FB683
:10636000F894FA9AF99A0FBE20915C01F999FECF40
:106370001FBA89ED90E092BD81BD20BD0FB6F894A3
:10638000FA9AF99A0FBE20915D01F999FECF1FBAD2
:1063900085EF90E092BD81BD20BD0FB6F894FA9ACA
:1063A000F99A0FBE40915E0150915F0160916001CA
:1063B000709161018AED90E00E949E2E40916201F1
:1063C0005091630160916401709165018EED90E0E0
:1063D0000E949E2E40916601509167016091680174
:1063E0007091690182EE90E00E949E2E20916A01D8
:1063F000F999FECF1FBA86EE90E092BD81BD20BD17
:106400000FB6F894FA9AF99A0FBE40912001509174
:106410002101609122017091230187EE90E021E338
:106420003CE20E9465194091240150912501609140
:106430002601709127018BEE90E021E33CE20E945F
:10644000651960913E0170913F018FEE90E041E34C
:106450005CE20E948B1960914001709141018AEFCA
:1064600090E041E35CE20E948B19609142017091DF
:1064700043018CEF90E041E35CE20E948B19209194
:106480008901F999FECF1FBA8EEF90E092BD81BDD0
:1064900020BD0FB6F894FA9AF99A0FBE81EF90E0FA
:1064A00040E050E060E070E00E949E2E86EF90E0B9
:1064B00040E050E060E070E00E949E2E1123A1F0C9
:1064C0008DE790E040E050E060E070E021E33CE2E6
:1064D0000E94651981E890E040E050E060E070E0E3
:1064E0000E949E2E0E94B82EF999FECF1FBA89E60F
:1064F00090E092BD81BD87E080BD0FB6F894FA9A16
:10650000F99A0FBE20E030E040E02836310539F03E
:10651000F999FECF32BD21BDF89A80B5480F2F5FA3
:106520003F4F88E02030380781F7F999FECF1FBA36
:1065300088E690E092BD81BD40BD0FB6F894FA9A0E
:10654000F99A0FBE1F9108951F93F999FECF89E61E
:1065500090E092BD81BDF89A10B58BE490E069E2BD
:106560007CE20E940D196093D5017093D60180934F
:10657000D7019093D8018FE490E069E27CE20E9419
:106580000D196093440470934504809346049093DE
:10659000470483E590E069E27CE20E940D19609374
:1065A000D1017093D2018093D3019093D40183E001
:1065B00090E00E94F82C6093DB017093DC018093E3
:1065C000DD019093DE0187E090E00E94F82C60935B
:1065D000DF017093E0018093E1019093E2018BE091
:1065E00090E00E94F82C6093E3017093E4018093A3
:1065F000E5019093E6018FE090E00E94F82C609313
:10660000EB017093EC018093ED019093EE0183E137
:1066100090E00E94F82C6093EF017093F00180935A
:10662000F1019093F20187E190E00E94F82C6093D1
:10663000F3017093F4018093F5019093F6018BE1DF
:1066400090E00E94F82C6093FB017093FC01809312
:10665000FD019093FE018FE190E00E94F82C609381
:10666000FF0170930002809301029093020283E283
:1066700090E00E94F82C60930302709304028093D0
:1066800005029093060287E290E00E94F82C609346
:106690004E0C70934F0C8093500C9093510C8FE2E2
:1066A00090E00E94F82C6093520C7093530C8093EE
:1066B000540C9093550C83E390E00E94F82C609367
:1066C0000702709308028093090290930A0287E3FD
:1066D00090E00E94F82C60930B0270930C02809360
:1066E0000D0290930E028BE390E00E94F82C6093D1
:1066F0000F027093100280931102909312028FE3A5
:1067000090E00E94F82C6093170270931802809317
:10671000190290931A0283E490E00E94F82C60938F
:106720001B0270931C0280931D0290931E0287E44B
:1067300090E00E94F82C60931F02709320028093D7
:10674000210290932202F999FECF8AE690E092BD51
:1067500081BDF89A80B580939E01F999FECF8BE6B2
:1067600090E092BD81BDF89A80B58093A301F9991C
:10677000FECF8CE790E092BD81BDF89A80B5809302
:10678000A4018CE690E00E94F82C6093A501709320
:10679000A6018093A7019093A80180E790E00E9452
:1067A000F82C6093A9017093AA018093AB01909398
:1067B000AC0184E790E00E94F82C6093AD017093E7
:1067C000AE018093AF019093B001F999FECF88E7B5
:1067D00090E092BD81BDF89A80B58093B10185E8C3
:1067E00090E00E94F82C6093320C7093330C8093ED
:1067F000340C9093350C89E890E00E94F82C60935B
:106800003A0C70933B0C80933C0C90933D0C8DE8BC
:1068100090E00E94F82C6093420C7093430C80939C
:10682000440C9093450C81E990E00E94F82C609311
:106830002E0C70932F0C8093300C9093310C85E9C3
:1068400090E00E94F82C6093360C7093370C809384
:10685000380C9093390C89E990E00E94F82C6093F1
:106860003E0C70933F0C8093400C9093410C88EC4D
:1068700090E00E94F82C6093280170932901809386
:106880002A0190932B018CEC90E00E94F82C6093ED
:106890002E0170932F01809330019093310180ED90
:1068A00090E00E94F82C609336017093370180933A
:1068B00038019093390184ED90E00E94F82C6093A8
:1068C0003201709333018093340190933501F9992B
:1068D000FECF88ED90E092BD81BDF89A80B580939F
:1068E0005701F999FECF89ED90E092BD81BDF89AEC
:1068F00080B580935C01F999FECF85EF90E092BD61
:1069000081BDF89A80B580935D018AED90E00E9488
:10691000F82C60935E0170935F0180936001909307
:1069200061018EED90E00E94F82C609362017093FB
:106930006301809364019093650182EE90E00E9470
:10694000F82C6093660170936701809368019093BF
:106950006901F999FECF86EE90E092BD81BDF89A6B
:1069600080B580936A0187EE90E069E27CE20E9444
:106970000D1960932001709321018093220190935F
:1069800023018BEE90E069E27CE20E940D19609396
:1069900024017093250180932601909327018FEEA7
:1069A00090E069E27CE20E94331990933F0180936A
:1069B0003E018AEF90E069E27CE20E9433199093F5
:1069C0004101809340018CEF90E069E27CE20E94FB
:1069D00033199093430180934201123068F0F99982
:1069E000FECF8EEF90E092BD81BDF89A80B5809386
:1069F0008901173009F46CC083E398E00E94382BBA
:106A0000133008F058C088E293E040E050E060EABC
:106A100070E40E949E2E8CE293E040E050E060E043
:106A200070E40E949E2E88E493E040E050E068E429
:106A300073E40E949E2E80E293E040E050E060E02C
:106A400070E00E949E2E84E293E040E050E060E01F
:106A500070E00E949E2E80E393E040E050E066E10B
:106A600073E40E949E2E84E393E040E050E060EAED
:106A700070EC0E949E2E88E393E040E050E066E1D7
:106A800073E40E949E2E8CE393E040E050E060E2CD
:106A900073E40E949E2E80E493E040E050E060EFBB
:106AA00071EC0E949E2E84E493E040E050E060E2AE
:106AB00073E40E949E2E173040F481EA93E040E098
:106AC00050E060E870E40E949E2E80E00E94BD2F9E
:106AD0000E947F760E9461381F9108950F931F9343
:106AE00020E030E010E02836310539F0F999FECF8A
:106AF00032BD21BDF89A80B5180F2F5F3F4F88E057
:106B00002030380781F7F999FECF88E690E092BDF2
:106B100081BDF89A00B5F999FECF12BC11BCF89A64
:106B200080B5813129F4011719F40E94A43213C0F1
:106B3000F999FECF1FBA12BC11BC81E180BD0FB61E
:106B4000F894FA9AF99A0FBE0E94B82E80E00113C9
:106B500081E00E94BD2F1F910F910895FC0180815B
:106B6000918191FF42C093FF40C0268D2130D9F022
:106B7000213030F0223011F1233009F036C02BC023
:106B800092FF33C023A134A145A156A1878DF99965
:106B9000FECF1FBA32BD21BD80BD0FB6F894FA9A60
:106BA000F99A0FBE22C092FF20C0678D70A183A109
:106BB00094A141E35CE20E948B1917C092FF15C0BB
:106BC000478D50A161A172A183A194A121E33CE270
:106BD0000E9465190AC083FF08C0428553856485F9
:106BE000758583A194A10E949E2E20E030E040E0B4
:106BF0002836310539F0F999FECF32BD21BDF89A1A
:106C000080B5480F2F5F3F4F88E02030380781F76D
:106C1000F999FECF88E690E092BD81BDF89A80B5E3
:106C2000481769F0F999FECF1FBA88E690E092BD47
:106C300081BD40BD0FB6F894FA9AF99A0FBE0E9432
:106C4000A432E0917502F091760280810E94FD3FAE
:106C50000895AF92BF92CF92DF92EF92FF920F937F
:106C60001F9380E092ECA1E0B0E08093D501909377
:106C7000D601A093D701B093D8011092440410928A
:106C80004504109246041092470480E49EE7A5E074
:106C9000B0E08093D1019093D201A093D301B0933F
:106CA000D4010F2EF0E0EF2EF0E0FF2EF8EC0F2FC6
:106CB000F2E41F2FF02DE092DB01F092DC01009353
:106CC000DD011093DE01E092DF01F092E00100931C
:106CD000E1011093E20120E030E048EC53E420931E
:106CE000E3013093E4014093E5015093E60180E035
:106CF00090E0A0E8BFE38093E7019093E801A093C0
:106D0000E901B093EA012093EB013093EC01409349
:106D1000ED015093EE012093EF013093F001409389
:106D2000F1015093F20180E090E0A0E8B0E480939C
:106D3000F3019093F401A093F501B093F601E09272
:106D4000FB01F092FC010093FD011093FE01E09223
:106D5000FF01F092000200930102109302020F2E35
:106D6000F0E0AF2EF0E0BF2EF0E0CF2EF0E4DF2E0B
:106D7000F02DA0920302B0920402C0920502D092BC
:106D8000060220E030E040EA51E420934E0C3093BC
:106D90004F0C4093500C5093510C8DEC9CECACEC90
:106DA000BEE38093520C9093530CA093540CB09379
:106DB000550C80E090E0AAE7B4E48093070290933A
:106DC0000802A0930902B0930A0280930B029093E9
:106DD0000C02A0930D02B0930E02E0920F02F0920B
:106DE0001002009311021093120280E090E0AAEFCB
:106DF000B4E48093170290931802A0931902B09301
:106E00001A0280931B0290931C02A0931D02B09360
:106E10001E02E0921F02F0922002009321021093C2
:106E2000220210929E016FEF6093A30180E5809390
:106E3000A40180E090E0A4E4B3E48093A5019093E2
:106E4000A601A093A701B093A80180E090E0A4E080
:106E5000B2E48093A9019093AA01A093AB01B093EF
:106E6000AC0180E090E0A1E9B3E48093AD019093A0
:106E7000AE01A093AF01B093B0016093B10180E087
:106E800090E8A4E8B3E480932E0C90932F0CA09389
:106E9000300CB093310C80E090E0A6E6B3E4809330
:106EA000360C9093370CA093380CB093390C80E0DB
:106EB00090E0ABE6B3E480933E0C90933F0CA0933C
:106EC000400CB093410C80E090E0A4E3B2EC8093DE
:106ED000320C9093330CA093340CB093350C80E0BB
:106EE00090E0A0EAB0EC80933A0C90933B0CA09316
:106EF0003C0CB0933D0C80E090E0A0E0B0E08093CB
:106F0000420C9093430CA093440CB093450C80E04A
:106F100090E0A4EBB2E48093280190932901A09320
:106F20002A01B0932B0180E090E0A8E4B2E48093C2
:106F30002E0190932F01A0933001B0933101209343
:106F4000360130933701409338015093390180E086
:106F500090E8ABE3B5E48093320190933301A093C2
:106F60003401B093350183E08093570186EE80931E
:106F70005C0182E380935D0180E090E0A0EEB0E4EC
:106F800080935E0190935F01A0936001B0936101D3
:106F9000A0926201B0926301C0926401D092650137
:106FA00080E090E0A0E2B2E48093660190936701F4
:106FB000A0936801B093690160936A011092240163
:106FC00010922501109226011092270110922001A3
:106FD00010922101109222011092230181E090E091
:106FE00090933F0180933E0186E990E090934101A8
:106FF00080934001109243011092420160938901F5
:107000000E94B82E0E947F76E0917502F091760280
:1070100080810E94FD3F0E94613882E198E00E94D9
:10702000452B1F910F91FF90EF90DF90CF90BF9075
:10703000AF900895EF92FF920F931F93CF93DF933A
:10704000EC018B898130B1F5EE8CFF8C08A119A180
:10705000C801B70120E030E040E050E00E9408C7DE
:10706000882341F1688D70E080E090E00E94A8C71D
:1070700020E030E040E251E40E94B8C9A801970145
:107080000E940FC76FA378A789A79AA7698D70E0A0
:1070900080E090E00E94A8C720E030E040E251E4A8
:1070A0000E94B8C9A80197010E940FC76BA77CA7CF
:1070B0008DA79EA7DF91CF911F910F91FF90EF9029
:1070C00008958BE891E00E941A380895E091CE016E
:1070D000F091CF012781308541855285B901CA01E0
:1070E00008952F923F924F925F926F927F928F926C
:1070F0009F92AF92BF92CF92DF92EF92FF920F9347
:107100001F93CF93DF931C01DC0111964C91453303
:1071100038F44233F8F4842F81508C3058F50AC08B
:10712000443628F4413630F44C3321F513C044364C
:1071300009F510C0D1011296EC911297F0E0EE0F14
:10714000FF1FE159FD4F208131818CEF9FE0821BB1
:10715000930B0BC0D1011296EC911297F0E0EE0F59
:10716000FF1FE159FD4F8081918114969C938E936E
:10717000139705C08FEF9FE0F10194838383D101C2
:107180001396ED90FC901497453348F4423308F081
:1071900053C0842F81508C3008F000C107C04C339D
:1071A00009F4C9C0443609F0F9C0DEC090E0FC0122
:1071B000E35BF04F4491440FFC01EE0FFF1FE75AD1
:1071C000F04F25913491F90145905490F901329690
:1071D000659074900CEF1FE00E191F0982E029C022
:1071E000E82FF0E0EE0FFF1FE20FF31F8590949061
:1071F0008F5FE82FF0E08150EE0FFF1FE20FF31FCB
:10720000C591D491081519058CF4B301882777FD31
:107210008095982F0E94AAC75B016C01B801641980
:107220007509882777FD8095982F44C08E5F3E01B1
:1072300024018417A8F273C04E52842F90E0FC0101
:10724000E35BF04F4491440FFC01EE0FFF1FE75A40
:10725000F04F25913491F90145905490F9013296FF
:107260006590749082E058C0E82FF0E0EE0FFF1FA9
:10727000E20FF31F859094908F5FE82FF0E081502C
:10728000EE0FFF1FE20FF31FC591D491E814F9042C
:107290000CF03FC0B301882777FD8095982F0E949E
:1072A000AAC75B016C01E418F508B701882777FDD0
:1072B0008095982F0E94AAC77B018C01C619D70917
:1072C000BE01882777FD8095982F0E94AAC79B0151
:1072D000AC01C801B7010E94B8C97B018C018418B8
:1072E0009508B401882777FD8095982F0E94AAC73A
:1072F0009B01AC01C801B7010E940FC79B01AC0103
:10730000C601B5010E9442C620E030E040E05EE3E5
:1073100023C08E5F3E012401841708F4A5CFBE016F
:10732000882777FD8095982F0E94AAC720E030E03B
:1073300040E05EE32AC0B701882777FD8095982F4B
:107340000E94AAC720E030E04AE754E40E94B8C98E
:1073500020E030E040E859E30E94B8C9F1016783BA
:107360007087818792871AC0B701882777FD80953B
:10737000982F0E94AAC720E030E04AEF53E40E9411
:10738000B8C920E030E040E859E30E94B8C9D10113
:1073900017966D937D938D939C931A97DF91CF9160
:1073A0001F910F91FF90EF90DF90CF90BF90AF9023
:1073B0009F908F907F906F905F904F903F902F9015
:1073C0000895CF92DF92EF92FF920F931F93CF9386
:1073D000DF936C01FC014387548765877687CB0177
:1073E000BA0120E030E040E051E40E94B8C90E94B8
:1073F00077C7DB01F6018181853340F4823308F0E1
:1074000068C081508C3008F0DCC007C08C3309F4B0
:10741000B2C0843609F0D5C0BFC090E0FC01E35B88
:10742000F04F1491110FFC01EE0FFF1FE75AF04FC0
:1074300065917491FB0125913491FB013296E590A1
:10744000F49082E03BC0E82FF0E0EE0FFF1FE60F64
:10745000F71F459154918F5FE82FF0E08150EE0FB8
:10746000FF1FE60FF71FC591D491CA17DB071CF564
:107470000CEF1FE0021B130B241B350BB9018827EF
:1074800077FD8095982F97012A1B3B0B442737FDEA
:107490004095542F0E948ECAEC1AFD0A970144278A
:1074A00037FD4095542F0E9403CB020F131FF601A6
:1074B0001683058386C08E5F7E019A01811708F4CA
:1074C000C2CF8CEF9FE0841B950BF60196838583DA
:1074D00078C08E5290E0FC01E35BF04F6491660F40
:1074E000FC01EE0FFF1FE75AF04F45915491FA014E
:1074F000E590F490FA0132960591149182E037C03C
:10750000E82FF0E0EE0FFF1FE40FF51F25913491F7
:107510008F5FE82FF0E08150EE0FFF1FE40FF51FA3
:10752000C591D491AC17BD07FCF4B701621B730B76
:10753000882777FD8095982F98012A1B3B0B4427BD
:1075400037FD4095542F0E948ECA0C1B1D0B9801CD
:10755000442737FD4095542F0E9403CBE20EF31EC3
:10756000F601F682E5822DC08E5F8E0179018617C5
:1075700008F4C6CF23C0BD01882777FD8095982FDA
:107580003CE0660F771F881F991F3A95D1F728EEC8
:1075900033E040E050E010C0BD01882777FD8095C2
:1075A000982F2CE0660F771F881F991F2A95D1F717
:1075B00024EF31E040E050E00E9403CBF601368337
:1075C0002583DF91CF911F910F91FF90EF90DF9076
:1075D000CF900895EF92FF920F931F938091FF0B2E
:1075E00082FD02C080E03FC0E091CC01F091CD016E
:1075F000E780F0840185128582E796E060E070E024
:107600000E94FA2AC801B7010E9477C7665F7F4FC0
:107610006D52714018F481E996E002C08CE796E063
:107620000E94262BE091CE01F091CF01E780F084FB
:107630000185128587E696E00E949F2AC801B7015E
:107640000E9477C7665F7F4F6D52714018F08CE7DC
:1076500096E002C081E996E00E94262B8BE996E035
:107660000E942B2B81E01F910F91FF90EF900895C6
:10767000EF92FF920F931F930E9421C4AB01BC01B4
:1076800080E696E00E94E92AE0911C01F0E0EE0F0E
:10769000FF1FE453FE4F0081118133E9E32E34E0F4
:1076A000F32EF8014781508561857285C70122E07C
:1076B0000E94FD2BF8014385548565857685C701B9
:1076C00020E00E94FD2BF8018081E8E4F4E0E80F5F
:1076D000F11D6081C70170E00E94C22A1F910F91C5
:1076E000FF90EF900895DF92EF92FF920F931F9318
:1076F0007B018C01D42E20E030E040EF52E40E9468
:1077000016C918165CF40F2EF0E0EF2EF0E0FF2EF5
:10771000F0EF0F2FF2E41F2FF02D14C0C801B701B6
:1077200020E030E040E050E00E9408C7882354F495
:107730000F2EF0E0EF2EF0E0FF2EF0E00F2FF0E044
:107740001F2FF02D60919601709197018091980103
:1077500090919901A80197010E9408C7882321F1FF
:107760008BE891E0B801A7010E94E139DD2079F0B2
:10777000C801B70120E030E040EF51E40E9416C993
:1077800018162CF48091CB0181608093CB0140913D
:1077900096015091970160919801709199018BE544
:1077A00095E020E00E94122C1F910F91FF90EF9026
:1077B000DF9008952F923F924F925F926F927F9247
:1077C0008F929F92AF92BF92CF92DF92EF92FF92F1
:1077D0000F931F93DF93CF93CDB7DEB7E3970FB629
:1077E000F894DEBF0FBECDBF9BAB8AAB48A359A3B5
:1077F0006AA37BA32CA30DA30E9421C46D8B7E8B57
:107800008F8B988FAAA9BBA996968C9190E095959D
:1078100087951C01442437FC4094542C86E695E05F
:107820000E94382BE091CC01F091CD011682158297
:1078300080E090E0A0E0B0E083879487A587B687DA
:10784000E081F0E0E85BFB4F1082E091CE01F09127
:10785000CF011682158283879487A587B687E0813A
:10786000F0E0E85BFB4F1082BCA1B0931E01AAA917
:10787000BBA9EC91F0E0E85BFB4F96968C9180837E
:10788000BCA1BB2321F48091890180938A012D89B9
:107890003E894F89588D298B3A8B4B8B5C8B7901B4
:1078A0008A0129863A864B865C861B8E1A8E31E0C9
:1078B000398F80E090E0A0EAB1E489839A83AB83BA
:1078C000BC835C016D018AA99BA90E947138AAA999
:1078D000BBA91796BC91BEA7EAA9FBA9F085FFA793
:1078E000AAA9BBA91996BC91B8ABEAA9FBA9F285D4
:1078F000F9AB0E9421C43B014C0169817A818B81E3
:107900009C812EA53FA548A959A90E9408C7882394
:1079100044F48EA59FA5A8A9B9A989839A83AB83AE
:10792000BC83C601B5012EA53FA548A959A90E944F
:1079300008C787FD06C08EA59FA5A8A9B9A95C01A7
:107940006D01298D222309F441C06EA57FA588A968
:1079500099A928A139A14AA15BA10E9416C91816AC
:107960000CF08FC1A40193012E193F09400B510B5C
:107970008CA1882329F484EC99E0A0E0B0E004C055
:107980008CED95E0A0E0B0E082179307A407B5075F
:1079900008F077C1AAA9BBA9EC916E2F70E0685BD3
:1079A0007B4F822DB9858B1BFB0180832D873E8702
:1079B0004F87588B698A7A8A8B8A9C8A28A139A139
:1079C0004AA15BA129833A834B835C836EA57FA583
:1079D00088A999A928A139A14AA15BA10E9408C739
:1079E00088230CF04DC1A401930189899A89AB8940
:1079F000BC89281B390B4A0B5B0B9CA1992329F0EE
:107A000088EB9BE0A0E0B0E004C088E893E1A0E050
:107A1000B0E082179307A407B50708F031C1AA8D1B
:107A2000BB8DAB2B09F412C18D859E85AF85B889BE
:107A3000820F931FA41FB51F8C8F9D8FAE8FBF8F9A
:107A40006D857E858F859889621B730B840B950BE2
:107A500029853A854B855C850E948ECA2C8D3D8D8B
:107A60004E8D5F8D0E9403CB220D331D441D551D8D
:107A7000243131054105510534F464E1262E312CC1
:107A8000412C512C14C0AAA9BBA996968C9190E0C8
:107A900044977C010027F7FC0095102F19012A015B
:107AA000E216F3060407150714F417012801EAA9E2
:107AB000FBA926A1822F869590E0A0E0B0E0821578
:107AC0009305A405B5052CF029863A864B865C867D
:107AD00010C0822F90E001979C01442737FD40950C
:107AE000542F221933094409550929873A874B87AE
:107AF0005C8789E795E0B201A1010E94E92A81E84B
:107B000095E049855A856B857C850E94E92A86E83F
:107B100095E0B601A50122E00E94FD2B8DE895E0DD
:107B200049815A816B817C8122E00E94122C4A8D0E
:107B30005B8D433051050CF489C069857A858B854E
:107B40009C850E94AAC720E030E040E850E40E94F3
:107B5000B8C97B018C0169817A818B819C81A601E6
:107B600095010E9441C620ED3FE049E450E40E94A7
:107B7000B8C99B01AC01C801B7010E940FC77B01C6
:107B80008C016C8D7D8D8E8D9F8D0E94AAC720E00B
:107B900030E04AE754E40E940FC75B016C0184E9BE
:107BA00095E0B801A70122E00E94FD2B8AE995E04B
:107BB000B601A50122E00E94122CC801B7012AE9F2
:107BC00039E949E15FE30E94B8C96D837E838F8301
:107BD00098879B01AC010E9442C6A60195010E94B4
:107BE0000FC77B018C016AA7FBA60CA71DA76D819F
:107BF0007E818F819885A60195010E94B8C920E0F9
:107C000030E040E05EE30E94B8C95B016C016EA306
:107C1000BFA2C8A6D9A680EA95E00E94262B8DEACD
:107C200095E04D815E816F81788522E00E94122C63
:107C300083EB95E0A701B80122E00E94122C89EBAA
:107C400095E0A501B60122E00E94122CAAA9BBA9C9
:107C5000EC912E2F30E0285B3B4F8985820DF90196
:107C600080832A8D3B8D2F5F3F4F3B8F2A8F84016E
:107C70007301A8A0B9A0CAA0DBA031E0398F01C070
:107C8000198E68A179A18AA19BA120E030E040EA89
:107C900051E40E9442C69B01AC016EA57FA588A954
:107CA00099A90E9416C918161CF48FEB95E031C0F3
:107CB000D401C3012D893E894F89588D821B930BB6
:107CC000A40BB50B895E9340A040B04038F080E033
:107CD0000E944D1C6D8A7E8A8F8A988E660C771C56
:107CE000881C991C6E187F08800A910A89899A89D4
:107CF000AB89BC89681A790A8A0A9B0A91E86916D5
:107D00009FE4790692E1890690E0990650F188EEA9
:107D100095E00E942B2BE091CC01F091CD011682D1
:107D2000158280E090E0A0E0B0E083879487A5878B
:107D3000B687E081F0E0E85BFB4F1082E091CE0176
:107D4000F091CF011682158283879487A587B68725
:107D5000E081F0E0E85BFB4F10828FEF80931E0123
:107D600062C0AA8DBB8D16970CF454C085E096E0D6
:107D70000E94382BE091CC01F091CD011682158242
:107D800080E090E0A0E0B0E083879487A587B68785
:107D9000E081F0E0E85BFB4F1082E091CE01F091D2
:107DA000CF011682158283879487A587B687E081E5
:107DB000F0E0E85BFB4F10828FEF80931E01BDA1C6
:107DC000BB2389F12D813E814F815885AAA9BBA98A
:107DD0005A962D933D934D935C935D972AA53BA5B1
:107DE0004CA55DA5C901DA01EAA9FBA9868F978F89
:107DF000A0A3B1A32EA13FA148A559A5C901DA01AD
:107E000082A393A3A4A3B5A381E0838B80E00E9407
:107E1000BD2F09C08EE69FE00E944B9A8EE69FE040
:107E20000E9437C150CDE3960FB6F894DEBF0FBE67
:107E3000CDBFCF91DF911F910F91FF90EF90DF9019
:107E4000CF90BF90AF909F908F907F906F905F90FA
:107E50004F903F902F90089560E080912D018823EE
:107E600009F461E080912C010E94D5C508959F928C
:107E7000AF92BF92CF92DF92EF92FF920F931F9338
:107E8000CF93DF937B018C01942EA22EE091CC0145
:107E9000F091CD01638574858585968520E030E07D
:107EA00040E751E40E9416C9181614F4BB2402C01E
:107EB000BB24B394C801B70120E030E849E853E49B
:107EC0000E9416C918165CF40F2EF0E0EF2EF0E8B1
:107ED000FF2EF9E80F2FF3E41F2FF02D14C0C80177
:107EE000B70120E030E040E050E00E9408C788235E
:107EF00054F40F2EF0E0EF2EF0E0FF2EF0E00F2F05
:107F0000F0E01F2FF02DC92CDD24F601EE0FFF1F2E
:107F1000E453FE4FC081D181CE01B801A7010E9478
:107F2000E139AA2081F0C801B70120E030E040EF3C
:107F300051E40E9416C9181634F4FE01E05CFF4FAC
:107F4000808181608083C801B70120E030E048E48F
:107F500052E40E9416C988237CF08CE690E0C89E0B
:107F6000F001C99EF00DD89EF00D1124E15EFE4F88
:107F7000E659FF4F81918083692D70E080E090E0A9
:107F80000E94A8C7AB01BC0180E595E020E00E94FB
:107F9000FD2B8FE194E0B801A70120E00E94122C94
:107FA000E091CC01F091CD0163857485858596853E
:107FB00020E030E040E751E40E9416C918162CF08A
:107FC000BB2079F40E94192F0CC0BB2051F00E94F5
:107FD00021C46093600C7093610C8093620C909349
:107FE000630CDF91CF911F910F91FF90EF90DF9085
:107FF000CF90BF90AF909F9008952F923F924F9255
:108000005F926F927F928F929F92AF92BF92CF9228
:10801000DF92EF92FF920F931F93DF93CF9300D0E5
:1080200000D0CDB7DEB78091C70B9091C80BA0915F
:10803000C90BB091CA0BE0917502F0917602838F63
:10804000948FA58FB68F1FE1C12E11E0D12ED09253
:108050007602C09275028093EF0B9093F00BA09381
:10806000F10BB093F20BE0902801F0902901009100
:108070002A0110912B01E092E701F092E8010093B0
:10808000E9011093EA0160E070E080E89FE3A80155
:1080900097010E940FC76093940B7093950B809388
:1080A000960B9093970B80912E0190912F01A091A8
:1080B0003001B09131018093F7019093F801A093C2
:1080C000F901B093FA01609132017091330180910E
:1080D00034019091350160932302709324028093C0
:1080E00025029093260260931302709314028093EA
:1080F000150290931602A80197010E94B8C90E9428
:108100007CC76093A40B7093A50B8093A60B9093F0
:10811000A70B6093B40B7093B50B8093B60B909341
:10812000B70BC60185960E941A38A090CB0BB09071
:10813000CC0BC090CD0BD090CE0B6090CF0B70903D
:10814000D00B8090D10B9090D20B2090D30B30901D
:10815000D40B4090D50B5090D60B8091460C90914B
:10816000470CA091480CB091490C89839A83AB834A
:10817000BC830091750210917602D80111966D9121
:108180007D918D919C9114979095809570956195B6
:108190007F4F8F4F9F4F0E94AAC72091880B30912D
:1081A000890B40918A0B50918B0B0E94B8C9609348
:1081B000560C7093570C8093580C9093590CF801FF
:1081C0006581768187819085909580957095619580
:1081D0007F4F8F4F9F4F0E94AAC720918C0B3091E9
:1081E0008D0B40918E0B50918F0B0E94B8C96093FC
:1081F0005A0C70935B0C80935C0C90935D0C809197
:10820000000C80FF26C000D000D08091FB0190912F
:10821000FC01A091FD01B091FE01EDB7FEB7818395
:108220009283A383B483C601B501A40193018201A3
:1082300071010F2EF0E8AF2EFFE4BF2EF3ECCF2E2E
:10824000F7E4DF2EF02D0E944B730F900F900F90EC
:108250000F9089819A81AB81BC818093460C909369
:10826000470CA093480CB093490C80E00E943C6BF3
:108270000F900F900F900F90CF91DF911F910F9162
:10828000FF90EF90DF90CF90BF90AF909F908F9036
:108290007F906F905F904F903F902F9008958FE167
:1082A00091E09093760280937502209A219A8091B2
:1082B0002C0161E00E9458C580912D01882329F48A
:1082C00080912C0161E00E94D5C50E9421C4609379
:1082D0005301709354018093550190935601549A21
:1082E0005C980E9461380E948E4D08952F923F92B3
:1082F0004F925F926F927F928F929F92AF92BF92B6
:10830000CF92DF92EF92FF920F931F93DF93CF9361
:10831000CDB7DEB72B970FB6F894DEBF0FBECDBF3B
:108320000CEC11E01C830B8389E891E09A8389832C
:108330001F821E8292E39D8380911E01AE81A81749
:1083400009F452C2EB81FC8180809180C4010E94BB
:108350007138FE81FF2329F5D40117966D917D9127
:108360008D919C911A9720E030E048E452E40E94FD
:1083700008C7882394F4F401638574858585968500
:1083800020E030E048E452E40E9408C788232CF43F
:10839000A981BA8111961C9204C0E981FA81808179
:1083A0008183D090FF0BD2FC2DC0D4011796ED90A5
:1083B000FD900D911C911A97C801B70120E030E0A3
:1083C00040E251EC0E9408C787FD0AC0C801B7010E
:1083D00020E030E041E953E40E9416C9181694F4F5
:1083E000809177028F5F809377028B3018F4B1E031
:1083F000BF8308C0E4E0DE2AD092FF0B0E94EA3A75
:10840000F1E0FF838091FF0B82FDEEC12224D401B5
:1084100013962D913C91149715968D919C911697DA
:10842000281739071CF4222423940FC08401005C10
:108430001F4FF801808180FF08C08D8163E00E949A
:108440006997D8018C918E7F8C93F40187A5E82FD2
:10845000F0E03C96EE0FFF1FEE0FFF1FE80DF91D39
:10846000D4011796AD90BD90CD90DC901A97A08264
:10847000B182C282D382382E3394B3E03B22F4011E
:1084800037A68389813009F0DAC0E384F484058556
:108490001685C801B70120E030E040EA51E40E94AF
:1084A00008C787FDC4C0C801B701A60195010E9495
:1084B00041C62B013C0120E030E040EA51E40E943B
:1084C00016C9181624F4D40196966C91B1C0C30154
:1084D000B20120E030E040EA51EC0E9408C787FD7D
:1084E000A6C0D4015A96ED90FD900D911C915D9718
:1084F000E886F9860A871B87C301B20154962D913D
:108500003D914D915C9157970E9442C67B018C0131
:10851000F401A3A4B4A4C5A4D6A4A60195010E9405
:1085200008C787FD11C0D4019796AD90BD90CD903E
:10853000DC909A97C801B701A60195010E9416C95F
:10854000181614F057016801F401A48AB58AC68A86
:10855000D78A688579858A859B85A30192010E94C7
:10856000B8C97B018C01C601B501D4015E962D917D
:108570003D914D915C9191970E94B8C92DEC3CECD6
:108580004CEC5DE30E94B8C99B01AC01C801B70186
:108590000E9442C67B018C01F40186A1C82EDD2415
:1085A000E7A5F0E03C96EE0FFF1FEE0FFF1FE80D72
:1085B000F91D6081718182819381D40117962D917B
:1085C0003D914D915C911A970E9441C6F40122A100
:1085D00033A144A155A10E94B8C92FED3FE445E560
:1085E00050E40E94B8C99B01AC01C801B7010E94C8
:1085F00042C67B018C01B601882777FD8095982FB4
:108600000E94AAC79B01AC01C801B7010E94B8C96A
:1086100029E23FEF4FE75BE30E94B8C90E9477C7AA
:1086200077FD05C0C616D7061CF4B60101C060E090
:10863000D401EC91F0E0E85BFB4F6083B5C0833080
:1086400009F07DC0F4014384548465847684C301B9
:10865000B20120E030E040EA51E40E9408C787FD03
:108660006AC0C301B201A60195010E9441C67B0107
:108670008C0120E030E040EA51E40E9416C918164F
:1086800024F4D40196968C9157C0C801B70120E01C
:1086900030E040EA51EC0E9408C787FD4CC0F4016D
:1086A000648975898689978920E030E040E450E448
:1086B0000E94B8C97B018C01E32DF0E03C96EE0FDF
:1086C000FF1FEE0FFF1FE80DF91DC601B501208148
:1086D0003181428153810E9441C62FED3FE445E53F
:1086E00050E40E94B8C99B01AC01C801B7010E94C7
:1086F00042C620E030E040E85EE30E94B8C9D40101
:1087000054966D937D938D939C9357975A962D9184
:108710003D914D915C915D970E94B8C9A60195016C
:108720000E9442C6A30192010E9416C918161CF0AD
:10873000F401808D01C080E0D401EC9131C0823021
:1087400041F50E9421C49B01AC01F4018785908909
:10875000A189B28979018A01E81AF90A0A0B1B0B6F
:10876000D801C70189589341A040B040E8F0E081AA
:10877000222011F480E001C08FEFF0E0E85BFB4FB6
:108780008083D4011F962D933D934D935C93529714
:108790000BC0D401EC91222011F480E001C08FEFD6
:1087A000F0E0E85BFB4F8083F40167817085818591
:1087B000928520E030E849E853E40E9416C9181673
:1087C00034F4D401EC91F0E0E85BFB4F108280912F
:1087D00075029091760285968816990629F42220D2
:1087E00011F0149A01C01498BE81BF5FBE83ED8161
:1087F000EE5CED830B811C810E5F1F4F1C830B838E
:1088000089819A8184599F4F9A838983B23009F074
:1088100093CD9F81992339F480917702882319F0B1
:108820008150809377028091FF0B82FF17C0E09107
:10883000CC01F091CD01E081F0E0E85BFB4F1082CC
:10884000E091CE01F091CF01E081F0E0E85BFB4FD9
:108850001082809127028860809327022B960FB6A2
:10886000F894DEBF0FBECDBFCF91DF911F910F9166
:10887000FF90EF90DF90CF90BF90AF909F908F9040
:108880007F906F905F904F903F902F900895FC01E4
:108890008081918180FD02C024E001C026E083FD3B
:1088A0002C5F84FD2C5F85FD2C5F86FD2C5F90FD89
:1088B0002C5F91FD2F5F92FD2C5F93FD2C5FAC012F
:1088C0004270507094FF19C02E5F3281452B09F021
:1088D0002E5F82FD2E5F30FD2C5F31FD2C5F32FD5F
:1088E0002C5F97FF11C0848190E00196813591053E
:1088F00014F080E590E0280F07C0452B09F02F5FAA
:1089000082FD2F5F97FD205F822F08958091E30203
:1089100090E00196817090708093E3028091520301
:108920008F5F80935203089580915203882319F436
:1089300020E030E008C09091E20285E3989F90012A
:10894000112428583D4FC9010895CF93DF93EC01BE
:10895000888181FF12C083E294E06DE40E94074F9A
:108960006E817F81882777FD8095982F0E94812ACC
:1089700083E294E060E20E94074F888182FF12C088
:1089800083E294E067E40E94074F68857985882731
:1089900077FD8095982F0E94812A83E294E060E21F
:1089A0000E94074F8881998191FF12C083E294E071
:1089B00064E50E94074F6E8D70E0882777FD8095F3
:1089C000982F0E94812A83E294E060E20E94074F80
:1089D000888183FF09C04A855B856C857D8589E335
:1089E00093E022E00E94FD2B888184FF09C04E8520
:1089F0005F85688979898CE393E022E00E94FD2BF2
:108A0000888185FF09C04A895B896C897D898FE3EC
:108A100093E022E00E94FD2B888186FF09C04E89E9
:108A20005F89688D798D82E493E024E00E94FD2BBC
:108A30008881998190FF09C04A8D5B8D6C8D7D8DF9
:108A400085E493E022E00E94FD2B8881998192FFCA
:108A500008C04F8D58A169A17AA188E493E00E94D3
:108A6000E92A8881998193FF08C04BA15CA16DA17F
:108A70007EA18BE493E00E94E92A8A8180FF09C0ED
:108A80004FA158A569A57AA58EE493E022E00E9443
:108A9000FD2B8A8181FF09C04BA55CA56DA57EA534
:108AA00081E593E022E00E94FD2B8A8182FF09C0CC
:108AB0004FA558A969A97AA984E593E022E00E940C
:108AC000FD2B8881998197FF04C08BA99CA90E94E6
:108AD000222A0E945B1BDF91CF9108950F931F9371
:108AE000CF93DF93EC018B01709148037250F80132
:108AF00040E050E020E030E01FC0672F763108F002
:108B000065E1DF01962F8D91480F511D4F3F5105B3
:108B100010F04F5F5040240F351F2F3F310510F0EC
:108B20002F5F3040915079F76150862F90E06F5F52
:108B30000196E80FF91F761B7723F9F68181281B30
:108B400031098081481B5109242B352B232B51F0EF
:108B50008091270282FF04C089EF92E00E942B2BB4
:108B600080E0CDC0F801219131913983288334FF11
:108B70000CC0D80112968D919C9113979B838A8388
:108B8000329637FF04C0419103C01B821A8240E134
:108B9000888180FF0EC0819191919D838C83A0E09C
:108BA000B0E080934E0390934F03A0935003B09393
:108BB0005103888199819C012270307094FF0EC00E
:108BC000232B21F0819191919F838E83888182FF55
:108BD00010C081919191998788870BC0232B19F040
:108BE00081918E831F82888182FF03C08191888753
:108BF0001986888183FF08C081919191A191B191DB
:108C00008A879B87AC87BD87888184FF08C0819154
:108C10009191A191B1918E879F87A88BB98B888103
:108C200085FF08C081919191A191B1918A8B9B8B15
:108C3000AC8BBD8B888186FF08C081919191A191F9
:108C4000B1918E8B9F8BA88FB98F8881998190FF6E
:108C500008C081919191A191B1918A8F9B8FAC8F26
:108C6000BD8F8881998191FF02C081918E8F88810B
:108C7000998192FF08C081919191A191B1918F8FBB
:108C800098A3A9A3BAA38881998193FF08C0819171
:108C90009191A191B1918BA39CA3ADA3BEA38A8115
:108CA00080FF08C081919191A191B1918FA398A764
:108CB000A9A7BAA78A8181FF08C081919191A1914A
:108CC000B1918BA79CA7ADA7BEA78A8182FF08C0E0
:108CD00081919191A191B1918FA798ABA9ABBAABBA
:108CE0008881998197FF08C0FCABEBABE40FF11DC5
:108CF000108281E0809349031092570381E0DF9155
:108D0000CF911F910F910895EF92FF920F931F93B0
:108D1000DF93CF9300D0CDB7DEB77C018B01CB01C1
:108D2000BE016F5F7F4F0E940116FC0189819A810D
:108D30000817190751F4D70112968D919C9113973A
:108D4000906813969C938E931297CF010F900F907B
:108D5000CF91DF911F910F91FF90EF900895EF92C7
:108D6000FF920F931F93DF93CF9300D0CDB7DEB761
:108D70007C018B01CB01BE016F5F7F4F4AE050E069
:108D80000E9461179C0189819A810817190731F4A3
:108D9000F70182819381906893838283C9010F9048
:108DA0000F90CF91DF911F910F91FF90EF90089559
:108DB000EF92FF920F931F93CF93DF938C017B0170
:108DC000DC0111961C921E9213961C921E92129711
:108DD000CB016EE470E00E94BC18BC010097B1F0BA
:108DE0006F5F7F4FC8010E94AF4660934E03709340
:108DF0004F038093500390935103F8018081918138
:108E0000816091838083CB0164839583C7016DE486
:108E100070E00E94BC18BC010097D1F06F5F7F4FDB
:108E2000C8010E94AF46D80117967C936E9316979F
:108E30008D919C9111979C01226011963C932E93E9
:108E40006F3F710529F020F0826090618D939C93B3
:108E5000F801808181FFC5C18681978187319105A5
:108E600099F08C31910581F08D31910569F08E3149
:108E7000910551F08032910539F08537910509F05F
:108E8000B0C102C0319601C0F70180818D34D1F7A5
:108E900001C0319680818032E1F701C03196808136
:108EA0008032E1F3D801D396EC93D397D496FC9318
:108EB0000DC0D80116968D919C9117978537910515
:108EC00011F0203231F02A3221F031962081222314
:108ED00081F7108281E080934903F80180819181BC
:108EE000906834C16F5F7F4FC8010E94AF46D801C0
:108EF00019967C936E9318978D919C9111979C0174
:108F0000246011963C932E936F3F710529F020F059
:108F1000846090618D939C93C70168E570E00E9426
:108F2000BC18BC01009779F06F5F7F4FC8010E94A9
:108F30008446F80162877387848795878081918151
:108F4000886091838083C70169E570E00E94BC1846
:108F5000BC01009791F06F5F7F4FC8010E9484466B
:108F6000D8011E966D937D938D939C9351978D910F
:108F70009C91119780618D939C93C7016AE570E085
:108F80000E94BC18BC01009779F06F5F7F4FC80149
:108F90000E948446F801628B738B848B958B808151
:108FA0009181806291838083C70165E470E00E94B3
:108FB000BC18BC01009791F06F5F7F4FC8010E9401
:108FC0008446D80156966D937D938D939C935997C3
:108FD0008D919C91119780648D939C93C70166E459
:108FE00070E00E94BC18BC01009779F06F5F7F4F62
:108FF000C8010E948446F801628F738F848F958F19
:1090000080819181916091838083C70164E570E0E4
:109010000E94BC18BC01009779F06F5F7F4FC801B8
:109020000E94AF46D8015E966C935E978D919C919D
:10903000119792608D939C93C70163E570E00E9445
:10904000BC18BC01009779F06F5F7F4FC8010E9488
:10905000AF46F801678F70A381A392A380819181AD
:10906000946091838083C70160E570E00E94BC1822
:10907000BC01009791F06F5F7F4FC8010E94AF461F
:10908000D80193966D937D938D939C9396978D9134
:109090009C91119798608D939C93C70169E470E04F
:1090A0000E94BC18BC010097A1F06F5F7F4FC80100
:1090B0000E948446F80167A370A781A792A78281C6
:1090C0009381816093838283808191819061918378
:1090D0008083C7016AE470E00E94BC18BC0100975D
:1090E000D9F06F5F7F4FC8010E948446D8019B96DC
:1090F0006D937D938D939C939E9712968D919C91E9
:109100001397826013969C938E9312978D919C91E6
:10911000119790618D939C93C70162E570E00E9466
:10912000BC18BC010097A1F06F5F7F4FC8010E947F
:109130008446F80167A770AB81AB92AB82819381C3
:109140008460938382838081918190619183808305
:10915000C7016AE270E00E94BC18EC010097D9F0E8
:10916000BC016F5F7F4FC8010E94AF4690E004C012
:10917000D7018D917D019827EC16FD06C9F796174A
:1091800051F08091270282FF04C089EF92E00E9493
:109190002B2B90E01EC0F8018281938197FD06C0C1
:1091A0008081918186709270892B29F58091570377
:1091B0008F5F809357038091270282FF04C089E16B
:1091C00093E00E942B2B90E080915703833008F0AE
:1091D00091E0892FDF91CF911F910F91FF90EF9038
:1091E0000895C70167E470E00E94BC18BC010097B5
:1091F00009F078CE91CE10925703EACFAF92BF928A
:10920000CF92DF92FF920F931F93DF93CF93CDB74F
:10921000DEB7C558D0400FB6F894DEBF0FBECDBF45
:109220008C0186E3C82ED12CCC0EDD1E5E01089485
:10923000A11CB11C80E090E00F5F1F4F0150104057
:10924000F801F4900F5F1F4FFF2091F0FAE0FF1636
:1092500079F02BE3F21611F491E007C0992329F479
:10926000F601E80FF11DF0828F5F8F3428F302C002
:109270008823B1F0F601E80FF11D1082C501B60197
:1092800040E00E94D846882359F089819A818670EF
:109290009270892B29F0C5010E940E1D0E94237631
:1092A000FF2041F6CB57DF4F0FB6F894DEBF0FBE5D
:1092B000CDBFCF91DF911F910F91FF90DF90CF90A5
:1092C000BF90AF900895CF93DF93EC018091270278
:1092D00080FF07C08FEE92E00E949F2ACE010E947D
:1092E000A544DF91CF9108959C018091520388237A
:1092F00089F0C9010E9463498091E2028F5F8093E7
:10930000E202823011F41092E20280915203815005
:1093100080935203089583E294E00E94F94E1092E4
:10932000440380914503882311F08EE101C08EE053
:109330008093D0010E945B1B40914A0350914B03E4
:1093400060914C0370914D034F5F5F4F6F4F7F4FA4
:1093500087EE92E00E94AF2A83EC92E00E94262BD7
:109360000895CF92DF92EF92FF920F931F93CF93C6
:10937000DF93EC01888181FF38C08E819F818E361A
:109380009105A9F480914E0390914F03A091500351
:10939000B091510380934A0390934B03A0934C03E5
:1093A000B0934D0383EC92E00E94262B8AC0803755
:1093B000910511F40E94311A8E819F818A59924041
:1093C000A1F480914A0390914B03A0914C03B0917A
:1093D0004D030196A11DB11D80934A0390934B0349
:1093E000A0934C03B0934D036FC0888180FF57C09A
:1093F00000914A0310914B0320914C0330914D038F
:10940000680179010894C11CD11CE11CF11C409138
:109410004E0350914F036091500370915103D70157
:10942000C60184279527A627B727892B81F1C80174
:10943000841B950B889700F18091D00187FF19C09C
:109440008091270282FF12C085E693E0B701A60152
:109450000E94D82A40914E0350914F0360915003CF
:10946000709151038AE793E00E94AF2A0E948B49D2
:109470002BC081508093D0011092440380E893E088
:109480000E94AF2A83EC92E00E94262B1DC04093DD
:109490004A0350934B0360934C0370934D030E9417
:1094A000864440914E0350914F0360915003709158
:1094B000510385EF92E00E94AF2A8091450380938B
:1094C00046038FEF8093D001DF91CF911F910F91D1
:1094D000FF90EF90DF90CF900895BF92CF92DF92F0
:1094E000EF92FF920F931F93CF93DF9380915203DC
:1094F000823008F02DC280914903882309F401C20B
:1095000080915203882309F4FCC122C28091D001CA
:1095100087FF04C0809144038823B1F080915303F6
:1095200090915403A0915503B0915603A701960161
:10953000281B390B4A0B5B0B293C310541055105B2
:1095400018F00E948B491FC080915203882309F0B4
:10955000ACC08091530390915403A0915503B091F6
:109560005603A7019601281B390B4A0B5B0BDA0146
:10957000C901895E9340A040B04008F496C08FE1D5
:1095800097E00E94262BC0925303D0925403E0929E
:109590005503F092560389C09091D00197FD0FC0FA
:1095A00080914603882359F08091E402882321F4B6
:1095B00091509093D0014DC0B092D0014AC080919B
:1095C000E402882309F445C08823880F880B802390
:1095D0008093450380914503882309F1113009F4F4
:1095E00067C0812F8450823030F484EE92E00E9474
:1095F00047448093480380914803181709F04EC0F0
:109600009091E30285E3989FE0011124C858DD4F53
:10961000CE0164EE72E041E00E946E452BC0A12FA6
:10962000B0E01197FD01EC51FD4FE081EE2351F0C8
:10963000EA3041F0ED3031F080914703882319F58D
:10964000EA3309F5AC51BD4F1C921092470311301B
:1096500019F4109244032CC09091E30285E3989F83
:10966000E0011124C858DD4FCE0164EE72E041E004
:109670000E94D846882321F0CE010E94B14908C13A
:109680000E948B4905C1EB3311F40093470380918D
:109690004703882319F01150109344038091440329
:1096A000803631F40E948B4953C101E09EE1B92E0E
:1096B00083E294E00E94AD4E181619060CF030C1FA
:1096C00010914403103608F02BC1C0925303D0927E
:1096D0005403E0925503F092560383E294E00E9413
:1096E000DA4EE12FF0E0EC51FD4F80831F5F1093C5
:1096F0004403113009F06ECF4FCF8091440388238B
:1097000009F4D5C025C10E9421C46093530370930E
:109710005403809355039093560382E19DE00E9489
:10972000198FEC014FEF8F3F940761F587E593E0C8
:109730000E94262B8EE69FE068E675E141E00E94DC
:1097400051994091330D5091340D6091350D7091C8
:10975000360D82E19DE00E94988782E19DE00E94A3
:10976000198FEC015FEF8F3F950729F48EE495E1A7
:109770000E942B2BB6C08EE69FE06FE375E141E0BF
:109780000E9451992091330D3091340D4091350D47
:109790005091360D2F5F3F4F4F4F5F4F2093330D4A
:1097A0003093340D4093350D5093360D8091440322
:1097B000E82FF0E0EC51FD4FC083182F1F5F10938E
:1097C0004403113041F4109245038091E40287FF75
:1097D00002C01093450380914503882301F11230A4
:1097E00008F465C0812F8450823030F484EE92E01A
:1097F0000E9447448093480380914803181709F05A
:1098000056C08091E30225E3829FC001112488584D
:109810009D4F64EE72E040E00E946E4535C0C12F5E
:10982000D0E0BE0161507040FB01EC51FD4FE08182
:10983000EA3071F0ED3009F079C00AC08091470339
:10984000882311F4EA3321F01F3508F07DC023C0CE
:109850006C517D4FFB01108203C0CC51DD4F18824B
:1098600010924703113019F41092440320C08091E4
:10987000E30225E3829FC001112488589D4F64EEC6
:1098800072E040E00E94D846882311F00E9486448E
:10989000109244035DC0EB3319F481E080934703D9
:1098A00080914703882319F01150109344032091AD
:1098B0002F0D3091300D4091310D5091320D80912E
:1098C000330D9091340DA091350DB091360D821766
:1098D0009307A407B50728F480914403803608F461
:1098E00012CF10923B0D86E293E00E94262B10923D
:1098F0004403109247038091010C8D7F8093010CEB
:1099000027C0109249030E9421C46B017C0183E2AD
:1099100094E00E94AD4E181619060CF4C6CEF6CD92
:1099200080913B0D882309F0E8CE12C080912F0D65
:109930009091300DA091310DB091320D82179307A7
:10994000A407B50709F07ACFEA3309F086CF80CFB4
:10995000DF91CF911F910F91FF90EF90DF90CF900B
:10996000BF9008954F925F92AF92BF92CF92DF92D5
:10997000EF92FF920F9320E28030920708F079C0B7
:1099800022E08030920708F04AC08A30910510F436
:109990008AE090E0A12C24E2B22E24EFC22ED12C3A
:1099A000EE24FF18DD20A1F4CC2009F012C001E163
:1099B000AA1CBB1C0A9509F431C0EE1CFF1CE81A56
:1099C000F90A20F4E80EF91E8894F2CF0894F0CF3B
:1099D00012C009E1AA1CBB1CCC1C0A9509F41EC0CC
:1099E000EE1CFF1CE81AF90A20F4E80EF91E889410
:1099F000F1CF0894EFCF01E2AA1CBB1CCC1CDD1CEC
:109A00000A9509F40BC0EE1CFF1CE81AF90A20F4B1
:109A1000E80EF91E8894F0CF0894EECF51C0ECE820
:109A2000F5E1282F2F7196958795969587959695B0
:109A30008795969587958E7FE80FF91FA590B5902D
:109A400025010590401805905008249DC001259DD2
:109A5000900DE12D880F991FEE1F880F991FEE1FA3
:109A6000880F991FEE1FA91ABE0ACC24DD241124E9
:109A700027C0EEE8F7E19C013F7096959695969584
:109A80009E7FE90FF11DA590B59025010590401826
:109A900005905008249DC001359DE02D259D900D19
:109AA000E11D349D900DE11D907F9295E2958E2FE2
:109AB000807F982BEF70A91ABE0ACC24DD241124D4
:109AC000B501C6010F91FF90EF90DF90CF90BF904E
:109AD000AF905F904F90089514BC80E488BDEEE68F
:109AE000F0E0808184608083109280001092820078
:109AF000EFE6F0E0108289E0809381008CED9FEF2B
:109B0000909389008093880080818260808308958B
:109B1000E0915803F09159030995089580E48093EA
:109B20007C001092650210926902109268021092F5
:109B3000700210926F021092660210926B021092E5
:109B40006A021092720210927102109267021092D1
:109B50006D0210926C02109274021092730287ECE4
:109B600080937A0080917A0086FDFCCF8091780006
:109B700090917900E0916E02F0E0E65BF04FE491A5
:109B800080917C00E770807EE82BE0937C008091E0
:109B90007A00806480937A0008951F920F920FB626
:109BA0000F920BB60F9211242F938F939F93EF93E5
:109BB000FF932091C6009091DF039F5F9F77809174
:109BC000E003981741F0E091DF03F0E0E15AFC4F29
:109BD00020839093DF03FF91EF919F918F912F91BD
:109BE0000F900BBE0F900FBE0F901F9018951F92F5
:109BF0000F920FB60F920BB60F9211248F939F9373
:109C0000EF93FF939091210480912204981731F4EF
:109C10008091C1008F7D8093C1000EC0E09122042D
:109C2000F0E0EF51FC4F9081809122048F5F8F73A1
:109C3000809322049093C600FF91EF919F918F91A2
:109C40000F900BBE0F900FBE0F901F901895AF9204
:109C5000BF92DF92EF92FF920F931F93CF93DF9308
:109C6000EC017A018B01DD24403081EE580780E061
:109C7000680780E0780711F0DD24D394E1E0AE2E90
:109C8000B12CEC85FD85DD2069F0C5010E8802C090
:109C9000880F991F0A94E2F7808360E079E08DE3F2
:109CA00090E005C0108260E874E88EE190E0A801C1
:109CB00097010E94E1CA21503040404050405695E3
:109CC00047953795279580E12030380720F0DD2033
:109CD00011F0DD24D6CFE885F9853083EA85FB8550
:109CE0002083EE85FF85408121E030E0C9010A88AC
:109CF00002C0880F991F0A94E2F7482B4083EE8533
:109D0000FF854081C9010B8802C0880F991F0A9402
:109D1000E2F7482B4083EE85FF854081C9010C881E
:109D200002C0880F991F0A94E2F7482B4083EE8502
:109D3000FF8580810D8802C0220F331F0A94E2F74D
:109D4000209528232083DF91CF911F910F91FF90C1
:109D5000EF90DF90BF90AF900895DC011496ED91E5
:109D6000FC911597E058FF4F2191808130E02058F9
:109D70003F4F281B31092F773070C9010895DC014E
:109D80001496ED91FC911597E058FF4F9081E058A3
:109D9000F040DF01AF57BF4F8C91981719F42FEFA8
:109DA0003FEF06C08C91E80FF11D8081282F30E035
:109DB000C9010895DC011496ED91FC911597E058C6
:109DC000FF4F9081E058F040DF01AF57BF4F8C91BB
:109DD000981719F42FEF3FEF0AC08C91E80FF11D8F
:109DE00090818C918F5F8F778C93292F30E0C90100
:109DF0000895FC0186819781DC01A05CBF4FFC01C6
:109E0000EF5BFF4F9C9180819817E1F70895CF9306
:109E1000DF93EC01EE81FF81E05CFF4F9081E05425
:109E2000F0409F5F9F73DF01AF5BBF4F8C9198172E
:109E3000E9F3E05CFF4F8081E054F040E80FF11D52
:109E40006083EE81FF81E05CFF4F9083EE85FF85AC
:109E5000208181E090E00D8802C0880F991F0A944C
:109E6000E2F7282B208381E090E0DF91CF910895E5
:109E7000109226041092250485E592E09093240424
:109E8000809323048FE593E0909328048093270424
:109E900081EE93E090932A048093290485EC90E06E
:109EA00090932C0480932B0484EC90E090932E04E8
:109EB00080932D0480EC90E09093300480932F04E5
:109EC00081EC90E0909332048093310486EC90E032
:109ED000909334048093330484E08093350483E0CA
:109EE0008093360487E08093370485E080933804BC
:109EF00081E08093390408951F920F920FB60F925C
:109F00000BB60F9211242F933F934F935F936F9350
:109F10007F938F939F93AF93BF93CF93DF93EF93F1
:109F2000FF9388B5805C88BD90913E04992361F4CD
:109F30008091480480933A0481115D9A809149048C
:109F400080933B0481115C9A70913F04772331F434
:109F500080914B0480933D0481112C9A80913A04A6
:109F6000891719F49F3F09F05D9880913D04871788
:109F700019F47F3F09F02C9880913B04891719F45C
:109F80009F3F09F05C9878948091620290916302FF
:109F9000019690936302809362028658914038F054
:109FA000109263021092620281E0809364028091B9
:109FB0007A0086FD43C060916E02862F90E040914A
:109FC000780050917900DC01AA0FBB1FED01C85940
:109FD000DD4F28813981420F531F59834883FC018B
:109FE000EB59FD4F80818F5F8083803210F183E0D9
:109FF000569547958A95E1F7A159BD4F11965C9307
:10A000004E93198218821082862F8F5F80936E0282
:10A01000833010F010926E02E0916E02F0E0E65B89
:10A02000F04FE49180917C00E770807EE82BE09314
:10A030007C0080917A00806480937A0072FF04C073
:10A040008EE69FE00E944D9A80913F048F5F80933F
:10A050003F0480913E048F5F80933E04FF91EF9117
:10A06000DF91CF91BF91AF919F918F917F916F9130
:10A070005F914F913F912F910F900BBE0F900FBEAC
:10A080000F901F9018951F920F920FB60F920BB65C
:10A090000F9211242F933F934F935F936F937F936E
:10A0A0008F939F93AF93BF93EF93FF9380915A0346
:10A0B000882309F07DC080E070915D03772381F4EF
:10A0C00070915C03772319F460915B0391F07093B6
:10A0D00089006093880010925B0310925C0308C0B3
:10A0E00060915C036058704060935C0370935D0303
:10A0F00081E0882309F05CC081E080935A0388E402
:10A100009EEE90938900809388008091810B882334
:10A1100009F42FC00E948152F8948823E1F47F3F14
:10A12000D1F010925B0310925C0310925D0380915A
:10A1300084009091850024E6820F911D68177907AD
:10A1400028F4909389008093880012C0709389004E
:10A15000609388000DC07058804060935B037093DB
:10A160005C0380935D0390E89093890010928800CF
:10A170001DC080914C0490914D04892B49F0809131
:10A180004C0490914D04019790934D0480934C049E
:10A1900010925B0310925C0310925D0310925E03B9
:10A1A0008CED9FEF909389008093880010925A0362
:10A1B000FF91EF91BF91AF919F918F917F916F919F
:10A1C0005F914F913F912F910F900BBE0F900FBE5B
:10A1D0000F901F901895FF920F931F93FFB6F8945E
:10A1E00084E090E00E94FF148C010E94A9152DB715
:10A1F0003EB7FFBE201B310BC9011F910F91FF908D
:10A2000008951F9384B7182F10FF04C081E993E0CD
:10A210000E94382B11FF04C089E993E00E94382B7B
:10A2200012FF04C088EA93E00E94382B13FF04C099
:10A2300088EB93E00E94382B15FF04C087EC93E075
:10A240000E94382B14BE1F9108952F923F924F9277
:10A250005F926F927F928F929F92AF92BF92CF92B6
:10A26000DF92EF92FF920F931F93CF93DF93EC0156
:10A27000888180FDE2C0898180FDDFC029C02E5F1A
:10A280003F4FC901A0E0B0E0841B950BA60BB70BB4
:10A29000B595A79597958795BC018816990608F4FA
:10A2A000C401881A990AF20191828082FE01E15A62
:10A2B000FF4F408151819B014617570708F49A01CF
:10A2C000421B530B51834083888181608883B5C0D2
:10A2D000ED96E880F9800A811B81ED97FE01E35B32
:10A2E000FF4FC801B70120813181428153810E9413
:10A2F000B8C93B014C014BE6242E312C2C0E3D1EDF
:10A30000C759DF4F48805980B20180E090E00E9439
:10A31000A8C75B016C01A097C801B70128813981EA
:10A320004A815B810E94B8C99B01AC01C601B5019D
:10A330000E94B8C90E947CC77B018C01F101718326
:10A340006083A496C601B501A40193010E94B8C917
:10A350000E947CC73B014C0179836883CD56D04075
:10A36000C201889F5001999F6001899F8827B00C86
:10A37000C11CD81EB00CC11CD81E11249701229FED
:10A38000C001339FD001239F2227900DA11DB21F32
:10A39000900DA11DB21F11243DE5432E512C4C0EF2
:10A3A0005D1EA6019501281B390B4A0B5B0BCA01E8
:10A3B000B901CF59DF4FE880F9800A811B81EE0C8B
:10A3C000FF1C001F111FA80197010E94E1CA49014B
:10A3D0000894811C911CF201918280829301229F3A
:10A3E000C001339FD001239F2227900DA11DB21FD2
:10A3F000900DA11DB21F1124A81AB90ACA0ADB0ABE
:10A40000C601B501A80197010E94E1CA2F5F3F4F25
:10A410003A932A93280D391D6096488159816A81A3
:10A420007B81CF56D040C901A0E0B0E084179507EA
:10A43000A607B7070CF023CF47CFDF91CF911F912D
:10A440000F91FF90EF90DF90CF90BF90AF909F90D3
:10A450008F907F906F905F904F903F902F900895D6
:10A46000FF920F931F93282F162F8091810B882323
:10A4700009F042C080914C0490914D04892BE1F584
:10A480002223D1F134E0A3E7B0E0FF24F39407E006
:10A4900048EA51E660E070E031502091800B822F55
:10A4A00090E08A9FF0018B9FF00D9A9FF00D112490
:10A4B000E25BFB4FF18200831086832F810F828342
:10A4C00043835483658376832F5F2093800B2031F1
:10A4D00010F01092800B8091010C80618093010C30
:10A4E0009FB7F8948091810B8F5F8093810B9FBF02
:10A4F000332391F681E001C080E01F910F91FF901E
:10A500000895BF92CF92DF92EF92FF920F931F9325
:10A51000CF93DF9380917E0B90917F0B892B09F075
:10A5200048C18091820B482F50E083E790E0489F1C
:10A53000E001499FD00D589FD00D1124C25BDB4F25
:10A54000D0937F0BC0937E0B898187FD3FC07894A9
:10A550008FEF9FEF9093DA018093D90180912702CA
:10A5600085FF21C08091820B8F5F8093820B8031A9
:10A5700010F01092820B10927F0B10927E0BF894C9
:10A580008091810B81508093810B8091810B882376
:10A5900029F48091010C8F7E8093010C28EE33E02A
:10A5A00040E050E0B5C383E790E0489FF001499F49
:10A5B000F00D589FF00D1124E25BFB4F818180FF6D
:10A5C00030C09091810B8281891748F010927F0BE7
:10A5D00010927E0B20ED37E040E050E099C32381DC
:10A5E0003481458156818091820B8F5F8093820BED
:10A5F000803110F01092820B10927F0B10927E0B24
:10A60000F8948091810B81508093810B8091810B14
:10A61000882309F07DC38091010C8F7E8093010C0B
:10A6200077C36085262F64FD5E9825FD5E9826FD24
:10A63000159867FD5E9883E790E0489FF001499F79
:10A64000F00D589FF00D1124E25BFB4F8081866076
:10A650008083789483E790E0489F9001499F300D74
:10A66000589F300D1124F901E25BFB4F8781843044
:10A6700079F4E281F0E0EE0FFF1FEE0FFF1FE20F13
:10A68000F31FE25BFB4F81859285A385B48512C0E1
:10A69000E281F0E0EE0FFF1FEE0FFF1FE20FF31F4E
:10A6A000E25BFB4F81859285A385B485880F991F56
:10A6B000AA1FBB1F8093830B9093840BA093850BE1
:10A6C000B093860B83E790E0489FF001499FF00D1F
:10A6D000589FF00D1124E25BFB4F808180FD03C089
:10A6E000CE010E942551E0917E0BF0917F0BE55940
:10A6F000FF4F80819181EB56F04090935F0C8093E7
:10A700005E0C10920A0C10920B0C10920C0C109212
:10A710000D0C1092060C1092070C1092080C10925F
:10A72000090CF8948085282F30E0C9018171907060
:10A73000419711F4459A01C04598C9018272907001
:10A74000829711F4479A01C04798C90184749070A8
:10A750008434910511F42A9801C02A9A287830701F
:10A760002838310511F4289A01C028988091680C86
:10A7700097818823C1F0943009F0D6C21092680CFA
:10A780008091020C9091030CA091040CB091050CE7
:10A790009C01AD01220F331F441F551F280F391F85
:10A7A0004A1F5B1FB5C2943009F4BEC281E080939A
:10A7B000680C7894E0917E0BF0917F0BD78086E057
:10A7C000C82ECD2024E0D21619F083E08D1987839E
:10A7D000F894CC20F1F0818184FF12C09085892FFC
:10A7E0008171803121F4329902C09F7E90879085DB
:10A7F000892F8272803221F4339902C09F7D908725
:10A800009085892F8474803421F4349902C09F7B11
:10A81000908780912802E159FF4FE080F18002810A
:10A820001381282F30E040E050E0E216F3060407E1
:10A83000150714F4A8019701B22E1E141F04100668
:10A8400011060CF002C210E0A7C0112321F081E034
:10A8500090E00E9488C4E0917E0BF0917F0B808590
:10A8600087FF23C025A136A147A150A585899689D8
:10A87000A789B08D281B390B4A0B5B0B25A336A388
:10A8800047A350A757FF11C0299A8091830B90913D
:10A89000840BA091850BB091860B280F391F4A1F9E
:10A8A0005B1F25A336A347A350A7808584FF23C041
:10A8B000218D328D438D548D81859285A385B485FC
:10A8C000281B390B4A0B5B0B218F328F438F548F20
:10A8D00057FF11C05F9A8091830B9091840BA091D8
:10A8E000850BB091860B280F391F4A1F5B1F218FE4
:10A8F000328F438F548F808585FF23C0258D368D01
:10A90000478D50A185859685A785B089281B390B71
:10A910004A0B5B0B258F368F478F50A357FF11C013
:10A92000469A8091830B9091840BA091850BB091F6
:10A93000860B280F391F4A1F5B1F258F368F478FC5
:10A9400050A3808586FF23C021A132A143A154A139
:10A9500081899289A389B489281B390B4A0B5B0B27
:10A9600021A332A343A354A357FF11C02B9A809174
:10A97000830B9091840BA091850BB091860B280FCF
:10A98000391F4A1F5B1F21A332A343A354A3299855
:10A990005F9846982B981F5F1B1508F456CF85E0EB
:10A9A000D82209F426C17894C0917E0BD0917F0BF8
:10A9B000C35ADF4F88819981CD55D040A0E0B0E0E7
:10A9C00020910A0C30910B0C40910C0C50910D0C05
:10A9D00082179307A407B50708F460C02091060CFE
:10A9E0003091070C4091080C5091090CCB59DF4F66
:10A9F00088819981AA81BB81BA01A901589F212D23
:10AA00005A9F302D412D599F200D311D4B1F689F9E
:10AA1000200D311D4B1F699F300D411D789F300D5A
:10AA2000411D6A9F400D799F400D469537952795AA
:10AA30004695379527951124269688819981820F0E
:10AA4000931F90935F0C80935E0CFE0132912291D4
:10AA50002817390720F430935F0C20935E0C209167
:10AA60005E0C30915F0C8EE2213E380790F08DE550
:10AA7000213C380740F084E08093280236952795E2
:10AA80003695279509C082E0809328023695279550
:10AA900003C081E080932802C90158C0FE01E1593A
:10AAA000FF4FC15ADF4F88819981CF55D040A0E038
:10AAB000B0E0208131814281538182179307A4073E
:10AAC000B5077CF0898182FD38C11092060C109286
:10AAD000070C1092080C1092090C898184608983FC
:10AAE0002CC1C759DF4F88819981C956D0402EE2C9
:10AAF000813E920708F04BC06BC0C359DF4FE8811D
:10AB0000F9810AC0C359DF4F88819981E61BF70B91
:10AB1000E817F90708F4FC018EE2E13EF80790F02F
:10AB20002DE5E13CF20740F084E080932802F695A1
:10AB3000E795F695E79509C082E080932802F6959F
:10AB4000E79503C081E080932802CF010E94B24CB8
:10AB50009B01AC012093020C3093030C4093040C36
:10AB60005093050C8091060C9091070CA091080C55
:10AB7000B091090C820F931FA41FB51F8093060C80
:10AB80009093070CA093080CB093090C32C0FE01FF
:10AB9000E75AFF4F815C9D4578F084E0809328025E
:10ABA00080819181A281B381F2E0880F991FAA1F51
:10ABB000BB1FFA95D1F715C082E0809328028081EF
:10ABC0009181A281B381880F991FAA1FBB1F09C061
:10ABD00081E080932802C75ADF4F88819981AA813A
:10ABE000BB818093020C9093030CA093040CB09350
:10ABF000050CCC2051F12B2D30E040E050E080914D
:10AC00000A0C90910B0CA0910C0CB0910D0C820FC2
:10AC1000931FA41FB51F80930A0C90930B0CA09355
:10AC20000C0CB0930D0CE0917E0BF0917F0BE15971
:10AC3000FF4F80819181A281B381821B930BA40B72
:10AC4000B50B80839183A283B383E0917E0BF09157
:10AC50007F0B87812091020C3091030C4091040CF2
:10AC60005091050C843039F079018A0116950795C9
:10AC7000F794E79402C079018A01CC2009F446C018
:10AC8000E159FF4F80819181A281B381EF56F0405D
:10AC9000181619061A061B061CF48085807FB1F56C
:10ACA0008091820B8F5F8093820B803110F0109225
:10ACB000820B10927F0B10927E0BF8948091810B87
:10ACC00081508093810B8091810B882329F480919E
:10ACD000010C8F7E8093010C8091810B882339F4C5
:10ACE0008EE69FE060EB77E140E00E945199A80179
:10ACF000970155954795379527952093020C3093EA
:10AD0000030C4093040C5093050C02C0A80197015A
:10AD1000B901CA01DF91CF911F910F91FF90EF9080
:10AD2000DF90CF90BF9008952091020C3091030CDA
:10AD30004091040C5091050CEBCF2091060C309102
:10AD4000070C4091080C5091090CCB59DF4F8881BA
:10AD50009981AA81BB81C556D040389F612D3A9F09
:10AD6000702D212D399F600D711D2B1F489F600D87
:10AD7000711D2B1F499F700D211D589F700D211DA6
:10AD80004A9F200D599F200D26957795679526950A
:10AD9000779567951124E0915E0CF0915F0CE617B2
:10ADA000F70708F4AACEAECECF93DF93C82FD0E03A
:10ADB00004C00E946D4A0E94B41C8091810B9E01C8
:10ADC000280F311D21313105A4F7DF91CF9108956E
:10ADD0002F923F924F925F926F927F928F929F92AB
:10ADE000AF92BF92CF92DF92EF92FF920F931F9399
:10ADF000DF93CF93CDB7DEB7EF970FB6F894DEBFF2
:10AE00000FBECDBF4C017EAB6DAB58AF4FAB09AFA2
:10AE10001AAF2BAF3CAFEDAEDA01AD90BD90CD9047
:10AE2000DD90BCABABABC601B501F4012081318133
:10AE3000428153810E9442C66BA37CA38DA39EA333
:10AE4000AFA9B8AD1496ED90FD900D911C91179798
:10AE5000C801B701F40124813581468157810E94E0
:10AE600042C66F8F78A389A39AA32091EF0B3091EC
:10AE7000F00B4091F10B5091F20B2FA738AB49AB7F
:10AE80005AAB8091C70B9091C80BA091C90BB091A0
:10AE9000CA0B8BA79CA7ADA7BEA72091940B30919E
:10AEA000950B4091960B5091970B2FA338A749A76C
:10AEB0005AA7D601C501B0588B8F9C8FAD8FBE8F1E
:10AEC000A801970150582F8B388F498F5A8FADA901
:10AED000BEA96D917D918D919C912BA13CA14DA11D
:10AEE0005EA10E9441C65B016C01EDA9FEA96481CF
:10AEF0007581868197812F8D38A149A15AA10E9421
:10AF000041C63B014C016B8D7C8D8D8D9E8DA401C6
:10AF100093010E94B8C97B018C016F89788D898D5E
:10AF20009A8DA60195010E94B8C99B01AC01C80188
:10AF3000B7010E9441C61B012C016B8D7C8D8D8D4C
:10AF40009E8DA60195010E94B8C97B018C016F8975
:10AF5000788D898D9A8DA40193010E94B8C99B01B7
:10AF6000AC01C801B7010E9442C69B01AC01C201FD
:10AF7000B1010E94B5C65B016C0120E030E040E009
:10AF800050E00E9408C7882354F4C601B5012BED98
:10AF90003FE049EC50E40E9442C65B016C01FDAD0C
:10AFA000FF2351F0C601B5012BED3FE049EC50E421
:10AFB0000E9441C65B016C01C601B5019F7729ADB6
:10AFC0003AAD4BAD5CAD0E94B8C93B014C012FE6D8
:10AFD00032E143E85AE30E9408C787FDE5C1E090EB
:10AFE000460CF090470C0091480C1091490CC80198
:10AFF000B70120E030E040E752E40E9416C918167D
:10B00000F4F4C801B7012DE83AE748E85CE30E9490
:10B01000B8C90E9477C79B016430710514F023E022
:10B0200030E0B901882777FD8095982F0E94AAC744
:10B030009B01AC01C401B3010E940FC702C0C4014F
:10B04000B3010E94E5C70E947CC77E8B6D8B2D8962
:10B050003E89232B21F441E050E05E8B4D8BAD897E
:10B06000BE89BD0180E090E00E94A8C77B018C01F1
:10B07000C601B501A80197010E940FC7698B7A8BA1
:10B080008B8B9C8B2FA538A949A95AA98BA59CA568
:10B09000ADA5BEA5281B390B4A0B5B0B2FA738AB00
:10B0A00049AB5AABCA01B9010E94AAC72FA138A562
:10B0B00049A55AA50E94B8C9A80197010E940FC7C7
:10B0C0006D877E878F87988B69897A898B899C8920
:10B0D00020E030E040E05FEB0E94B8C929893A895E
:10B0E0004B895C890E94B8C920E030E040E85FE30A
:10B0F0000E9442C669877A878B879C876BA57CA54F
:10B100008DA59EA50E94AAC72FA138A549A55AA51D
:10B110000E94B8C969837A838B839C83A1E0B0E0E5
:10B12000BFAFAEAF99240DC1892D992787FD9095AA
:10B1300083709070892B41F40E946D4A0E94B41C68
:10B140008EE69FE00E944B9AB8E1B9150CF446C018
:10B150006B8D7C8D8D8D9E8D29893A894B895C897B
:10B160000E94B8C97B018C016F89788D898D9A8D79
:10B1700029853A854B855C850E94B8C99B01AC0145
:10B18000C801B7010E9442C67B018C016B8D7C8D8A
:10B190008D8D9E8D29853A854B855C850E94B8C929
:10B1A0005B016C016F89788D898D9A8D29893A8927
:10B1B0004B895C890E94B8C99B01AC01C601B501ED
:10B1C0000E9441C66B8F7C8F8D8F9E8F9394C70199
:10B1D000D8018F8B988FA98FBA8F61C0EEADFFAD6C
:10B1E000BF0180E090E00E94A8C729893A894B8975
:10B1F0005C890E94B8C97B018C01C8010E940CC700
:10B200006D837E838F839887B701C8010E941BCA14
:10B210003B014C01AFA9B8ADED90FD900D911C9193
:10B2200017FB109517F91095EBA9FCA92080318028
:10B2300042805380C801B7012D813E814F815885DE
:10B240000E94B8C95B016C01C201B101A401930164
:10B250000E94B8C99B01AC01C601B5010E9442C65B
:10B260006B8F7C8F8D8F9E8FC801B701A4019301D6
:10B270000E94B8C97B018C01C201B1012D813E81C0
:10B280004F8158850E94B8C99B01AC01C801B70124
:10B290000E9441C66F8B788F898F9A8F992469811C
:10B2A0007A818B819C812D853E854F8558890E94AE
:10B2B00042C669837A838B839C8300D000D0CDB64D
:10B2C000DEB60894C11CD11C6BA17CA18DA19EA1EE
:10B2D0002B8D3C8D4D8D5E8D0E9442C67B018C0175
:10B2E0006F8D78A189A19AA12F89388D498D5A8DAA
:10B2F0000E9442C69B01AC0180E89FE4A3ECB7E446
:10B30000F60180839183A283B383C801B7010F2E16
:10B31000F0E8EF2EFFE4FF2EF3EC0F2FF7E41F2FE2
:10B32000F02DA980BA80CB80DC800E944B732EADBB
:10B330003FAD2F5F3F4F3FAF2EAF0F900F900F905D
:10B340000F904EAD5FAD8D899E894817590708F45F
:10B35000EBCE00D000D0ADA9BEA96D917D918D91AD
:10B360009C91139714962D913D914D915C91179757
:10B370001C96AD90BD90CD90DC901F970F2EF0E8FD
:10B38000EF2EFFE4FF2EF3EC0F2FF7E41F2FF02D2D
:10B39000EDB7FEB7E182F282038314830E944B7300
:10B3A0000F900F900F900F90EF960FB6F894DEBFAE
:10B3B0000FBECDBFCF91DF911F910F91FF90EF9006
:10B3C000DF90CF90BF90AF909F908F907F906F90C5
:10B3D0005F904F903F902F9008952F923F924F9201
:10B3E0005F926F927F928F929F92AF92BF92CF9215
:10B3F000DF92EF92FF920F931F93DF93CF93CDB71E
:10B40000DEB761970FB6F894DEBF0FBECDBF3090A8
:10B41000800B232D30E03F872E8783E790E0289F25
:10B42000A001299F500D389F500D1124425B5B4FA6
:10B430005C874B877FB7F8946091820B5091800BAB
:10B440005D87651729F06F3011F460E001C06F5F10
:10B4500020E030E040E050E003E710E018C0862F25
:10B4600090E0809FF001819FF00D909FF00D1124DE
:10B47000E25BFB4F83819481A581B6816F3011F42B
:10B4800060E001C06F5F280F391F4A1F5B1F283C17
:10B490008FEA380780E0480780E0580730F49D8540
:10B4A0006917E9F602C03A9402C023E730E0361685
:10B4B00099F0832D90E0829FF001839FF00D929F81
:10B4C000F00D1124E25BFB4F808181FD05C033202C
:10B4D00051F70FE0302EEBCFAD853A16B1F0232DAA
:10B4E00030E083E790E0289FF001299FF00D389F1E
:10B4F000F00D1124E25BFB4F808181FF06C0BFE0AD
:10B500003B1611F4332401C03394ED853E16F9F453
:10B5100083E790E02E853F85289F8001299F100DAD
:10B52000389F100D1124025B1B4FD80111968C918E
:10B530001197806811968C9311977FBF8C918460CE
:10B540008C938B859C850E942551F801D5C5232DB0
:10B5500030E03A87298783E790E0289FF001299F10
:10B56000F00D389FF00D1124E25BFB4F8181806864
:10B5700081837FBF3D85332311F40FE002C00D8529
:10B580000150402F50E0598B488B83E790E0489F53
:10B59000F001499FF00D589FF00D1124E25BFB4F25
:10B5A0002281AE85BF85A89FF001A99FF00DB89FAD
:10B5B000F00D1124223031F4E25BFB4F82818230A6
:10B5C00031F431C0E25BFB4F8281823061F503E7E9
:10B5D00010E028893989209FF001219FF00D309FCC
:10B5E000F00D1124E25BFB4F8081826080834E85E9
:10B5F0005F85409FF001419FF00D509FF00D112499
:10B60000E25BFB4F8081846080838B859C850E94F8
:10B61000255189859A85809FF001819FF00D909F2B
:10B62000F00D112467C583E790E0AE85BF85A89F24
:10B630007001A99FF00CB89FF00C1124EEE4F4E027
:10B64000EE0EFF1E28893989289F8001299F100D41
:10B65000389F100D11240E0F1F1FD70199966D9161
:10B660007D918D919C919C97F80121A532A543A5D0
:10B6700054A50E9441C65B016C01D7019D966D9156
:10B680007D918D919C91D097F80125A536A547A570
:10B6900050A90E9441C67B018C01C601B501A601DB
:10B6A00095010E94B8C95B016C01C801B701A801EE
:10B6B00097010E94B8C99B01AC01C601B5010E9467
:10B6C00042C60E9425CA4B015C01C0904E0CD0902E
:10B6D0004F0CE090500CF090510CA70196010E9485
:10B6E00016C918164CF020E030E040E85FE32B83E9
:10B6F0003C834D835E830AC0C701B601A501940156
:10B700000E940FC76B837C838D839E8383E790E0C9
:10B710004E855F85489FD001499FB00D589FB00D61
:10B720001124A25BBB4F18962C91189730E04889E2
:10B730005989489FF001499FF00D589FF00D112441
:10B74000E25BFB4F808590E0282B392B26FF32C02F
:10B75000D1966D917D918D919C91D49721A932A91B
:10B7600043A954A90E9441C64B015C01E894B7F873
:10B77000C090520CD090530CE090540CF090550CAB
:10B78000C501B401A70196010E9416C9181694F4C8
:10B79000C701B601A50194010E940FC72B013C010E
:10B7A0006B817C818D819E81A30192010E9408C7DB
:10B7B000882324F44B805C806D807E8083E790E05A
:10B7C000EE85FF85E89FD001E99FB00DF89FB00D91
:10B7D0001124A25BBB4F28893989289FF001299F3A
:10B7E000F00D389FF00D1124E25BFB4FD5966D9163
:10B7F0007D918D919C91D89725A936A947A950ADE7
:10B800000E9441C64B015C01E894B7F8E0917502D3
:10B81000F0917602C788D08CE18CF28CC501B4011E
:10B82000A70196010E9416C9181684F4C701B60133
:10B83000A50194010E940FC76B017C01C301B201F5
:10B84000A70196010E9408C7882314F473016201BE
:10B8500003E710E048895989409FF001419FF00DAE
:10B86000509FF00D1124E25BFB4FC701B60121ADE3
:10B8700032AD43AD54AD0E94B8C96B017C018E85D9
:10B880009F85809FF001819FF00D909FF00D112406
:10B89000E25BFB4F11AD02ADB3ACA4ACC701B60186
:10B8A000212F302F4B2D5A2D0E9408C787FD06C02F
:10B8B000812F902FAB2DBA2D6C017D0183E790E095
:10B8C000A889B989A89FF001A99FF00DB89FF00D34
:10B8D0001124E25BFB4FEB5BFF4FC082D182E2821F
:10B8E000F382E554F04030E08085807F803809F4B1
:10B8F00031E020E083E790E04E855F85489FF001CE
:10B90000499FF00D589FF00D1124E25BFB4F80859D
:10B91000807F803809F421E0321761F103E710E0FD
:10B9200088899989809FF001819FF00D909FF00D8B
:10B930001124E25BFB4F808182608083AE85BF85EE
:10B94000A09FF001A19FF00DB09FF00D1124E25BCC
:10B95000FB4F8081846080838B859C850E9425516C
:10B9600029853A85209FF001219FF00D309FF00D31
:10B970001124C0C34D85242F30E083E790E0289F39
:10B980005001299FB00C389FB00C11248EE494E034
:10B99000A80EB91EADE4B0E0AA0EBB1EF501C08032
:10B9A000D180E280F38023EB3FEFA20EB31E4F83E2
:10B9B0003F81332319F44FE04F8303C05F8151501F
:10B9C0005F838F81882E9924D50111968C911197D0
:10B9D00081FF0CC0D9964C90D997DA965C90DA9793
:10B9E000DB966C90DB97DC967C9013C0C701B601A8
:10B9F000A70196010E94B8C9F501EF5BFF4F2081B6
:10BA00003181428153810E9442C60E9425CA2B0186
:10BA10003C0123E730E0829EF001839EF00D929E70
:10BA2000F00D1124E25BFB4FEB5BFF4F10810181B6
:10BA3000F280D380E554F040F98BE88BB201C3016A
:10BA4000212F302F4F2D5D2D0E9416C988230CF415
:10BA5000A1C0E889F989E35BFF4F60817181828130
:10BA60009381212F302F4F2D5D2D0E9408C78823F1
:10BA700091F1A889B9898C918E7F8C93E889F98995
:10BA8000EF5AFF4FC080718062805380E02E0D2DF1
:10BA90006C2D772D862D952D212F3E2D4F2D5D2D33
:10BAA0000E9408C787FD04C01C2DE72CF62C052D2D
:10BAB00023E730E0829EF001839EF00D929EF00D10
:10BAC0001124E556FB4F812F9E2DAF2DB02F808383
:10BAD0009183A283B38343E750E0849EF001859E67
:10BAE000F00D949EF00D1124ED56FB4FE080F18097
:10BAF00002811381F501E75BFF4F608171818281D3
:10BB000093819701A8010E9408C7882399F181E5D4
:10BB100090E0A80EB91ED501DC901196CC9011973B
:10BB200012967C90129713966C90EFEAFFEFAE0E90
:10BB3000BF1E6D2D7C2D872D962D9701A8010E948B
:10BB400008C787FD04C0ED2CFC2C072D162D29E419
:10BB500030E0A20EB31EC701D801F50180839183A6
:10BB6000A283B38327EB3FEFA20EB31ED5018C91C6
:10BB70008E7F8C9323E730E0829EF001839EF00D50
:10BB8000929EF00D1124E556FB4FC080D180E280DB
:10BB9000F38066C041E550E0A40EB51ED5011C91AE
:10BBA0001196EC9011971296FC90129713960C91A7
:10BBB000EFEAFFEFAE0EBF1E612F7E2D8F2D902F6F
:10BBC0009201A3010E9408C7882324F4142DE52CB8
:10BBD000F62C072D29E430E0A20EB31E812F9E2DF6
:10BBE000AF2DB02FF50180839183A283B38327EB20
:10BBF0003FEFA20EB31E43E750E0849EF001859E06
:10BC0000F00D949EF00D1124E156FB4FC080D180C1
:10BC1000E280F380B201C301A70196010E9408C728
:10BC200087FD04C0C201D3016C017D0183E790E070
:10BC3000889EF001899EF00D989EF00D1124E25B24
:10BC4000FB4FE35BFF4FC082D182E282F382ED546F
:10BC5000F04080818E7F8083D5018C918E7F8C9384
:10BC6000BF81B31571F0E3E7F0E08E9E50018F9E27
:10BC7000B00C9E9EB00C11242EE434E0A20EB31E34
:10BC800097CE83E790E049855A85489F7001499F88
:10BC9000F00C589FF00C11248EE494E0E80EF91E8D
:10BCA000A9E4B0E0EA0EFB1EF7016080718082809B
:10BCB000938027EB3FEFE20EF31E3F8138874885E4
:10BCC0004F3011F4188603C058855F5F5887888508
:10BCD000282E3324E3E7F0E02E9ED0012F9EB00DF6
:10BCE0003E9EB00D1124A25BBB4FBA83A983D7013E
:10BCF00011968C91119781FF0CC0D9961C91D99700
:10BD0000DA964C90DA97DB965C90DB97DC960C9198
:10BD100015C0C401B301A40193010E94B8C9F70181
:10BD2000EF5BFF4F20813181428153810E9442C6E7
:10BD30000E9425CA162F472E582E092FF701E35BC4
:10BD4000FF4FF98BE88B612F742D852D902F20816B
:10BD50003181428153810E9416C9F701EF5AFF4F8A
:10BD600018160CF0A8C0A080B180C280D380C40196
:10BD7000B301A60195010E9408C787FD03C06401B5
:10BD8000530118C0C601B501A60195010E94B8C9AA
:10BD9000F701EF5BFF4F20813181428153810E9487
:10BDA00042C60E9425CAA889B9896D937D938D9357
:10BDB0009C931397E9E4F0E0EE0EFF1ED701AD92DD
:10BDC000BD92CD92DD927D01CC901196DC901197C1
:10BDD00012960C91129713961C91E8EFFFEFEE0E5E
:10BDE000FF1ED701BC901196AC90119712969C90B3
:10BDF000129713968C90EBEBFFEFEE0EFF1EB60141
:10BE0000C8012B2D3A2D492D582D0E9408C787FDBA
:10BE100004C0CB2CDA2C092D182D23E730E0229E0C
:10BE2000F001239EF00D329EF00D1124E156FB4FE0
:10BE30006080718082809380B601C801A401930163
:10BE40000E9408C787FD04C0C601D8013C014D010E
:10BE500043E750E0249E8001259E100D349E100D76
:10BE60001124025B1B4F075B1F4FD8016D927D921F
:10BE70008D929C92139709541040F701E35BFF4F9A
:10BE8000D701AB5BBF4F60817181828193812D911E
:10BE90003D914D915C910E9408C7882341F4F701C0
:10BEA000808182608083D8018C9184608C93F701BB
:10BEB00080818E7FB4C0D7018C9186608E7F8C93F9
:10BEC000A080B180C280D380C601B501A4019301D6
:10BED0000E9416C918161CF06401530115C0C60152
:10BEE000B501A60195010E94B8C9F701EF5BFF4FAC
:10BEF00020813181428153810E9442C60E9425CA1D
:10BF0000162F472E582E092FE9E4F0E0EE0EFF1E03
:10BF1000D701AD92BD92CD92DC921397E8E0F0E0AC
:10BF2000EE0EFF1ED701DC901196CC901197129661
:10BF3000BC9012971396AC90EFEAFFEFEE0EFF1E47
:10BF40006D2D7C2D8B2D9A2D212F342D452D502F8D
:10BF50000E9408C787FD04C01D2D4C2C5B2C0A2DA8
:10BF60002DE430E0E20EF31E812F942DA52DB02F8D
:10BF7000F70180839183A283B38328EF3FEFE20E22
:10BF8000F31ED701DC901196CC9011971296BC90BD
:10BF900012971396FC90612F742D852D902F2D2DC7
:10BFA0003C2D4B2D5F2D0E9408C787FD04C01D2D21
:10BFB0004C2C5B2C0F2D23E730E0229EF001239EBA
:10BFC000F00D329EF00D1124E156FB4F6080718020
:10BFD00082809380612F742D852D902FA401930171
:10BFE0000E9408C787FD06C0812F942DA52DB02F74
:10BFF0003C014D0143E750E0249EF001259EF00DE9
:10C00000349EF00D1124E25BFB4FE75BFF4F608233
:10C01000718282829382E954F040808184608083BF
:10C0200058858D85581719F0E980FA8048CEE98146
:10C03000FA81EF5AFF4F10810181F280E380612F76
:10C04000702F8F2D9E2DA40193010E9408C787FD9C
:10C0500006C0812F902FAF2DBE2D3C014D01E981EF
:10C06000FA81E75BFF4F608271828282938213E7DD
:10C07000E12EF12CAF818A2F90E08E9D80018F9D63
:10C08000100D9E9D100D1124025B1B4FC8010E94D4
:10C0900025512FB7F894F80181818F778183FF8133
:10C0A000FF3011F41F8203C03F813F5F3F834F8108
:10C0B000842F90E08E9DF0018F9DF00D9E9DF00DE0
:10C0C0001124E25BFB4F8181806881832FBF8091C7
:10C0D000800B481779F68B859C850E94255183E754
:10C0E00090E0AE85BF85A89FF001A99FF00DB89F95
:10C0F000F00D1124E25BFB4F81818F778183619684
:10C100000FB6F894DEBF0FBECDBFCF91DF911F9168
:10C110000F91FF90EF90DF90CF90BF90AF909F90E6
:10C120008F907F906F905F904F903F902F900895E9
:10C130002F923F924F925F926F927F928F929F9237
:10C14000AF92BF92CF92DF92EF92FF920F931F9325
:10C15000DF93CF93CDB7DEB76B970FB6F894DEBF02
:10C160000FBECDBF4C011B014B8F25E530E0820E89
:10C17000931ED401AD90BD90CD90DC90EBEAFFEF23
:10C180008E0E9F1ED40118968C9180732091460CC0
:10C190003091470C4091480C5091490C8823D9F0BC
:10C1A00070900E0C60900F0C5090100C4090110C81
:10C1B000C901DA017C018D01672D762D852D942D25
:10C1C000A80197010E9408C787FD09C0872D962DF9
:10C1D000A52DB42D02C0C901DA017C018D01C60173
:10C1E000B50120E034E244E75BE40E94B8C9A8014D
:10C1F00097010E940FC72B013C018091FF0B90E03B
:10C20000E6E096958795EA95E1F7B82FB170BC8B7B
:10C210008091810B8A30C0F5C301B20120E034E285
:10C2200044E758E40E9408C7882374F5E090810B26
:10C2300060E074E284E798E4A30192010E9441C6A1
:10C2400020E030E040E450E40E94B8C95B016C019A
:10C25000FF240894E11CF11C0027F7FC0095102F27
:10C26000C801B7010E94AAC79B01AC01C601B50174
:10C270000E940FC79B01AC01C301B2010E9442C6DC
:10C280002B013C01E1E0EC8BC301B2010E9477C7B6
:10C29000D40113966D937D938D939C9316978EE6A0
:10C2A0009FE00E944B9AF401E159FF4F6081718138
:10C2B000828193810E94AAC76F8B788F898F9A8F12
:10C2C000C301B2012F89388D498D5A8D0E940FC745
:10C2D0000E9477C75B016C01F4016084762C64FED8
:10C2E00030C0D1016D917D918D919C919F7720E01F
:10C2F00034E244E75BE40E94B8C97B018C016F899A
:10C30000788D898D9A8D2091EB013091EC014091CF
:10C31000ED015091EE010E94B8C99B01AC01C8012A
:10C32000B7010E940FC70E9477C769837A838B8306
:10C330009C836A157B058C059D053CF05B016C01B7
:10C3400004C019821A821B821C8275FE30C0F10162
:10C3500064817581868197819F7720E034E244E78C
:10C360005BE40E94B8C97B018C016F89788D898D4F
:10C370009A8D2091EF013091F0014091F10150919F
:10C38000F2010E94B8C99B01AC01C801B7010E942B
:10C390000FC70E9477C76D837E838F8398876A1546
:10C3A0007B058C059D053CF05B016C0104C01D8282
:10C3B0001E821F82188676FE32C0D10118966D91BA
:10C3C0007D918D919C911B979F7720E034E244E70B
:10C3D0005BE40E94B8C97B018C016F89788D898DDF
:10C3E0009A8D2091F3013091F4014091F501509123
:10C3F000F6010E94B8C99B01AC01C801B7010E94B7
:10C400000FC70E9477C769877A878B879C876A15D1
:10C410007B058C059D053CF05B016C0104C0198611
:10C420001A861B861C8667FE30C0F10164857585FF
:10C43000868597859F7720E034E244E75BE40E949D
:10C44000B8C97B018C016F89788D898D9A8D209177
:10C45000F7013091F8014091F9015091FA010E94E1
:10C46000B8C99B01AC01C801B7010E940FC70E9467
:10C4700077C76D877E878F87988B6A157B058C05BC
:10C480009D053CF05B016C0104C01D861E861F8665
:10C49000188AC601B5016139F1E07F07F0E08F0726
:10C4A000F0E09F0724F461E971E080E090E029E585
:10C4B00030E0820E931ED4016D937D938D939C93F7
:10C4C0001397E7EAFFEF8E0E9F1E0E94AAC77B011B
:10C4D0008C01F401E159FF4F608171818281938168
:10C4E0000E94AAC79B01AC01C801B7010E94B8C94C
:10C4F0006B017C0160E074E284E79BE4A701960194
:10C500000E940FC72B013C01D40118968C911897FB
:10C51000082F10E084FF2DC019966D917D918D91AB
:10C520009C911C970E94AAC79B01AC01C701B60150
:10C530000E940FC70E9477C769837A838B839C838D
:10C54000C301B201F10120813181428153810E94F6
:10C55000B8C9D40199966D937D938D939C939C97C4
:10C56000017110700031110569F4DC01CB01B05884
:10C5700004C080E090E0A0E0B0E0F40181A792A7C1
:10C58000A3A7B4A7D40118968C911897082F10E090
:10C5900085FF2DC01D966D917D918D919C91509739
:10C5A0000E94AAC79B01AC01C701B6010E940FC738
:10C5B0000E9477C76D837E838F839887C301B20102
:10C5C000F10124813581468157810E94B8C9D40187
:10C5D0009D966D937D938D939C93D097027210706E
:10C5E0000032110569F4DC01CB01B05804C080E0D1
:10C5F00090E0A0E0B0E0F40185A796A7A7A7B0ABB4
:10C60000D40118968C911897082F10E086FF2DC042
:10C6100051966D917D918D919C9154970E94AAC7DE
:10C620009B01AC01C701B6010E940FC70E9477C7EA
:10C6300069877A878B879C87C301B201F1012085C6
:10C640003185428553850E94B8C9D401D1966D9336
:10C650007D938D939C93D4970474107000341105CE
:10C6600069F4DC01CB01B05804C080E090E0A0E0A8
:10C67000B0E0F40181AB92ABA3ABB4ABD40118969C
:10C680001C91189717FF2FC055966D917D918D9134
:10C690009C9158970E94AAC79B01AC01C701B601A3
:10C6A0000E940FC70E9477C76D877E878F87988B00
:10C6B000C301B201F10124853585468557850E9465
:10C6C000B8C9D401D5966D937D938D939C93D897DB
:10C6D0001878103841F4DC01CB01B058F40185AB77
:10C6E00096ABA7ABB0AFF401EB5AFF4F60817181FD
:10C6F00082819381A30192010E94B8C9D401D99685
:10C700006D937D938D939C93DC9718968C91E82F75
:10C71000F0E0FB8BEA8BCF01887890708838910528
:10C7200029F028EA3BE03E8B2D8B04C088E99BE092
:10C730009E8B8D8B79EA272E6FE5362E53E6452E9C
:10C7400048E5542E66247724AA24BB2480E190E097
:10C75000062C02C0880F991F0A94E2F7AA89BB89A8
:10C760008A239B23892B41F1E1E0F0E0EC0FFD1FD0
:10C77000EA0DFB1D60817181828193810E94AAC7AD
:10C780007B018C01ED89FE89EA0DFB1D60817181C1
:10C79000828193810E94A8C79B01AC01C801B701A7
:10C7A0000E94B8C96B017C01B101C201A7019601C9
:10C7B0000E9408C7882324F4C101D2016C017D01C5
:10C7C0000894611C711CE4E0F0E0AE0EBF1EF4E0C2
:10C7D0006F16710429F0D701C60116012D01B6CFDD
:10C7E000D4011296BC900B2D10E0000F111F000F0A
:10C7F000111FF401E00FF11F81859285A385B48597
:10C80000B595A79597958795F40181A392A3A3A3C6
:10C81000B4A3858F968FA78FB0A3818F928FA38F9C
:10C82000B48F60E070E080E89FE321AD32AD43ADAE
:10C8300054AD0E940FC72DE330E0820E931ED40149
:10C840006D937D938D939C9313970C0F1D1FF8018F
:10C8500061817281838194810E94AAC79B01AC018E
:10C86000C701B6010E940FC70E947CC724E230E0D6
:10C87000820E931ED4016D937D938D939D934D01F4
:10C880000E94A8C720E030E040E858E40E94B8C900
:10C8900020E034E244E75BE40E940FC70E947CC7BB
:10C8A000F40160837183828393832BE93FEF820ECF
:10C8B000931E84010F5B1F4F85E590E0880E991E43
:10C8C000D4012D913D914D915C91EBEAFFEF8E0EDD
:10C8D0009F1ECA01B9010E9442C6A70196010E948B
:10C8E000B8C9D401D9962D913D914D915C91DC97B9
:10C8F0000E94B8C920E034E244E75BE40E940FC71D
:10C90000F801608371838283938360914E0C7091F0
:10C910004F0C8091500C9091510C20E030E040E0A1
:10C920005FE30E94B8C91B012C01D4011896BC9189
:10C93000B98B6B2E7724B6FF5AC0F401E1A8F2A898
:10C9400003A914A9F2E0BF16F9F46091520C70919A
:10C95000530C8091540C9091550C20E030E040E055
:10C960005FE30E94B8C9D401D9962D913D914D91B4
:10C970005C91DC970E94B8C9A80197015F770E947B
:10C980000FC77B018C0135C057016801E894D7F8C7
:10C990006091520C7091530C8091540C9091550CF5
:10C9A00020E030E040E05FE30E94B8C97B018C01E9
:10C9B000C601B501A80197010E9416C91816BCF45A
:10C9C000C801B701F40121AD32AD43AD54AD0E94B1
:10C9D000B8C9A60195010E940FC77B018C01C20155
:10C9E000B101A80197010E9408C7882314F48201AD
:10C9F0007101F989F7FF3CC020E762227724E091BA
:10CA00007502F0917602672831F16789708D818D0A
:10CA1000928D20E030E040E05FE30E94B8C9D4018D
:10CA2000D9962D913D914D915C91DC970E94B8C9AA
:10CA3000F40125A936A947A950AD5F770E940FC719
:10CA40005B016C01C801B701A60195010E9408C7EE
:10CA500087FD0EC00FC06789708D818D928D20E09B
:10CA600030E040E05FE30E94B8C95B016C0102C0A6
:10CA700057016801D40112968C91823048F4E090FD
:10CA80000E0CF0900F0C0091100C1091110C0AC0BC
:10CA9000823081F4E090120CF090130C0091140C91
:10CAA0001091150CC801B701A60195010E9408C795
:10CAB000882314F486017501F401D1ACC2ACB3AC87
:10CAC000A4ACC801B7012D2D3C2D4B2D5A2D0E9431
:10CAD00008C787FD06C08D2D9C2DAB2DBA2D7C017E
:10CAE0008D0121E530E0820E931ED401ED92FD927E
:10CAF0000D931C931397F40112930293F292E29216
:10CB0000DF011E930E93FE92EE924D01E7EBFFEFD5
:10CB10008E0E9F1ED401D996AD90BD90CD90DC9025
:10CB2000DC97C801B701A80197010E94B8C9F401B8
:10CB3000EF5BFF4F20813181428153810E9442C6C9
:10CB40007B018C01C601B501A60195010E94B8C9FF
:10CB50009B01AC01C801B7010E9416C9882324F0CB
:10CB6000F4018181826081838401075A1F4FD801BB
:10CB70002D913D914D915C9160E074E284EF90E0E5
:10CB80000E94E1CAE9E6F0E08E0E9F1ED4012D93CB
:10CB90003C93E7E9FFEF8E0E9F1E8EE69FE00E941A
:10CBA0004B9A0E94ED59F80180819181A281B38155
:10CBB0008F5C9740A040B04018F02C89222329F0C8
:10CBC00084E0D40117968C9320C081E0F401878320
:10CBD000E281F0E0EE0FFF1FEE0FFF1FE80DF91DE1
:10CBE00081859285A385B485F40185A396A3A7A327
:10CBF000B0A781A392A3A3A3B4A3858F968FA78F79
:10CC0000B0A3818F928FA38FB48FFB8DFF2331F060
:10CC100086E490E090934D0480934C048091800BC7
:10CC20008F5F8093800B803110F01092800B809189
:10CC3000010C80618093010C9FB7F8948091810B67
:10CC40008F5F8093810B9FBF6B960FB6F894DEBF0A
:10CC50000FBECDBFCF91DF911F910F91FF90EF904D
:10CC6000DF90CF90BF90AF909F908F907F906F900C
:10CC70005F904F903F902F9008952F923F924F9248
:10CC80005F926F927F928F929F92AF92BF92CF925C
:10CC9000DF92EF92FF920F931F93DF93CF93CDB765
:10CCA000DEB7A1970FB6F894DEBF0FBECDBF182F29
:10CCB0006A8F8091FF0B8E7F8093FF0B81E00E9433
:10CCC000D4568A8D60E00E9430528B8B8091800B0D
:10CCD000282E3324112371F083E790E0289EF00181
:10CCE000299EF00D389EF00D1124E25BFB4F80E190
:10CCF00081830CC083E790E0289EF001299EF00D0F
:10CD0000389EF00D1124E25BFB4F118283E790E027
:10CD1000289EF001299EF00D389EF00D1124E25B53
:10CD2000FB4F10822A8D222311F482E0808383E757
:10CD300090E0289E7001299EF00C389EF00C112482
:10CD40008701025B1B4FD80118961C920E94BF6A94
:10CD5000E0914C0CF0914D0CFD8BEC8B2BEB3BE000
:10CD60003A8B298B87E5682E84E0782E6E0C7F1C29
:10CD700044245524AA24BB24085F1F4F4801C8013E
:10CD80000D969D8F8C8FCF01A0E0B0E08E8F9F8F8E
:10CD9000A8A3B9A34B8EF501ED51F44F8081918189
:10CDA000A281B3818E8B9F8BA88FB98FE989FA8975
:10CDB00080819181A281B3812E893F89488D598DCF
:10CDC000281B390B4A0B5B0BD3012D933D934D93DD
:10CDD0005C93139757FD0DC021E030E0042C02C096
:10CDE000220F331F0A94E2F7F4018081822B8083A3
:10CDF0000CC088279927DC01821B930BA40BB50B71
:10CE0000F30180839183A283B383F3E04F1649F546
:10CE10002C893D892436310521F1AC8DBD8D6D9174
:10CE20007D918D919C910E94AAC77B018C016E8D92
:10CE30007F8D88A199A10E94A8C79B01AC01C80160
:10CE4000B7010E94B8C92AE037ED43E25CE30E94D3
:10CE5000B8C90E9477C7EC8DFD8D60837183828392
:10CE60009383D301ED90FD900D911C91B1E0CB2EF9
:10CE7000D12CCC0EDD1ECA0CDB1CC801B7010E94F0
:10CE8000AAC7F501E857F44F2081318142815381CF
:10CE90000E94B8C9F6016083718382839383E11491
:10CEA000F1040105110561F020E130E00B8C02C0B6
:10CEB000220F331F0A94E2F7D4018C91822B8C93BA
:10CEC000E989FA898E899F89A88DB98D819391937B
:10CED000A193B193FA8BE98B0894411C511C24E077
:10CEE00030E0A20EB31E620E731E30E1A316B10431
:10CEF00009F050CF83E790E0289E8001299E100D15
:10CF0000389E100D1124025B1B4FD80118968C918E
:10CF1000807F59F4BB89BB2309F41BC11092810B9C
:10CF20008091800B8093820B14C16D847E848F84EA
:10CF300098886091640C7091650C8091660C90915A
:10CF4000670CA40193010E9442C66093640C709325
:10CF5000650C8093660C9093670CF80125853685E7
:10CF600047855089C184D284E384F484C216D306F1
:10CF7000E406F506A4F481899289A389B48982170D
:10CF80009307A407B5075CF485899689A789B08DB6
:10CF900082179307A407B50714F481E036C083E72E
:10CFA00090E0289EF001299EF00D389EF00D11248E
:10CFB000E25BFB4F21893289438954892C153D0559
:10CFC0004E055F055CF485899689A789B08D8C151F
:10CFD0009D05AE05BF0514F4128218C083E790E0EA
:10CFE000289EF001299EF00D389EF00D1124E25B81
:10CFF000FB4F85899689A789B08D82179307A4076F
:10D00000B50714F482E001C083E0828383E790E0F7
:10D010009C01229EC001239E900D329E900D1124F2
:10D020009C01225B3B4FD9011296EC91F0E0EE0F90
:10D03000FF1FEE0FFF1FE80FF91FE25BFB4F81851B
:10D040009285A385B48521593F4FF901808391834F
:10D05000A283B3832F563040D90118968C91482E65
:10D060005524C20180779070892B09F456C029811C
:10D070003A814B815C81ED80FE800F811885CA0169
:10D08000B9010E94B8C95B016C01C801B701A801D0
:10D0900097010E94B8C99B01AC01C601B5010E946D
:10D0A00042C67B018C0164015301E894D7F846FE27
:10D0B0000EC029853A854B855C85CA01B9010E945D
:10D0C000B8C99B01AC01C801B7010E9442C60E94C9
:10D0D00025CA962E872E782E692ED601C501750198
:10D0E0008D01692D782D872D962D9501AD010E941A
:10D0F00008C787FD04C0E92CF82C072D162D83E7FF
:10D1000090E0289EF001299EF00D389EF00D11242C
:10D11000ED55FB4FC701D80106C0F901EB5AFF4F8F
:10D12000D401C301BF7780839183A283B38383E754
:10D1300090E0FC012E9EC0012F9E900D3E9E900D12
:10D140001124825B9B4FBE016F5F7F4F4A8D0E940F
:10D150009860A1960FB6F894DEBF0FBECDBFCF91F9
:10D16000DF911F910F91FF90EF90DF90CF90BF90D4
:10D17000AF909F908F907F906F905F904F903F9077
:10D180002F9008952F923F924F925F926F927F92CD
:10D190008F929F92AF92BF92CF92DF92EF92FF92C7
:10D1A0000F931F93DF93CF93CDB7DEB760970FB682
:10D1B000F894DEBF0FBECDBF1B012C012D833E8333
:10D1C0004F835887E986FA860B871C87AD86BE8613
:10D1D000CF86D88A0E94AAC72091880B3091890BEC
:10D1E00040918A0B50918B0B0E94B8C92091D70BAC
:10D1F0003091D80B4091D90B5091DA0B0E9442C666
:10D200003B014C01CB01D4018093D70B9093D80BF9
:10D21000A093D90BB093DA0B6D817E818F819885B5
:10D220000E94AAC720918C0B30918D0B40918E0BE0
:10D2300050918F0B0E94B8C92091DB0B3091DC0B11
:10D240004091DD0B5091DE0B0E9442C65B016C01E8
:10D25000CB01D6018093DB0B9093DC0BA093DD0B0D
:10D26000B093DE0BC801B7010E94AAC72091900BB2
:10D270003091910B4091920B5091930B0E94B8C941
:10D280002091DF0B3091E00B4091E10B5091E20BCC
:10D290000E9442C67B018C01CB01D8018093DF0B39
:10D2A0009093E00BA093E10BB093E20BB301C401A8
:10D2B0009501A6010E946A6C882309F49EC021147E
:10D2C00031044104510449F420E83FE443EC57E4BD
:10D2D00029833A834B835C830CC08091D70B909158
:10D2E000D80BA091D90BB091DA0B89839A83AB83C9
:10D2F000BC832D813E814F81588521153105410523
:10D30000510559F40F2EF0E82F2EFFE43F2EF3ECD9
:10D310004F2EF7E45F2EF02D08C02090DB0B3090ED
:10D32000DC0B4090DD0B5090DE0B89859A85AB8538
:10D33000BC850097A105B10559F40F2EF0E86F2EBA
:10D34000FFE47F2EF3EC8F2EF7E49F2EF02D08C024
:10D350006090DF0B7090E00B8090E10B9090E20BFF
:10D3600000D000D00DB71EB70F5F1F4F6091C70BE5
:10D370007091C80B8091C90B9091CA0B2D853E8589
:10D380004F855889620F731F841F951F0E94AAC77B
:10D390002091940B3091950B4091960B5091970BE7
:10D3A0000E94B8C95B016C018DA19EA1AFA1B8A577
:10D3B000F80180839183A283B38369817A818B8111
:10D3C0009C81A2019101840173010E944B730F9013
:10D3D0000F900F900F9080E00E943C6B89A58823EE
:10D3E00011F00E94D11C0E9421C4609340047093EC
:10D3F0004104809342049093430460960FB6F894DE
:10D40000DEBF0FBECDBFCF91DF911F910F91FF9077
:10D41000EF90DF90CF90BF90AF909F908F907F90D4
:10D420006F905F904F903F902F9008952F923F9272
:10D430004F925F926F927F928F929F92AF92BF9224
:10D44000CF92DF92EF92FF920F931F93DF93CF93D0
:10D45000CDB7DEB72090460C3090470C4090480C7A
:10D460005090490C6090BB0B7090BC0B8090BD0B32
:10D470009090BE0B660E771E881E991E6092E30B7D
:10D480007092E40B8092E50B9092E60B8091BF0BBB
:10D490009091C00BA091C10BB091C20B820F931F52
:10D4A000A41FB51F8093E70B9093E80BA093E90BA3
:10D4B000B093EA0B8091C30B9091C40BA091C50B64
:10D4C000B091C60B8E0D9F1DA01FB11F8093EB0B5B
:10D4D0009093EC0BA093ED0BB093EE0B8091C70BE8
:10D4E0009091C80BA091C90BB091CA0B8A0D9B1DDE
:10D4F000AC1DBD1D8093EF0B9093F00BA093F10B2F
:10D50000B093F20B8D899E89AF89B88D8093460CBC
:10D510009093470CA093480CB093490C8A8D60E01F
:10D520000E943D662092460C3092470C4092480C77
:10D530005092490C80E00E943C6B898D882311F049
:10D540000E94D11C0E9421C4609340047093410446
:10D550008093420490934304CF91DF911F910F91E8
:10D56000FF90EF90DF90CF90BF90AF909F908F9003
:10D570007F906F905F904F903F902F900895809193
:10D58000000C85FD57C02091160C3091170C40916E
:10D59000180C5091190C8091E30B9091E40BA09121
:10D5A000E50BB091E60B281739074A075B0744F4EF
:10D5B0002093E30B3093E40B4093E50B5093E60B81
:10D5C00020911A0C30911B0C40911C0C50911D0C99
:10D5D0008091E70B9091E80BA091E90BB091EA0BD9
:10D5E000281739074A075B0744F42093E70B309369
:10D5F000E80B4093E90B5093EA0B20911E0C3091FD
:10D600001F0C4091200C5091210C8091EB0B9091BC
:10D61000EC0BA091ED0BB091EE0B281739074A07E0
:10D620005B0744F42093EB0B3093EC0B4093ED0B32
:10D630005093EE0B0895EF92FF920F931F93609318
:10D64000F30B7093F40B8093F50B9093F60B2093F0
:10D65000F70B3093F80B4093F90B5093FA0BE092D1
:10D66000FB0BF092FC0B0093FD0B1093FE0B1F9134
:10D670000F91FF90EF9008954F925F926F927F927B
:10D680009F92AF92BF92CF92DF92EF92FF920F9351
:10D690001F93DF93CF9300D000D0CDB7DEB7982E85
:10D6A0006091BB0B7091BC0B8091BD0B9091BE0B38
:10D6B0000E94AAC72091880B3091890B40918A0B58
:10D6C00050918B0B0E94B8C97B018C016091BF0BFC
:10D6D0007091C00B8091C10B9091C20B0E94AAC7A0
:10D6E00020918C0B30918D0B40918E0B50918F0BB4
:10D6F0000E94B8C95B016C016091C30B7091C40BAF
:10D700008091C50B9091C60B0E94AAC72091900BE7
:10D710003091910B4091920B5091930B0E94B8C99C
:10D7200069837A838B839C8329813A814B815C81D5
:10D73000C901DA018093D30B9093D40BA093D50B3E
:10D74000B093D60BC801B7012091560C3091570CFD
:10D750004091580C5091590C0E9441C62B013C013C
:10D76000CB01D3018093CB0B9093CC0BA093CD0B2B
:10D77000B093CE0BC601B50120915A0C30915B0CD1
:10D7800040915C0C50915D0C0E9441C67B018C0164
:10D79000CB01D8018093CF0B9093D00BA093D10BEA
:10D7A000B093D20B992011F1C201D3018093D70B12
:10D7B0009093D80BA093D90BB093DA0BC701D80183
:10D7C0008093DB0B9093DC0BA093DD0BB093DE0B0F
:10D7D00029813A814B815C81C901DA018093DF0B99
:10D7E0009093E00BA093E10BB093E20B0F900F909E
:10D7F0000F900F90CF91DF911F910F91FF90EF90BD
:10D80000DF90CF90BF90AF909F907F906F905F9090
:10D810004F90089580E00E943C6B8091CB0B9091DB
:10D82000CC0BA091CD0BB091CE0B8093690C909353
:10D830006A0CA0936B0CB0936C0C8091CF0B909101
:10D84000D00BA091D10BB091D20B80936D0C909323
:10D850006E0CA0936F0CB093700C8091D30B9091D1
:10D86000D40BA091D50BB091D60B8093710C9093F3
:10D87000720CA093730CB093740C6091C70B7091F1
:10D88000C80B8091C90B9091CA0B0E94AAC7209126
:10D89000E7013091E8014091E9015091EA010E94CD
:10D8A000B8C96093750C7093760C8093770C909345
:10D8B000780C8091460C9091470CA091480CB09147
:10D8C000490C8093790C90937A0CA0937B0CB093C5
:10D8D0007C0C089581E008959F92AF92BF92CF9201
:10D8E000DF92EF92FF920F931F93CF93DF930EE699
:10D8F0001FE0C80165EB77E140E00E945199C80143
:10D900000E94E5B6E0902A0CF0902B0C00912C0CB4
:10D9100010912D0C80911E0C90911F0CA091200C49
:10D92000B091210CE81AF90A0A0B1B0B88279927DA
:10D93000DC018E199F09A00BB10B8093C30B909350
:10D94000C40BA093C50BB093C60B00D000D000D081
:10D95000EDB7FEB73196EE0CFF1C001F111F809132
:10D96000030290910402A0910502B0910602CDB786
:10D97000DEB789839A83AB83BC8399249394948282
:10D98000958260E070E080E090E020E030E040E0F0
:10D9900050E0AA24BB2465010E94166A80912A0CDB
:10D9A00090912B0CA0912C0CB0912D0C8093C30B5B
:10D9B0009093C40BA093C50BB093C60BCDB6DEB647
:10D9C0000894C11CD11C2091E3013091E4014091E5
:10D9D000E5015091E601CA01B9010E9442C60E94C8
:10D9E00077C77B018C0160910302709104028091E2
:10D9F00005029091060220E030E040E450E40E94ED
:10DA00000FC7F601608371838283938394821582AA
:10DA100060E070E080E090E020E030E040E050E046
:10DA2000AA24BB2465010E94166ACDB6DEB608940E
:10DA3000C11CD11C2091E3013091E4014091E5012A
:10DA40005091E601CA01B9010E9442C620E030E0CF
:10DA500040E050EC0E94B8C90E9477C77B018C015E
:10DA60006091030270910402809105029091060278
:10DA700020E030E040E450E40E940FC7E6016883F4
:10DA800079838A839B839C829D8260E070E080E042
:10DA900090E020E030E040E050E0AA24BB246501A3
:10DAA0000E94166A80912A0C90912B0CA0912C0C4C
:10DAB000B0912D0C8093C30B9093C40BA093C50B16
:10DAC000B093C60BEDB7FEB736960FB6F894FEBF0F
:10DAD0000FBEEDBFDF91CF911F910F91FF90EF909F
:10DAE000DF90CF90BF90AF909F9008959F92AF929C
:10DAF000BF92CF92DF92EF92FF920F931F93CF933B
:10DB0000DF930EE61FE0C8016CEB77E140E00E9476
:10DB10005199C8010E94E5B62091260C3091270C3E
:10DB20004091280C5091290C80911A0C90911B0C5B
:10DB3000A0911C0CB0911D0C281B390B4A0B5B0BE0
:10DB400088279927DC01821B930BA40BB50B8093CC
:10DB5000BF0B9093C00BA093C10BB093C20B00D02E
:10DB600000D000D0EDB7FEB73196220F331F441F0F
:10DB7000551F8091FF0190910002A0910102B09188
:10DB80000202CDB7DEB789839A83AB83BC83992425
:10DB900093949482958260E070E080E090E0EE24BF
:10DBA000FF248701AA24BB2465010E94166A809184
:10DBB000260C9091270CA091280CB091290C8093F1
:10DBC000BF0B9093C00BA093C10BB093C20B0DB7CA
:10DBD0001EB70F5F1F4F6091DF017091E0018091D0
:10DBE000E1019091E20120E030E040EA50E40E943F
:10DBF000B8C90E9477C76B017C016091FF017091E9
:10DC00000002809101029091020220E030E040E4A5
:10DC100050E40E940FC7F80160837183828393836D
:10DC20009482158260E070E080E090E0A7019601A8
:10DC3000EE24FF248701AA24BB2465010E94166AF2
:10DC4000CDB6DEB60894C11CD11C2091DF01309105
:10DC5000E0014091E1015091E201CA01B9010E9445
:10DC600042C620E030E040EA50EC0E94B8C90E9471
:10DC700077C77B018C016091FF0170910002809158
:10DC800001029091020220E030E040E450E40E9462
:10DC90000FC7E601688379838A839B839C829D8278
:10DCA00060E070E080E090E0A8019701EE24FF249E
:10DCB0008701AA24BB2465010E94166A0DB71EB70E
:10DCC0000F5F1F4F6091DF017091E0018091E101D2
:10DCD0009091E2010E9477C79B01AC018091FF0106
:10DCE00090910002A0910102B0910202F80180839C
:10DCF0009183A283B3839482158260E070E080E018
:10DD000090E0EE24FF2487010E94166A8091260C81
:10DD10009091270CA091280CB091290C8093BF0BF7
:10DD20009093C00BA093C10BB093C20B8DB79EB75D
:10DD300006960FB6F8949EBF0FBE8DBFDF91CF91B0
:10DD40001F910F91FF90EF90DF90CF90BF90AF9019
:10DD50009F9008959F92AF92BF92CF92DF92EF92E1
:10DD6000FF920F931F930EE61FE0C80163EC77E16B
:10DD700040E00E945199C8010E94E5B66091220CD2
:10DD80007091230C8091240C9091250C2091160CFD
:10DD90003091170C4091180C5091190C621B730BA9
:10DDA000840B950B22273327A901261B370B480B21
:10DDB000590B2093BB0B3093BC0B4093BD0B50937E
:10DDC000BE0B00D000D000D0EDB7FEB73196660F85
:10DDD000771F881F991F2091FB013091FC01409112
:10DDE000FD015091FE01ADB7BEB711962D933D9345
:10DDF0004D935C931497992493949482958220E098
:10DE000030E040E050E0EE24FF248701AA24BB2448
:10DE100065010E94166A8091220C9091230CA091BA
:10DE2000240CB091250C8093BB0B9093BC0BA0935A
:10DE3000BD0BB093BE0B0DB71EB70F5F1F4F6091A8
:10DE4000DB017091DC018091DD019091DE0120E029
:10DE500030E040EA50E40E94B8C90E9477C76B01E5
:10DE60007C016091FB017091FC018091FD0190911A
:10DE7000FE0120E030E040E450E40E940FC7F801CA
:10DE8000608371838283938394821582C701B60174
:10DE900020E030E040E050E0EE24FF248701AA2497
:10DEA000BB2465010E94166ACDB6DEB60894C11C7B
:10DEB000D11C2091DB013091DC014091DD015091BA
:10DEC000DE01CA01B9010E9442C620E030E040EA0A
:10DED00050EC0E94B8C90E9477C77B018C01609109
:10DEE000FB017091FC018091FD019091FE0120E009
:10DEF00030E040E450E40E940FC7D6016D937D935B
:10DF00008D939C93139714969C92149715969C92BC
:10DF1000C801B70120E030E040E050E0EE24FF24EB
:10DF20008701AA24BB2465010E94166A0DB71EB79B
:10DF30000F5F1F4F6091DB017091DC018091DD016B
:10DF40009091DE010E9477C72091FB013091FC0186
:10DF50004091FD015091FE01F801208331834283FD
:10DF600053839482158220E030E040E050E0EE24BC
:10DF7000FF2487010E94166A8091220C9091230C45
:10DF8000A091240CB091250C8093BB0B9093BC0BFB
:10DF9000A093BD0BB093BE0B8DB79EB706960FB680
:10DFA000F8949EBF0FBE8DBF1F910F91FF90EF9011
:10DFB000DF90CF90BF90AF909F9008952F923F92A7
:10DFC0004F925F926F927F928F929F92AF92BF9289
:10DFD000CF92DF92EF92FF920F931F93DF93CF9335
:10DFE000CDB7DEB72B970FB6F894DEBF0FBECDBF0F
:10DFF0009B878A872091B90B2987DC018C9122238A
:10E0000009F0A7C083FF34C01A962D913D914D9120
:10E010005C911D978091870B882351F0CA01B9014B
:10E0200023E333E34BEC51E40E94B8C99B01AC01FC
:10E03000CA01B9012091F30B3091F40B4091F50B1B
:10E040005091F60B0E9441C6DC019B01AC0120936C
:10E05000CB0B3093CC0B4093CD0B5093CE0BCB011D
:10E060008093D70B9093D80BA093D90BB093DA0B76
:10E07000EA85FB85808184FF32C02685378540890B
:10E0800051898091870B882351F0CA01B90123E39C
:10E0900033E34BEC51E40E94B8C99B01AC01CA01C7
:10E0A000B9012091F70B3091F80B4091F90B509189
:10E0B000FA0B0E9441C6DC019B01AC012093CF0BFF
:10E0C0003093D00B4093D10B5093D20BCB01809364
:10E0D000DB0B9093DC0BA093DD0BB093DE0BAA85DA
:10E0E000BB858C9185FFDBC052962D913D914D9162
:10E0F0005C9155978091870B882351F0CA01B90133
:10E1000023E333E34BEC51E40E94B8C99B01AC011B
:10E11000CA01B9012091FB0B3091FC0B4091FD0B22
:10E120005091FE0B0E9441C6DC019B01AC01209383
:10E13000D30B3093D40B4093D50B5093D60BCB011C
:10E140008093DF0B9093E00BA093E10BB093E20B75
:10E15000A6C083FF34C0E090D70BF090D80B00919D
:10E16000D90B1091DA0BEA85FB852285338544852E
:10E1700055858091870B882351F0CA01B90123E3AB
:10E1800033E34BEC51E40E94B8C99B01AC01C801D8
:10E19000B7010E9442C6DC019B01AC012093D70B62
:10E1A0003093D80B4093D90B5093DA0BCB0180936B
:10E1B000CB0B9093CC0BA093CD0BB093CE0BAA8539
:10E1C000BB858C9184FF34C0E090DB0BF090DC0BBE
:10E1D0000091DD0B1091DE0B1E962D913D914D911E
:10E1E0005C9151978091870B882351F0CA01B90146
:10E1F00023E333E34BEC51E40E94B8C99B01AC012B
:10E20000C801B7010E9442C6DC019B01AC0120930A
:10E21000DB0B3093DC0B4093DD0B5093DE0BCB011B
:10E220008093CF0B9093D00BA093D10BB093D20BD4
:10E23000EA85FB85808185FF32C0E090DF0BF0909E
:10E24000E00B0091E10B1091E20B228933894489A4
:10E2500055898091870B882351F0CA01B90123E3C6
:10E2600033E34BEC51E40E94B8C99B01AC01C801F7
:10E27000B7010E9442C6DC019B01AC012093DF0B79
:10E280003093E00B4093E10B5093E20BCB01809372
:10E29000D30B9093D40BA093D50BB093D60B2091B6
:10E2A000D70B3091D80B4091D90B5091DA0B2983C1
:10E2B0003A834B835C832090DB0B3090DC0B4090E7
:10E2C000DD0B5090DE0B8091DF0B9091E00BA09165
:10E2D000E10BB091E20B8D839E83AF83B887CA01B7
:10E2E000B9012091560C3091570C4091580C509127
:10E2F000590C0E9442C62091DB013091DC01409113
:10E30000DD015091DE010E94B8C920E030E040E01C
:10E310005FE30E9442C60E94E5C73B014C01C20177
:10E32000B10120915A0C30915B0C40915C0C5091E2
:10E330005D0C0E9442C62091DF013091E0014091C6
:10E34000E1015091E2010E94B8C920E030E040E0D4
:10E350005FE30E9442C60E94E5C75B016C016D81CC
:10E360007E818F8198852091E3013091E401409175
:10E37000E5015091E6010E94B8C920E030E040E09C
:10E380005FE30E9442C60E94E5C77B018C01C40185
:10E39000B3010E9477C76093E30B7093E40B809303
:10E3A000E50B9093E60BC601B5010E9477C7609319
:10E3B000E70B7093E80B8093E90B9093EA0BC8018D
:10E3C000B7010E9477C76093EB0B7093EC0B8093BF
:10E3D000ED0B9093EE0BAA85BB858C9186FF4AC10D
:10E3E0008091270283FD46C15696ED90FD900D91D8
:10E3F0001C9159976090E7017090E8018090E901C5
:10E400009090EA01C801B701A40193010E94B8C924
:10E410009B01AC018091870B882351F0CA01B9019F
:10E4200023E333E34BEC51E40E94B8C99B01AC01F8
:10E43000CA01B9010E9477C75B016C01B985BB2392
:10E4400021F48091BA0B882359F1E0917502F09183
:10E45000760264A575A586A597A520E030E046E183
:10E4600053E40E9408C787FD0BC0C801B7019F771E
:10E4700020E030E040E253E40E9416C918161CF474
:10E48000AA24BB2465018091C70B9091C80BA09171
:10E49000C90BB091CA0B8A0D9B1DAC1DBD1DF2C0EE
:10E4A000E0917502F091760264A575A586A597A501
:10E4B00020E030E046E153E40E9408C787FD26C013
:10E4C0008091C70B9091C80BA091C90BB091CA0B5A
:10E4D000A6019501281B390B4A0B5B0BCA01B90138
:10E4E0000E94AAC77B018C01E89417F9C401B3010B
:10E4F00020E030E040E253E40E94B8C99B01AC0147
:10E50000C801B7010E9416C9181644F4A092C70B9F
:10E51000B092C80BC092C90BD092CA0BA092EF0B5D
:10E52000B092F00BC092F10BD092F20BAA85BB8592
:10E530008D919C91119790FF3FC08091870BC09067
:10E540004A0CD0904B0C8823D1F05A966D917D9156
:10E550008D919C915D972FE737EB4AE85BE30E9432
:10E56000B8C97B018C01B601882777FD8095982F6B
:10E570000E94AAC79B01AC01C801B70113C0B60134
:10E58000882777FD8095982F0E94AAC7EA85FB858A
:10E59000228D338D448D558D0E94B8C92EE333EC06
:10E5A0004EE259E30E94B8C96093460C7093470C41
:10E5B0008093480C9093490C69817A818B819C816E
:10E5C000A2019101ED80FE800F8118850E946A6C86
:10E5D000882391F48091EF0B9091F00BA091F10BB7
:10E5E000B091F20B8093C70B9093C80BA093C90B0B
:10E5F000B093CA0B80E025C0AA85BB852D913C91C4
:10E60000C90188739070892BD1F426FD02C060E0A7
:10E6100017C060E02091EF0B3091F00B4091F10BAF
:10E620005091F20B8091C70B9091C80BA091C90B30
:10E63000B091CA0B281739074A075B0709F061E058
:10E64000862F2B960FB6F894DEBF0FBECDBFCF91AD
:10E65000DF911F910F91FF90EF90DF90CF90BF90CF
:10E66000AF909F908F907F906F905F904F903F9072
:10E670002F9008958091C70B9091C80BA091C90B62
:10E68000B091CA0B8093EF0B9093F00BA093F10B1A
:10E69000B093F20B4BCF2F923F924F925F926F92BB
:10E6A0007F928F929F92AF92BF92CF92DF92EF9222
:10E6B000FF920F931F93DF93CF93CDB7DEB73B014C
:10E6C0004C0119012A0120E83FE443EC57E40E9481
:10E6D00008C7882341F46090CB0B7090CC0B8090DE
:10E6E000CD0B9090CE0BC201B10120E83FE443EC8A
:10E6F00057E40E9408C7882341F42090CF0B309044
:10E70000D00B4090D10B5090D20BC801B70120E83C
:10E710003FE443EC57E40E9408C7882341F4E090AB
:10E72000D30BF090D40B0091D50B1091D60B6092C7
:10E73000CB0B7092CC0B8092CD0B9092CE0B209293
:10E74000CF0B3092D00B4092D10B5092D20BE09273
:10E75000D30BF092D40B0093D50B1093D60BC401BE
:10E76000B3012091560C3091570C4091580C5091A8
:10E77000590C0E9442C63B014C01C201B1012091DB
:10E780005A0C30915B0C40915C0C50915D0C0E94D6
:10E7900042C61B012C01C401B30120E83FE443EC55
:10E7A00057E40E9408C78823F1F0C401B301209107
:10E7B000DB013091DC014091DD015091DE010E94CE
:10E7C000B8C920E030E040E05FE30E9442C60E940A
:10E7D000E5C70E9477C76093E30B7093E40B8093C7
:10E7E000E50B9093E60BC201B10120E83FE443EC56
:10E7F00057E40E9408C78823F1F0C201B1012091BB
:10E80000DF013091E0014091E1015091E2010E946D
:10E81000B8C920E030E040E05FE30E9442C60E94B9
:10E82000E5C70E9477C76093E70B7093E80B80936E
:10E83000E90B9093EA0BC801B70120E83FE443ECF1
:10E8400057E40E9408C78823F1F0C801B70120915E
:10E85000E3013091E4014091E5015091E6010E940D
:10E86000B8C920E030E040E05FE30E9442C60E9469
:10E87000E5C70E9477C76093EB0B7093EC0B809316
:10E88000ED0B9093EE0BC601B50120E83FE443EC9D
:10E8900057E40E9408C78823B1F0C601B501209152
:10E8A000E7013091E8014091E9015091EA010E94AD
:10E8B000B8C90E9477C76093EF0B7093F00B8093F9
:10E8C000F10B9093F20B6D897E898F89988D20E8EA
:10E8D0003FE443EC57E40E9408C7882361F08D8928
:10E8E0009E89AF89B88D8093460C9093470CA09376
:10E8F000480CB093490C81E061E00E943D66CF91E5
:10E90000DF911F910F91FF90EF90DF90CF90BF901C
:10E91000AF909F908F907F906F905F904F903F90BF
:10E920002F9008953F924F925F926F927F928F92B5
:10E930009F92AF92BF92CF92DF92EF92FF920F938E
:10E940001F93582E462E342E6090CB0B7090CC0B1C
:10E950008090CD0B9090CE0BA090CF0BB090D00BB1
:10E96000C090D10BD090D20BE090D30BF090D40B91
:10E970000091D50B1091D60B8091000C8160809393
:10E98000000C552011F00E94AA6E442011F00E9444
:10E99000766D332011F00E946C6C552041F0609030
:10E9A000320C7090330C8090340C9090350C4420D5
:10E9B00041F0A0903A0CB0903B0CC0903C0CD09031
:10E9C0003D0C332041F0E090420CF090430C00915C
:10E9D000440C1091450C81E00E943C6B00D000D0AB
:10E9E0008091FB019091FC01A091FD01B091FE018D
:10E9F000EDB7FEB781839283A383B483C401B301CF
:10EA0000A60195010F2EF0E8AF2EFFE4BF2EF3EC28
:10EA1000CF2EF7E4DF2EF02D0E944B731092AE0F35
:10EA20000F900F900F900F900E94341A1F910F912A
:10EA3000FF90EF90DF90CF90BF90AF909F908F901E
:10EA40007F906F905F904F903F9008956F927F926C
:10EA50008F929F92AF92BF92CF92DF92EF92FF92EE
:10EA60000F931F93362FF42FA22F370148018823CD
:10EA700011F0E0E012C0662331F060E87FE483EC3F
:10EA800097E4E0E023C0442339F060E87FE483ECBE
:10EA900097E49B01AC0139C0E1E06091690C709191
:10EAA0006A0C80916B0C90916C0C6093D70B7093F7
:10EAB000D80B8093D90B9093DA0BEE2339F43323E0
:10EAC00029F420E83FE443EC57E412C020916D0C98
:10EAD00030916E0C40916F0C5091700C2093DB0BB9
:10EAE0003093DC0B4093DD0B5093DE0BEE2369F487
:10EAF000FF2359F40F2EF0E8EF2EFFE4FF2EF3EC86
:10EB00000F2FF7E41F2FF02D10C0E090710CF09044
:10EB1000720C0091730C1091740CE092DF0BF09268
:10EB2000E00B0093E10B1093E20BAA2359F40F2E94
:10EB3000F0E8AF2EFFE4BF2EF3ECCF2EF7E4DF2E8C
:10EB4000F02D08C0A090750CB090760CC090770C9A
:10EB5000D090780C00D000D0EDB7FEB76182728201
:10EB6000838294820E944B738091790C90917A0CED
:10EB7000A0917B0CB0917C0C8093460C9093470C39
:10EB8000A093480CB093490C0F900F900F900F90EA
:10EB90001F910F91FF90EF90DF90CF90BF90AF90BB
:10EBA0009F908F907F906F9008951F93182F909152
:10EBB000FF0B90FF42C0882309F43FC042C0916020
:10EBC0009093FF0B5E9A5E9A159A0E942C3F112338
:10EBD00041F560E070E080E090E040E020E00E94DD
:10EBE000373F60E070E080E090E041E020E00E948C
:10EBF000373F60E070E080E090E040E00E94733BCF
:10EC00008EE69FE06BED77E140E00E9451998EE641
:10EC10009FE00E94E5B68091000C88608093000C14
:10EC200010C08EE69FE06AEC77E140E00E945199C7
:10EC30008EE69FE00E94E5B604C08091000C83FF41
:10EC4000BECF1F910895EF92FF920F931F930E94E2
:10EC5000B41C8EE69FE00E944B9A0E9421C49B0147
:10EC6000AC018091810B882349F0209340043093BC
:10EC7000410440934204509343043CC080914004BB
:10EC800090914104A0914204B091430479018A011A
:10EC9000E81AF90A0A0B1B0B809144049091450471
:10ECA000A0914604B09147040097A105B10549F031
:10ECB0008E159F05A007B10720F480E00E94D5754E
:10ECC00005C08091000C877F8093000C8091D1015A
:10ECD0009091D201A091D301B091D4010097A105E8
:10ECE000B10541F08E159F05A007B10718F481E02A
:10ECF0000E94D5751F910F91FF90EF9008952F926C
:10ED00003F924F925F926F927F928F929F92AF92BB
:10ED1000BF92CF92DF92EF92FF920F931F93DF93F8
:10ED2000CF93CDB7DEB728970FB6F894DEBF0FBEEE
:10ED3000CDBF8091DB019091DC01A091DD01B0910C
:10ED4000DE018D839E83AF83B8872090320C309094
:10ED5000330C4090340C5090350CC201B10120911D
:10ED60002E0C30912F0C4091300C5091310C0E94A0
:10ED700042C69B01AC016D817E818F8198850E9486
:10ED8000B8C90E9477C76093160C7093170C8093D4
:10ED9000180C9093190CA090DF01B090E001C09086
:10EDA000E101D090E20160903A0C70903B0C8090B1
:10EDB0003C0C90903D0CC401B3012091360C309175
:10EDC000370C4091380C5091390C0E9442C69B017F
:10EDD000AC01C601B5010E94B8C90E9477C7609313
:10EDE0001A0C70931B0C80931C0C90931D0C80913B
:10EDF000E3019091E401A091E501B091E6018983DE
:10EE00009A83AB83BC83E090420CF090430C00915A
:10EE1000440C1091450CC801B70120913E0C309173
:10EE20003F0C4091400C5091410C0E9442C69B0106
:10EE3000AC0169817A818B819C810E94B8C90E9452
:10EE400077C760931E0C70931F0C8093200C9093D7
:10EE5000210C6D817E818F819885A20191010E9494
:10EE6000B8C90E9477C76093220C7093230C8093DB
:10EE7000240C9093250CC601B501A40193010E94B6
:10EE8000B8C90E9477C76093260C7093270C8093B3
:10EE9000280C9093290C69817A818B819C81A8012F
:10EEA00097010E94B8C90E9477C760932A0C70939B
:10EEB0002B0C80932C0C90932D0CAA24BB24F501D1
:10EEC000E552FE4FE080F1800281138158E8C52EA3
:10EED0005BE0D52ECA0CDB1C60E070E080E89FE3AD
:10EEE000A80197010E940FC7D6016D937D938D9362
:10EEF0009C93139748E9C42E4BE0D42ECA0CDB1C1C
:10EF0000F501E95FFD4FC801B701208131814281E0
:10EF100053810E94B8C90E947CC7F6016083718347
:10EF20008283938338EAC32E3BE0D32ECA0CDB1CCA
:10EF3000F501E95EFD4FC801B701208131814281B1
:10EF400053810E94B8C90E947CC7D6016D937D93FE
:10EF50008D939C931397E4E0F0E0AE0EBF1EF0E1BA
:10EF6000AF16B10409F0ABCFC0900702A090080221
:10EF70006090090220900A02E0901702F0901802B7
:10EF80000091190210911A026C2D7A2D862D922D66
:10EF9000A80197010E9408C787FD06C08C2D9A2DF5
:10EFA000A62DB22D7C018D016D817E818F8198858A
:10EFB000A80197010E94B8C99B01AC0160E070E014
:10EFC00080E090E40E940FC70E9425CA9B01AC011B
:10EFD000C801B7010E94B8C960930E0C70930F0C62
:10EFE0008093100C9093110CC0900F02A09010020F
:10EFF0006090110220901202E0901F02F090200217
:10F0000000912102109122026C2D7A2D862D922DD5
:10F01000A80197010E9408C787FD06C08C2D9A2D74
:10F02000A62DB22D7C018D0169817A818B819C8115
:10F03000A80197010E94B8C99B01AC0160E070E093
:10F0400080E090E40E940FC70E9425CA9B01AC019A
:10F05000C801B7010E94B8C96093120C7093130CD9
:10F060008093140C9093150C8091FF0B8D7F8093EF
:10F07000FF0B28960FB6F894DEBF0FBECDBFCF9121
:10F08000DF911F910F91FF90EF90DF90CF90BF9095
:10F09000AF909F908F907F906F905F904F903F9038
:10F0A0002F90089588E10FB6F89480936000109235
:10F0B00060000FBE579A3E9A239A3D9A3F9A229A31
:10F0C000569A5E9A569A5E9A0D9A159A0C9A149AC6
:10F0D0003A98429A3B98439A3C98449A249A2C989E
:10F0E000559A5D980E94A81980E090E0A8E4B2E4E7
:10F0F0008093460C9093470CA093480CB093490C16
:10F1000084E690E090934B0C80934A0C90934D0CC6
:10F1100080934C0C20E030E040E050E02093DF0B87
:10F120003093E00B4093E10B5093E20B2093DB0B09
:10F130003093DC0B4093DD0B5093DE0B2093D70B09
:10F140003093D80B4093D90B5093DA0B10924804AC
:10F150001092490410924A0410924B041092C70B6B
:10F160001092C80B1092C90B1092CA0B1092C30BCD
:10F170001092C40B1092C50B1092C60B1092BF0BCD
:10F180001092C00B1092C10B1092C20B1092BB0BCD
:10F190001092BC0B1092BD0B1092BE0B80E090E061
:10F1A000A0EAB1E480934E0C90934F0CA093500CC6
:10F1B000B093510C8DEC9CECACECBEE38093520C04
:10F1C0009093530CA093540CB093550C20935A0C6D
:10F1D00030935B0C40935C0C50935D0C2093560C69
:10F1E0003093570C4093580C5093590C88E893E196
:10F1F000A0E0B0E08093020C9093030CA093040C69
:10F20000B093050C81E0809328021092600C10925C
:10F21000610C1092620C1092630C2093640C30937A
:10F22000650C4093660C5093670C8093FF0B80E055
:10F2300090E8A4E8B3E480932E0C90932F0CA09355
:10F24000300CB093310C80E090E0A6E6B3E48093FC
:10F25000360C9093370CA093380CB093390C80E0A7
:10F2600090E0ABE6B3E480933E0C90933F0CA09308
:10F27000400CB093410C80E090E0A4E3B2EC8093AA
:10F28000320C9093330CA093340CB093350C80E087
:10F2900090E0A0EAB0EC80933A0C90933B0CA093E2
:10F2A0003C0CB0933D0C2093420C3093430C4093A4
:10F2B000440C5093450C1092680C8EE69FE00E941F
:10F2C0007EC30E94E12C4091D5015091D6016091FE
:10F2D000D7017091D80183E294E00E94274E64E642
:10F2E00070E080E090E00E942FC48BE893E00E94E1
:10F2F000262B0E9401510E944F410E946E350E94B0
:10F300007F760E94221A0E94A9190E946C4D80E00B
:10F310000E94FD3F82ED9CE00E94AE7E08950E9417
:10F32000B62908950E9452780895FC0189E18183ED
:10F330001482148E13A216A2E05CFF4F1082339643
:10F340001082B996108233961082369711921192DC
:10F3500010828091000C8D7F8093000C0895FC0139
:10F36000E759FF4F1192119210828091000C8D7F0E
:10F370008093000C8091010C887F8093010C8FE2B8
:10F380008093C30F1092C40F1092FB0F0895FC01DD
:10F39000E659FF4F8081EA56F040882351F0E75943
:10F3A000FF4F81E080838091010C82608B7F80938E
:10F3B000010C0895DA01FB0190E02EE28C9180327D
:10F3C00029F0983009F421938C9181939F5F9B30B1
:10F3D00011F01196F3CF1082CF01089582ED9CE0D9
:10F3E0000E94957908950F931F93CF93DF93EC01BB
:10F3F0008B01C659DF4F8881CA56D0408823C1F09F
:10F40000C759DF4F1882C956D040CE01805C9F4F4C
:10F410000E94FD89CE01B80141E00E94E195882358
:10F4200019F08AE19FE002C08CE29FE00E94262B47
:10F43000DF91CF911F910F910895FC0180913C0DB8
:10F44000882361F0E759FF4F10828091010C897F7A
:10F450008093010C8FEE97E10E94262B08950F9365
:10F460001F93CF93DF93EC018B01C659DF4F888147
:10F47000CA56D0408823E9F0C759DF4F1882C956D1
:10F48000D040CE01805C9F4F0E94FD89CE01B80123
:10F490000E942295882331F4CE01B8010E94309554
:10F4A000882319F08DEF9EE002C08AE09FE00E9461
:10F4B000262BDF91CF911F910F9108950F931F93EA
:10F4C000CF93DF939C01EC01C559DF4F88818823DE
:10F4D00081F08901005C1F4FC8010E946888C80143
:10F4E0000E94FD8918828BEE9EE00E94262B1092CE
:10F4F000AE0FDF91CF911F910F910895EF92FF9280
:10F500000F931F93CF93DF93EC017B01C659DF4F1D
:10F510008881CA56D040882349F18E01005C1F4F74
:10F52000C8010E94FD89C759DF4F1882C956D040D3
:10F53000CE0160E00E94078AC801B70146E50E943B
:10F540002695882319F485EC9EE00DC08EE69FE099
:10F5500062EE77E140E00E945199C559DF4F81E0AA
:10F56000888389ED9EE0B7010E94192BDF91CF912E
:10F570001F910F91FF90EF900895CF93DF93EC01CF
:10F58000C659DF4F8881CA56D0408823A1F0CF5991
:10F59000DF4F488159816A817B8183EA9EE00E9426
:10F5A000D82AFE01729162915291429181E294E0D7
:10F5B0000E94AF2A04C085EB9EE00E94262BDF91BB
:10F5C000CF910895BF92CF92DF92EF92FF920F9367
:10F5D0001F93DF93CF93CDB7DEB76D970FB6F89437
:10F5E000DEBF0FBECDBF8C01D62EC72EB42E06595E
:10F5F0001F4FF80180810A561040882309F468C023
:10F6000007591F4FF80110820956104080E4E82E78
:10F61000F12CE00EF11E1C821982C7010E94FD89A7
:10F62000DE011196F801B3968DE101900D928150A3
:10F63000E1F7C701BE016F5F7F4F4D2D5C2D21E0CB
:10F640000E94B3948823F1F18D2D9C2D6FE270E020
:10F650000E94E6189C01009721F48D2D9C2D9C01A1
:10F6600002C02F5F3F4FBB2091F480E79EE0B901BD
:10F670000E940E2B0D5A1F4FF8014081518162816B
:10F680007381035510408DE79EE00E94AF2A0F5909
:10F690001F4FF80110821182128213820E50104007
:10F6A000F80180819181A281B381065F1F4FF8012B
:10F6B00080839183A283B38384E89EE00E94262BFB
:10F6C00081E007C0BB2021F482E99EE00E94262B46
:10F6D00080E06D960FB6F894DEBF0FBECDBFCF9120
:10F6E000DF911F910F91FF90EF90DF90CF90BF902F
:10F6F0000895EF92FF920F931F93DF93CF93CDB7AF
:10F70000DEB76D970FB6F894DEBF0FBECDBF8C018C
:10F7100019821C8282E59EE00E94262BC80160E0CF
:10F720000E94078A0B5F1F4F7E010894E11CF11CA9
:10F73000C701B8010E945087C70160E040E00E9405
:10F74000289782E69EE00E94262B6D960FB6F894CD
:10F75000DEBF0FBECDBFCF91DF911F910F91FF9004
:10F76000EF900895CF92DF92EF92FF920F931F9345
:10F77000CF93DF937C018B01EA011CC0F7018081EC
:10F78000992787FD90950E9438CB6C01F801808104
:10F79000992787FD90950E9438CB2197C816D906E6
:10F7A00021F0FC2DF81B8F2F08C00894E11CF11CE0
:10F7B0000F5F1F4F209711F780E0DF91CF911F91CE
:10F7C0000F91FF90EF90DF90CF900895DF92EF922E
:10F7D000FF920F931F93CF93DF937C01EB0104C043
:10F7E0000894E11CF11C2196F701D080DD2081F006
:10F7F0008D2D992787FD90950E9438CB8C018881AB
:10F80000992787FD90950E9438CB0817190741F377
:10F810008D2D992787FD90950E9438CB182F8881D0
:10F82000992787FD90950E9438CB181B812FDF9177
:10F83000CF911F910F91FF90EF90DF900895CF929D
:10F84000DF92EF92FF920F931F93DF93CF93CDB789
:10F85000DEB7C456D0400FB6F894DEBF0FBECDBFA2
:10F860007C019B0180E490E0E80EF91ED7011C9218
:10F87000E0ECFFEFEE0EFF1EDB014D915C91119766
:10F880009EE7C92E9FEFD92EC422D522E0E8F0E0F2
:10F89000CE2ADF2ADA82C98254FF34C012968D91B3
:10F8A0009C9113979C838B8357FD02C044E00CC04E
:10F8B000FB01A3A9B4A9FD0101900020E9F731974C
:10F8C000EA1BFB0BED8345E0D9018C9181FF0AC057
:10F8D000FE01E40FF11D16968D919C91179792836E
:10F8E00081834E5FF901808182FF1FC0FE01E40F1A
:10F8F000F11DD90118968D919C911997928381835E
:10F900004E5F13C041FD02C042E004C0FB0186818E
:10F910008B8343E0D9018C9182FF07C0FE01E40F85
:10F92000F11D18968C9181834F5FF901808183FFCF
:10F930000DC0BE01640F711D82859385A485B585B8
:10F94000FB0181839283A383B4834C5FD9018C91A3
:10F9500084FF0FC0BE01640F711D1E968D919D9195
:10F960000D90BC91A02DFB0181839283A383B4836E
:10F970004C5FD9018C9185FF0FC0BE01640F711DD2
:10F9800052968D919D910D90BC91A02DFB0181838C
:10F990009283A383B4834C5FD9018C9186FF0FC0FF
:10F9A000BE01640F711D56968D919D910D90BC9175
:10F9B000A02DFB0181839283A383B4834C5FD90183
:10F9C0008D919C91119790FF0FC0BE01640F711D26
:10F9D0005A968D919D910D90BC91A02DFB01818334
:10F9E0009283A383B4834C5FD9018D919C9111972D
:10F9F00091FF07C0FE01E40FF11D5E968C9181839B
:10FA00004F5FF9018081918192FF0DC0BE01640FAB
:10FA1000711D878D90A1A1A1B2A1FB018183928369
:10FA2000A383B4834C5FD9018D919C91119793FF6F
:10FA30000FC0BE01640F711D93968D919D910D9025
:10FA4000BC91A02DFB0181839283A383B4834C5F7F
:10FA5000D90112968C91129780FF0FC0BE01640FDE
:10FA6000711D97968D919D910D90BC91A02DFB01DC
:10FA700081839283A383B4834C5FD90112968C91C6
:10FA8000129781FF0FC0BE01640F711D9B968D916F
:10FA90009D910D90BC91A02DFB0181839283A38346
:10FAA000B4834C5FD9018D919C91119797FF35C01C
:10FAB000D3966D917C91D49794FF1BC0FB0101906C
:10FAC0000020E9F73197E61BF70B3E2F242F9E2FDE
:10FAD000DE0111960AC08D01020F111DFB018191FB
:10FAE000BF01F80180832F5F91509923A1F7430F45
:10FAF00014C020E030E0DE011196842F820F8D01CA
:10FB0000080F111DFB018191BF01F80180832F5F58
:10FB10003F4F2031310589F7405F142F20E030E05E
:10FB2000A0E0B0E0BE016F5F7F4F1FC0512F1631C4
:10FB300008F055E1FB01952F8191280F311D2F3FD2
:10FB4000310510F02F5F3040A20FB31FAF3FB1055A
:10FB500010F0AF5FB040915079F75150852F90E091
:10FB60005F5F0196680F791F151B1123F9F6BE011F
:10FB70006F5F7F4FFB01E40FF11D20834F5FFB019F
:10FB8000E40FF11DA083F0E8CF16D10429F485E03D
:10FB900096E00E942B2B07C04F5FC701805C9F4FF0
:10FBA00050E00E94798D80E490E0E80EF91ED701C4
:10FBB0008C91882321F08CE39EE00E94262BCC5967
:10FBC000DF4F0FB6F894DEBF0FBECDBFCF91DF91F0
:10FBD0001F910F91FF90EF90DF90CF900895EF92DB
:10FBE000FF920F931F93CF93DF93EC0180913C0D15
:10FBF0008823B9F18091010C8B7F8093010C6623DF
:10FC000061F16091EB017091EC018091ED019091B7
:10FC1000EE0120E030E040E05FE30E94B8C97B01E4
:10FC20008C0181E061E040E021E00E942675609156
:10FC3000F3017091F4018091F5019091F6012DECA2
:10FC40003CEC4CE45FE30E94B8C97B018C0180E08E
:10FC500060E041E020E00E942675C759DF4F81E057
:10FC60008883DF91CF911F910F91FF90EF900895BE
:10FC70008F929F92AF92BF92CF92DF92EF92FF92BC
:10FC80000F931F93FC0180913C0D882309F45BC006
:10FC9000E759FF4F10828091010C84608093010C22
:10FCA000662309F450C00E94E5290E940A6C00D026
:10FCB00000D08DB69EB60894811C911CA090320C89
:10FCC000B090330CC090340CD090350C60913A0C4D
:10FCD00070913B0C80913C0C90913D0C2091360C26
:10FCE0003091370C4091380C5091390C0E9442C62B
:10FCF0007B018C016091EB017091EC018091ED0131
:10FD00009091EE0120E030E040E05FE30E94B8C94E
:10FD1000F4016083718382839383C601B501A801D6
:10FD200097010F2EF0E8EF2EFFE4FF2EF3EC0F2FDC
:10FD3000F7E41F2FF02D570168010E944B730F90BD
:10FD40000F900F900F901F910F91FF90EF90DF9009
:10FD5000CF90BF90AF909F908F900895FF920F9398
:10FD60001F93CF93DF93EC018C0106591F4FF801CD
:10FD700010826FE144E00E94128B882329F48FE205
:10FD80009EE00E94262B22C0FF24F394F801F0820B
:10FD90008091010C81608093010CCE0160E00E9493
:10FDA000078ACE0160E071E041E00E94E27A882398
:10FDB00069F0F8018081882349F0C759DF4FF88244
:10FDC0008091010C82608B7F8093010CDF91CF9139
:10FDD0001F910F91FF900895FC01E759FF4F10828A
:10FDE000E956F040CF010E94AE7E0895CF93DF9395
:10FDF000DC01EB01BA0180E090E020E2FE01E80FB7
:10FE0000F91F208301968B309105C1F747E030E060
:10FE100023C0282F8E3219F0E9E0FAE108C04A30F9
:10FE200049F14AE038E017C03196981719F19491DA
:10FE30009923D1F7431720F0803210F08F3708F064
:10FE40002FE5822F81568A3108F42052FE01E30FFC
:10FE5000F11D20833F5F11968C91882311F08F3222
:10FE6000C1F6FB01B183A08390E08881803219F054
:10FE700091E001C090E0892FDF91CF9108958D30FE
:10FE800010F046E002C0482F4695249A2C9A279AF3
:10FE9000259A2698809164008B7F80936400242F9C
:10FEA00030E0C9019595879580658CBD40FF02C003
:10FEB00080E004C080E0463009F081E08DBD089507
:10FEC000FF920F931F93CF93DF938B010E9421C466
:10FED000EB01FF24FA9409C00E9421C46C1B7D0B26
:10FEE0006017710710F080E008C0FEBC0DB407FE7B
:10FEF000FDCF8EB58F3F81F781E0DF91CF911F91CC
:10FF00000F91FF9008950F931F938C01FC01828144
:10FF10000E943F7FF801808160E00E94D5C51F915B
:10FF20000F910895FF920F931F93DF93CF93CDB757
:10FF3000DEB72A970FB6F894DEBF0FBECDBF8C0197
:10FF4000F62E2F83388749875A870E94837FC801FE
:10FF50006CE271E00E94607FFE0137969E012F5F88
:10FF60003F4F86E0D9011D928A95E9F78F2D806475
:10FF7000898383818A8382818B8381818C838F8132
:10FF80008D83D901F90190E069E0AE014A5F5F4FCE
:10FF9000308120E0990F892F832787FD96272F5FD7
:10FFA000283011F0330FF6CF3196E417F50781F7BB
:10FFB000990F91609E839E01295F3F4F8C918EBD6A
:10FFC0000DB407FEFDCF1196A217B307B9F7BCE039
:10FFD000FB1631F48FEF8EBD0DB407FEFDCF8EB54D
:10FFE0009FEF2FEF2EBD0DB407FEFDCF8EB587FF1F
:10FFF00007C0992319F4F801838305C09150F2CF0B
:020000021000EC
:10000000D80113968C932A960FB6F894DEBF0FBED4
:10001000CDBFCF91DF911F910F91FF900895FC010B
:10002000808161E00E94D5C58FEF8EBD0DB407FEC3
:10003000FDCF0895CF93DF93EC010E94837FCE0123
:1000400068E572E00E94607F882389F08DEF8EBDA5
:100050000DB407FEFDCFCE0168E572E00E94607F1F
:10006000882329F0CE010E940F8081E006C082E142
:100070008983CE010E940F8080E0DF91CF910895A7
:10008000AF92BF92CF92DF92EF92FF920F931F93A6
:10009000CF93DF93EC015A016B017801890167E38B
:1000A00020E030E040E050E00E94927FCE0167E126
:1000B000A80197010E94927F882311F089E013C064
:1000C0008C81833039F0E9E0AA0CBB1CCC1CDD1C10
:1000D000EA95D1F7CE0169E1A60195010E94927FD0
:1000E000882339F087E08983CE010E940F8080E069
:1000F00004C0CE010E940F8081E0DF91CF911F915B
:100100000F91FF90EF90DF90CF90BF90AF90089548
:100110000F931F93CF93DF938C01EA0140E050E0EF
:10012000A0E0B0E0252F3327FE01EA0FFB1F8081FE
:1001300090E028273927220F331F275F374EF90118
:1001400085919491542F4427482759271196F2E01E
:10015000A030BF0739F76EBD0DB407FEFDCF888113
:100160008EBDE98182E090E00DB407FEFDCFEEBDCB
:1001700022E08030920731F0FE01E80FF91FE081A4
:100180000196F2CF0DB407FEFDCF5EBD0DB407FEA4
:10019000FDCF4EBD0DB407FEFDCF8FEF8EBD0DB46C
:1001A00007FEFDCF8EB5F80183838F71853011F482
:1001B00081E007C083E1F8018183C8010E940F80BC
:1001C00080E0DF91CF911F910F9108950F931F93BE
:1001D000CF93DF93EC018B010E94837FCE0168E512
:1001E00072E00E94607F882361F0CE016CEFA8016D
:1001F0000E948880882329F0CE010E940F8081E030
:1002000006C085E18983CE010E940F8080E0DF91E6
:10021000CF911F910F910895CF92DF92EF92FF92AD
:100220000F931F93CF93DF93EC017A018B01690148
:100230008C81833039F029E0EE0CFF1C001F111F68
:100240002A95D1F7CE0168E1A80197010E94927F1B
:10025000882311F086E023C0CE016EEFA6010E9434
:1002600088808823E9F0CE0168E572E00E94607F13
:10027000882311F487E113C0CE016DE020E030E067
:1002800040E050E00E94927F882341F48FEF8EBDC2
:100290000DB407FEFDCF8EB5882379F086E1898302
:1002A000CE010E940F8080E0DF91CF911F910F91CE
:1002B000FF90EF90DF90CF900895CE010E940F80C5
:1002C00081E0F2CF8091630F80FF3EC040915F0FCD
:1002D0005091600F6091610F7091620F8091680F73
:1002E0009091690F2FE53DE00E940C81882371F108
:1002F0008091630F81FF23C04091640F5091650F7F
:100300006091660F7091670F411551056105710588
:10031000B1F080915F0F9091600FA091610FB0914B
:10032000620F480F591F6A1F7B1F8091680F9091C1
:10033000690F2FE53DE00E940C81882339F0809100
:10034000630F8E7F8093630F81E0089580E00895AE
:10035000CF93DF93EC010E94837FCE016CE020E01D
:1003600030E040E050E00E94927F882339F083E043
:100370008983CE010E940F8080E004C0CE010E94DC
:100380000F8081E0DF91CF910895CF93DF93EC014F
:100390009A01AB018C81833039F069E0220F331F61
:1003A000441F551F6A95D1F7CE0162E10E94927FEA
:1003B000882339F085E08983CE010E940F8080E098
:1003C00004C0CE010E940F8081E0DF91CF9108959B
:1003D000BF92CF92DF92EF92FF920F931F93CF9332
:1003E000DF93EC016B017A010E9421C48B01BB24D5
:1003F000BA9409C00E9421C4601B710B6D527140F8
:1004000010F081E15FC0BEBC0DB407FEFDCF8EB51C
:100410008B838F3F79F38E3F11F08FE053C0D7016C
:100420001197E114F104D9F08FEF8EBD20E030E098
:100430009FEF0BC00DB407FEFDCF8EB5F601E20FA6
:10044000F31F80839EBD2F5F3F4F2A173B0790F31A
:100450000DB407FEFDCF8EB5AC0DBD1D8C931B8278
:100460008FEF8EBD0DB407FEFDCF3EB58FEF8EBD75
:100470000DB407FEFDCF2EB5A0E0B0E060E070E067
:1004800015C0472F5527F601EA0FFB1F808190E02A
:1004900048275927440F551F475F574EFA0185914A
:1004A0009491762F6627682779271196AE15BF0598
:1004B00040F3932F80E030E0822B932B8617970731
:1004C00039F08BE18983CE010E940F8080E004C067
:1004D000CE010E940F8081E0DF91CF911F910F919B
:1004E000FF90EF90DF90CF90BF900895EF92FF9232
:1004F0000F931F938C017B010E94837FC801B7017A
:1005000040E052E00E94E8811F910F91FF90EF9030
:100510000895CF92DF92EF92FF920F931F93CF93A4
:10052000DF93EC017A018B0169018C81833039F012
:1005300059E0EE0CFF1C001F111F5A95D1F7CE0198
:1005400061E1A80197010E94927F882339F084E03D
:100550008983CE010E940F8080E006C0CE01B601E3
:1005600040E052E00E94E881DF91CF911F910F910E
:10057000FF90EF90DF90CF900895DF92EF92FF927F
:100580000F931F937B018C01D42E80915F0F90916C
:10059000600FA091610FB091620F8E159F05A007AB
:1005A000B107E1F00E946281882311F1D2FC0CC0F6
:1005B0008091680F9091690FB801A7012FE53DE088
:1005C0000E9489828823A1F01092630FE0925F0F4E
:1005D000F092600F0093610F1093620F83E0D822B6
:1005E0008091630F8D298093630F2FE53DE002C05A
:1005F00020E030E0C9011F910F91FF90EF90DF9054
:1006000008956F927F928F929F92AF92BF92CF92F6
:10061000DF92EF92FF920F931F93CF93DF935C01D2
:10062000142F7093690F6093680FDC0157961C922A
:1006300082E090E0A0E0B0E0F50180839183A283A6
:10064000B3831092630F8FEF9FEFAFEFBFEF8093F5
:100650005F0F9093600FA093610FB093620F1092A1
:10066000640F1092650F1092660F1092670F44236B
:1006700021F466247724430144C0453008F022C1A8
:1006800060E070E080E090E040E00E94BD82EC011C
:10069000009709F417C1412F50E041505040FA0132
:1006A000B4E0EE0FFF1FBA95E1F7E80FF91FE2542F
:1006B000FE4F8081EE5BF14090E08F779070892B48
:1006C00009F000C1E653FE4F80819181A281B38180
:1006D00084369105A105B10508F4F4C0A4E0440FE7
:1006E000551FAA95E1F7C40FD51FCA53DE4F688086
:1006F00079808A809B80611471048104910409F4DB
:10070000E1C0C401B30140E00E94BD82EC0100974A
:1007100009F4D8C08B859C858050924009F0D2C0E6
:100720006889662309F4CEC0EE85FF85309709F409
:10073000C9C08D85882309F4C5C0D50152966C9334
:10074000529714968C9314971D961C9201E010E01A
:1007500008C04F5FD5011D964C934150483008F0BA
:10076000B1C0D5011D964C911D9714968C9190E0C7
:100770009801042E02C0220F331F0A94E2F7821759
:10078000930739F78E899F89009721F09C0140E0FB
:1007900050E004C02CA13DA14EA15FA1D50115964A
:1007A0002D933D934D935C93189752968C9188238B
:1007B00041F02093640F3093650F4093660F509380
:1007C000670F6F01EE24FF24C60CD71CE81CF91C30
:1007D000F501C38AD48AE58AF68A09891A89118FB4
:1007E000008F70E080E090E0258136814781508560
:1007F0000E948ECA6C0D7D1D8E1D9F1DD5015A96BF
:100800006D937D938D939C935D97F5E0000F111F81
:10081000FA95E1F701501E4F012F11270695980117
:1008200040E050E0260F371F481F591FF50126876B
:100830003787408B518B8B899C89009721F07C01F5
:1008400000E010E004C0E8A0F9A00AA11BA1C401C7
:10085000B301621B730B840B950B6E0D7F1D801F04
:10086000911FD5011D960C901D9704C096958795F4
:10087000779567950A94D2F7F50161877287838728
:100880009487653FFFE07F07F0E08F07F0E09F0768
:1008900020F48CE057968C9315C0655F7F4F8040A5
:1008A000904018F480E1F5010AC08CA59DA5AEA585
:1008B000BFA5F501828F938FA48FB58F80E2878BC0
:1008C00081E001C080E0DF91CF911F910F91FF90F7
:1008D000EF90DF90CF90BF90AF909F908F907F90E0
:1008E0006F90089542600E94BD8208958F929F92FA
:1008F000AF92BF92CF92DF92EF92FF920F931F932E
:10090000CF93DF93EC016A017B014801590142302A
:1009100051056105710508F44BC089859A85AB8541
:10092000BC850196A11DB11D84179507A607B707C1
:1009300008F43EC08F89803129F4252F362F472FA8
:1009400055270BC08032A1F59A01AB0197E056956F
:100950004795379527959A95D1F78B899C89AD89CD
:10096000BE89280F391F4A1F5B1FCA01B90141E028
:100970000E9472849C010097D9F08F89803149F4DC
:10098000F601F070EE0FFF1FE20FF31F91828082DD
:100990000DC0F601EF77F070EE0FFF1FEE0FFF1F97
:1009A000E20FF31F80829182A282B38281E001C0B4
:1009B00080E0DF91CF911F910F91FF90EF90DF903A
:1009C000CF90BF90AF909F908F900895CF92DF927D
:1009D000EF92FF920F931F93CF93DF93EC017A0175
:1009E0008B016901423051056105710508F453C05E
:1009F00089859A85AB85BC850196A11DB11D84179B
:100A00009507A607B70708F446C08F89803129F4F7
:100A10005527412F302F2F2D0BC08032E1F59A0141
:100A2000AB0167E056954795379527956A95D1F7BD
:100A30008B899C89AD89BE89280F391F4A1F5B1F8E
:100A4000CA01B90140E00E9472849C01009719F12B
:100A50008F89803159F4F701F070EE0FFF1FE20F1C
:100A6000F31F80819181A0E0B0E00EC0F701EF7725
:100A7000F070EE0FFF1FEE0FFF1FE20FF31F8081DC
:100A80009181A281B381BF70F60180839183A2839B
:100A9000B38381E001C080E0DF91CF911F910F917E
:100AA000FF90EF90DF90CF900895AF92BF92CF92DA
:100AB000DF92EF92FF920F931F93DF93CF9300D0BB
:100AC00000D0CDB7DEB76C017A018B0182E090E0F7
:100AD000A0E0B0E0F60180839183A283B3835E013E
:100AE0000894A11CB11CC601B801A70195010E9480
:100AF000E684882341F1C601B801A70100E010E0B7
:100B000020E030E00E9476848823E9F0E980FA80D2
:100B10000B811C81F6018789803151F4F8EFEF16C3
:100B2000FFEFFF06F0E00F07F0E01F07E0F209C05B
:100B300088EFE8168FEFF8068FEF08078FE01807A9
:100B400090F281E001C080E00F900F900F900F9025
:100B5000CF91DF911F910F91FF90EF90DF90CF9099
:100B6000BF90AF9008952F923F924F925F926F92F5
:100B70007F928F929F92AF92BF92CF92DF92EF922D
:100B8000FF920F931F93DF93CF93CDB7DEB72F97CD
:100B90000FB6F894DEBF0FBECDBF1C014A875B873E
:100BA0006C877D873F872E87DC0119968D919D91FB
:100BB0000D90BC91A02D0196A11DB11D8E839F8328
:100BC000A887B987F901008111812281338101153C
:100BD00011052105310549F0480159010894811C8E
:100BE000911CA11CB11C1D8210C0D1018D909D9043
:100BF000AD90BC901D828A859B85AC85BD85019793
:100C0000A105B10511F491E09D83750164014424AF
:100C1000552432018E010F5F1F4FF10181859285AE
:100C2000A385B485481659066A067B0608F090C06D
:100C30008E819F81A885B9858C159D05AE05BF0560
:100C400050F4F2E08F2E912CA12CB12CE2E0CE2EAC
:100C5000D12CE12CF12CC101B701A60198010E9411
:100C6000E684882309F474C089819A81AB81BC81B0
:100C7000A70196012F5F3F4F4F4F5F4F0097A10590
:100C8000B10519F049015A010DC0281939094A095D
:100C90005B098A859B85AC85BD85281739074A077E
:100CA0005B0759F00894411C511C611C711C08948D
:100CB000C11CD11CE11CF11CB0CFC101A601B701C0
:100CC0000FEF1FEF2FEF3FE00E947684882399F407
:100CD0003FC0260137010894410851086108710896
:100CE000C101B301A201970186010E947684882385
:100CF00079F1730162018C149D04AE04BF0448F3C2
:100D0000AE85BF854D915D916D917C9141155105E9
:100D10006105710539F0C101950184010E94768455
:100D20008823B1F0EE85FF8580829182A282B38212
:100D3000FD81FF2359F00894811C911CA11CB11C5A
:100D4000D1018D929D92AD92BC92139781E001C02A
:100D500080E02F960FB6F894DEBF0FBECDBFCF91C7
:100D6000DF911F910F91FF90EF90DF90CF90BF9098
:100D7000AF909F908F907F906F905F904F903F903B
:100D80002F900895CF93DF93EC019C01295F3F4F93
:100D90008D819E8141E050E060E070E00E94B3856B
:100DA0008823A1F08F89988DA98DBA8D0097A10510
:100DB000B10559F48F819885A985BA858F8B988F55
:100DC000A98FBA8F89818068898381E0DF91CF9173
:100DD0000895CF92DF92EF92FF920F931F93DF93CC
:100DE000CF9300D000D0CDB7DEB77C01FC0187895E
:100DF000908DA18DB28D89839A83AB83BC8300E0F3
:100E000010E06E010894C11CD11C49815A816B818C
:100E10007C81D70115968D919C91169796010E9421
:100E2000E684882379F1D7011596ED91FC91169708
:100E30008481080F111DB0E100301B0718F52981CE
:100E40003A814B815C818789803131F4285F3F4F43
:100E500040405040D0F205C0285F3F4F4F4F5F40A9
:100E6000A0F2C801A0E0B0E019E0880F991FAA1F06
:100E7000BB1F1A95D1F7F701838B948BA58BB68B8B
:100E800081E001C080E00F900F900F900F90CF9104
:100E9000DF911F910F91FF90EF90DF90CF90089519
:100EA000CF93DF93EC01FB018B818823D1F57E8307
:100EB0006D8387898031C9F582E08B831F8A188E04
:100EC000198E1A8E808D918DA0E0B0E025E0880FFC
:100ED000991FAA1FBB1F2A95D1F78B8B9C8BAD8BBB
:100EE000BE8B0FC083E08B83828D938DA48DB58DD7
:100EF0008F8B988FA98FBA8FCE010E94E9868823A5
:100F000081F081E089831F82188619861A861B86E4
:100F10001C861D861E861F86188A198A1A8A1C82BC
:100F200001C080E0DF91CF9108958032D1F7DACF10
:100F30006F927F928F929F92AF92BF92CF92DF92E9
:100F4000EF92FF920F931F93CF93DF93EC017A01FF
:100F50008B012B81222309F489C08B899C89AD895F
:100F6000BE8984179507A607B70708F47FC08EC00F
:100F7000EB86FC860D871E871F82188619861A86C7
:100F80000DC0E114F1040105110551F41F8218860A
:100F900019861A861B861C861D861E8681E067C000
:100FA0002B853C854D855E85ED81FE81858590E0B4
:100FB0000996215030404040504039014A01082EE6
:100FC00004C096948794779467940A94D2F72F5F1D
:100FD0003F4F4F4F5F4F0894E108F1080109110995
:100FE0005701680104C0D694C794B794A7948A9512
:100FF000D2F70894E11CF11C011D111DA614B704C1
:10100000C804D90428F0211531054105510549F4DA
:101010008F89988DA98DBA8D8F839887A987BA8774
:1010200016C0A618B708C808D90811C04F8158853E
:1010300069857A858D819E8194010E94E684089459
:10104000A108B108C108D108882331F40FC037E0E6
:10105000832E912C8C0E9D1EA114B104C104D104C9
:1010600029F7EB86FC860D871E8798CF80E0DF91FD
:10107000CF911F910F91FF90EF90DF90CF90BF9095
:10108000AF909F908F907F906F900895223009F0DD
:1010900078CF6ECFCF93DF93EC01462F6F857889A1
:1010A00089899A890E94BD82AC01009719F420E0D9
:1010B00030E00AC08C81282F30E065E0220F331F1A
:1010C0006A95E1F7240F351FC901DF91CF9108958B
:1010D0000F931F93CF93DF938C01FC0183818823AF
:1010E000F1F1818187FF38C0C80161E00E944A8820
:1010F000EC010097A1F18881853E89F1F801838197
:10110000823040F483899489A589B6898C8F9D8F1C
:10111000AE8FBF8FF8018789908D9B8F8A8F8789CB
:10112000908DA18DB28DCD01AA27BB279D8B8C8B75
:10113000E0915D0DF0915E0D309751F0BE016A5E59
:101140007F4FCE0148960995888D998D9B8B8A8B10
:10115000F80181818F7781830E94628104C081E0E0
:10116000F801808380E0DF91CF911F910F91089566
:101170006F927F928F929F92AF92BF92CF92DF92A7
:10118000EF92FF920F931F93DF93CF9300D000D085
:10119000CDB7DEB77C015A016B01DC0113968C914F
:1011A0001397813009F091C011968C9181FF8DC009
:1011B000A0C00097A105B10511F481E087C0F70137
:1011C0006384748485849684C701B601A5010E9456
:1011D0009887882309F479C0D70115968D919C9141
:1011E0001697A114B104C104D10489F457964D9106
:1011F0005D916D917C915A970E945585882309F4E1
:1012000064C0F701178A108E118E128E44C0D70168
:1012100017964D915D916D917C911A979E012F5F6C
:101220003F4F0E94E684882309F44FC0D7011596EA
:10123000ED91FC91169749815A816B817C81878958
:10124000803149F4483FBFEF5B07B0E06B07B0E087
:101250007B0748F020C0483F8FEF58078FEF6807A3
:101260008FE07807C0F4CF010E945585882369F18B
:10127000D70117964D915D916D917C911A971596B6
:101280008D919C9116970FEF1FEF2FEF3FE00E947B
:1012900076848823D1F0F701A38AB48AC58AD68AD6
:1012A000818180688183C7010E946888882369F0F2
:1012B000B601A5016A147B048C049D0410F4B401EA
:1012C000A301C7010E94988701C080E00F900F9092
:1012D0000F900F90CF91DF911F910F91FF90EF90A2
:1012E000DF90CF90BF90AF909F908F907F906F9046
:1012F0000895F70183899489A589B689841795078C
:10130000A607B70708F055CFE0CF1F93CF93DF9321
:10131000EC01142FE62FF0E080915F0F9091600FA9
:10132000A091610FB091620F8F87988BA98BBA8BB8
:101330006C83B5E0EE0FFF1FBA95E1F7E15AF24F6B
:101340002489358940E050E0A901332722272F8BDB
:10135000388F498F5A8F828D938DA0E0B0E0282B73
:10136000392B4A2B5B2B2F8B388F498F5A8F8385D4
:1013700090E088719070009751F4848D958DA68DC2
:10138000B78D8B8B9C8BAD8BBE8B81E00CC0409757
:1013900051F5CE010E94E986882321F41B8A1C8A1C
:1013A0001D8A1E8A84E08B83812F8F7089831F8220
:1013B000188619861A861B861C861D861E8614FFB3
:1013C00018C0CE0140E050E060E070E00E94B888B4
:1013D000882379F408C04B895C896D897E89CE01A8
:1013E0000E94988702C01B8280E0DF91CF911F91FD
:1013F000089515FDF0CF81E0F8CF0F931F938C0176
:101400000E946888F80113821F910F910895CF936D
:10141000DF93EC01662331F0A396D0935C0DC0936B
:101420005B0DA3978EA1882321F0CE0183960E94A5
:10143000FD89CE0183962596BE010E945087DF91DB
:10144000CF910895CF93DF93EC0140E050E060E04E
:1014500070E00E94B888882369F0CE0161E00E94A4
:101460004A88FC01009731F085EE80831B820E9440
:10147000628101C080E0DF91CF910895BF92CF9249
:10148000DF92EF92FF920F931F93CF93DF93EC01C4
:10149000B62E1C82198248830E9421C46B01888168
:1014A00061E00E9458C5888161E00E94D5C52698F8
:1014B000259A279A089A8BE08A830E943F7F80E0D2
:1014C0009FEF9EBD0DB407FEFDCF8F5F8A30C9F739
:1014D00009C00E9421C46C197D09615D774010F03C
:1014E00081E06FC0CE0160E020E030E040E050E0FD
:1014F0000E94927F813069F7CE016BE321E030E0FA
:1015000040E050E00E94927F813011F08AE159C0A2
:101510001FEFCE0168E02AEA31E040E050E00E948F
:10152000927F853011F481E00DC080E01EBD0DB4C6
:1015300007FEFDCF9EB58F5F8430C1F79B839A3A3B
:1015400031F482E08C838C81823051F40DC00E9492
:1015500021C46C197D09615D7740D8F282E031C009
:10156000EE24FF2487010FC0E12CF12C012D60E453
:10157000162F09C00E9421C46C197D09615D774056
:1015800010F08AE01EC0CE0167E320E030E040E0CA
:1015900050E00E94927FCE0169E2A80197010E946B
:1015A000927F882339F78C81823029F5CE016AE356
:1015B00020E030E040E050E00E94927F882331F04C
:1015C00088E08983CE010E940F8021C08FEF8EBDFD
:1015D0000DB407FEFDCF8EB5807C803C11F483E016
:1015E0008C8380E09FEF9EBD0DB407FEFDCF2EB52E
:1015F0008F5F8330C1F7CE010E940F808EE08B1584
:1016000018F488E1898303C0BA8281E001C080E0D8
:10161000DF91CF911F910F91FF90EF90DF90CF90CE
:10162000BF9008950F931F93CF93DF93EC01262F64
:10163000642F422F0E943E8A8823C9F08E010B5FDF
:101640001F4FC801BE0141E00E940183882339F485
:10165000C801BE0140E00E940183882341F0CE0111
:1016600061E00E94078A882319F081E001C080E0D0
:10167000DF91CF911F910F9108953F924F925F920A
:101680006F927F928F929F92AF92BF92CF92DF9292
:10169000EF92FF920F931F93DF93CF93CDB7DEB7F7
:1016A0002A970FB6F894DEBF0FBECDBF3C01162FB0
:1016B000072F5A874987DC0111968C91119781FF7A
:1016C000FAC182FF17C053964D915D916D917C9147
:1016D00056971B968D919D910D90BC91A02D8417CE
:1016E0009507A607B70731F0C3010E9498878823A2
:1016F00009F4E1C1812F902F9C0138872F83E98560
:10170000FA85FE83ED839BC1D3011596ED91FC9183
:101710001697DA01C90119E0B695A79597958795AF
:101720001A95D1F794809A949822AFEFAA2EA1E04F
:10173000BA2EA222B322992009F052C0A114B104FA
:1017400009F04EC0D30117964D915D916D917C913A
:101750001A97411551056105710571F1CF019E017F
:101760002F5F3F4F0E94E684882309F4A4C129819A
:101770003A814B815C81D3011596ED91FC911697CE
:101780008789803149F4283FBFEF3B07B0E04B0722
:10179000B0E05B0748F019C0283FEFEF3E07EFEFDE
:1017A0004E07EFE05E0788F4D30117962D933D9323
:1017B0004D935C931A9714C0F3018789908DA18D86
:1017C000B28D0097A105B10531F4C3010E94C28614
:1017D000882331F470C1F30187839087A187B28792
:1017E000D30113968C91139715960D911C91169712
:1017F0008230B9F41B96CD90DD90ED90FC901E9751
:10180000E9E0F694E794D794C794EA95D1F7F80104
:10181000828D938DA48DB58DC80ED91EEA1EFB1E38
:1018200020C0D80114966C9170E080E090E0F30144
:1018300027813085418552852250304040405040BC
:101840000E948ECA6B017C01F80186859785A0896C
:10185000B189C80ED91EEA1EFB1EC90CD11CE11CA1
:10186000F11CA114B104C9F42D813E8120503240F5
:10187000E8F5D3011B962D913D914D915C911E97FA
:1018800053968D919D910D90BC91A02D28173907ED
:101890004A075B0710F045E001C041E0C701B6010F
:1018A0000E94BD82009709F406C140E052E04A1947
:1018B0005B094D805E804415550508F42A019C01A2
:1018C0002A0D3B1DC9016F817885A2010E94A818CD
:1018D000A40CB51CB0E0AB16B2E0BB0609F093C097
:1018E0000E946281882309F08EC0E5C0ED81FE81EF
:1018F000E050F44060F580915F0F9091600FA091EF
:10190000610FB091620F8C159D05AE05BF0571F496
:101910008FEF9FEFAFEFBFEF80935F0F9093600F5C
:10192000A093610FB093620F1092630F8091680FC4
:101930009091690FB701A6012F8138850E940C8113
:10194000882309F4B8C0412C72E0572E5CC0D30143
:101950001596ED91FC911697848189193E803694F5
:10196000831508F4382E032D10E020E030E080913C
:10197000680F9091690FB701A6010E9440808823EB
:1019800009F499C00F811885460157012CC0809138
:101990005F0F9091600FA091610FB091620F881658
:1019A0009906AA06BB0671F48FEF9FEFAFEFBFEF6A
:1019B00080935F0F9093600FA093610FB093620FBD
:1019C0001092630F8091680F9091690FB8010E9487
:1019D000E68000501E4F0894811C911CA11CB11C74
:1019E000882309F468C0882D8C19831580F28091B2
:1019F000680F9091690F0E941A80882309F45BC0D8
:101A0000532C550C4424920140E050E0F3018385AF
:101A10009485A585B685820F931FA41FB51F838764
:101A20009487A587B6872F813885240D351D388783
:101A30002F838D819E81841995099E838D83D30187
:101A40001B962D913D914D915C911E97ED81FE81EC
:101A5000EF2B09F059CE53968D919D910D90BC912D
:101A6000A02D82179307A407B50740F4D30153961E
:101A70002D933D934D935C9356970BC080915D0DD4
:101A800090915E0D892B59F0E985FA85EF2B39F09D
:101A9000D30111968C911197806811968C93F30164
:101AA000818183FF05C0C3010E946888882319F0E3
:101AB00049855A8505C081E0D3018C934FEF5FEFD4
:101AC000CA012A960FB6F894DEBF0FBECDBFCF91E4
:101AD000DF911F910F91FF90EF90DF90CF90BF901B
:101AE000AF909F908F907F906F905F904F903F90BE
:101AF00008950E943D8B08953F924F925F926F929E
:101B00007F928F929F92AF92BF92CF92DF92EF928D
:101B1000FF920F931F93DF93CF93CDB7DEB72A9732
:101B20000FB6F894DEBF0FBECDBF3C0158874F8380
:101B3000DC0113968C911397882309F439C111960F
:101B40008C9180FF35C14FC1F401EC19FD09F88774
:101B5000EF837C836B839301295F3F4F3E832D830B
:101B60008F8198859A8389831BC1D3011B962D9100
:101B70003D914D915C911E97F901F170FA87E987CB
:101B80001596ED91FC91169749015A0119E0B6940A
:101B9000A794979487941A95D1F734803A94382073
:101BA00013968C91823049F4C28CD38CE48CF58CE2
:101BB000C80CD91CEA1CFB1C46C089859A85892B58
:101BC00001F53320F1F4211531054105510551F49A
:101BD000F3018789908DA18DB28D87839087A1872E
:101BE000B2870FC0D30117964D915D916D917C9195
:101BF0001A97CF012D813E810E94E684882309F443
:101C0000D7C0F30105811681D80114966C9170E05C
